******************************************************************************
               TMS320C6x Linker PC v7.4.21                     
******************************************************************************
>> Linked Wed Sep 06 17:42:40 2017

OUTPUT FILE NAME:   <TMS320C6678_main_with_arguments.out>
ENTRY POINT SYMBOL: "_c_int00"  address: 8f006000


MEMORY CONFIGURATION

         name            origin    length      used     unused   attr    fill
----------------------  --------  ---------  --------  --------  ----  --------
  L2SRAM                00800000   00019f00  00012814  000076ec  RW X
  L2HEAP                00819f00   00046100  00000000  00046100  RW X
  L1PSRAM               00e00000   00008000  00000000  00008000  RW X
  L1DSRAM               00f00000   00008000  00000000  00008000  RW  
  MSMCSRAM              0c000000   00400000  00395a80  0006a580  RW X
  DDRUNCACHED           80000000   00fffe00  00000000  00fffe00  RW X
  IBL_VERSIONS          80fffe00   00000100  00000000  00000100  RW  
  DDR                   81000000   0f3c0000  0e00704e  013b8fb2  RW X
  DDRCINE               903c0000   0fc40000  0fc40000  00000000  RW X


SEGMENT ALLOCATION MAP

run origin  load origin   length   init length attrs members
----------  ----------- ---------- ----------- ----- -------
00800000    00800000    00010f68   00000000    rw-
  00800000    00800000    0000fe48   00000000    rw- .far
  0080fe48    0080fe48    00000120   00000000    rw- .cio
  0080ff68    0080ff68    00001000   00000000    rw- .stack
00810f68    00810f68    000018ac   000018ac    rw-
  00810f68    00810f68    000018a4   000018a4    rw- .fardata
  0081280c    0081280c    00000008   00000008    rw- .neardata
0c380000    0c380000    00015880   00015880    r-x
  0c380000    0c380000    00015880   00015880    r-x .text
0c395c00    0c395c00    00000200   00000200    r-x
  0c395c00    0c395c00    00000200   00000200    r-x .vecs
8f000000    8f000000    00005126   00005126    r--
  8f000000    8f000000    00005126   00005126    r-- .const
8f005140    8f005140    00000c00   00000c00    r-x
  8f005140    8f005140    00000c00   00000c00    r-x .sysbios
8f006000    8f006000    00001328   00001328    r-x
  8f006000    8f006000    00000400   00000400    r-x boot
  8f006400    8f006400    00000f28   00000f28    r-- .cinit
903c0000    903c0000    0fc40000   00000000    rw-
  903c0000    903c0000    0fc40000   00000000    rw- .sect_cine_data


SECTION ALLOCATION MAP

 output                                  attributes/
section   page    origin      length       input sections
--------  ----  ----------  ----------   ----------------
.init_array 
*          0    00800000    00000000     UNINITIALIZED

xdc.meta   0    00800000    000000f8     COPY SECTION
                  00800000    000000f8     EVM_C6674_configuration_pe66.oe66 (xdc.meta)

.far       0    00800000    0000fe48     UNINITIALIZED
                  00800000    0000f500     EVM_C6674_configuration_pe66.oe66 (.far)
                  0080f500    00000800     EVM_C6674_configuration_pe66.oe66 (.far:taskStackSection)
                  0080fd00    00000140     rts6600_elf.lib : defs.obj (.far)
                  0080fe40    00000008                     : trgdrv.obj (.far)

.cio       0    0080fe48    00000120     UNINITIALIZED
                  0080fe48    00000120     rts6600_elf.lib : trgmsg.obj (.cio)

.sysmem    0    0080ff68    00000000     UNINITIALIZED

.bss       0    0080ff68    00000000     UNINITIALIZED

.pinit     0    0080ff68    00000000     UNINITIALIZED

.switch    0    0080ff68    00000000     UNINITIALIZED

.data      0    0080ff68    00000000     UNINITIALIZED

.stack     0    0080ff68    00001000     UNINITIALIZED
                  0080ff68    00000008     boot.ae66 : boot.oe66 (.stack)
                  0080ff70    00000ff8     --HOLE--

.sect_LL2 
*          0    00810f68    00000000     UNINITIALIZED

.sect_doppler_data_LL2 
*          0    00810f68    00000000     UNINITIALIZED

.args      0    00810f68    00000000     UNINITIALIZED

.fardata   0    00810f68    000018a4     
                  00810f68    00000500     EVM_C6674_configuration_pe66.oe66 (.fardata:ti_sysbios_family_c66_tci66xx_CpIntc_Module_State_0_dispatchTab__A)
                  00811468    00000488     EVM_C6674_configuration_pe66.oe66 (.fardata)
                  008118f0    000001e0     rts6600_elf.lib : defs.obj (.fardata:_ftable)
                  00811ad0    00000180     EVM_C6674_configuration_pe66.oe66 (.fardata:ti_sysbios_timers_timer64_Timer_Module_State_0_device__A)
                  00811c50    0000012c     EVM_C6674_configuration_pe66.oe66 (.fardata:ti_sdo_utils_NameServer_Object__table__V)
                  00811d7c    00000004     rts6600_elf.lib : defs.obj (.fardata)
                  00811d80    000000a8     EVM_C6674_configuration_pe66.oe66 (.fardata:ti_sysbios_heaps_HeapMem_Object__table__V)
                  00811e28    000000a0     rts6600_elf.lib : lowlev.obj (.fardata:_stream)
                  00811ec8    000000a0     EVM_C6674_configuration_pe66.oe66 (.fardata:ti_sdo_ipc_Ipc_Module_State_0_procEntry__A)
                  00811f68    0000009c     EVM_C6674_configuration_pe66.oe66 (.fardata:ti_uia_loggers_LoggerStopMode_Object__table__V)
                  00812004    00000004     --HOLE--
                  00812008    00000098     EVM_C6674_configuration_pe66.oe66 (.fardata:ti_sysbios_family_c66_tci66xx_CpIntc_Module_State_0_hostIntToSysInt__A)
                  008120a0    00000090     EVM_C6674_configuration_pe66.oe66 (.fardata:ti_sdo_ipc_SharedRegion_Module_State_0_regions__A)
                  00812130    00000080     EVM_C6674_configuration_pe66.oe66 (.fardata:ti_sdo_ipc_GateMP_Module_State_0_remoteSystemGates__A)
                  008121b0    00000080     EVM_C6674_configuration_pe66.oe66 (.fardata:ti_sysbios_knl_Swi_Module_State_0_readyQ__A)
                  00812230    00000080     EVM_C6674_configuration_pe66.oe66 (.fardata:ti_sysbios_knl_Task_Module_State_0_readyQ__A)
                  008122b0    00000080     EVM_C6674_configuration_pe66.oe66 (.fardata:ti_sysbios_timers_timer64_Timer_Module_State_0_gctrl__A)
                  00812330    00000080     EVM_C6674_configuration_pe66.oe66 (.fardata:ti_sysbios_timers_timer64_Timer_Module_State_0_handles__A)
                  008123b0    00000080     EVM_C6674_configuration_pe66.oe66 (.fardata:ti_sysbios_timers_timer64_Timer_Module_State_0_intFreqs__A)
                  00812430    00000078     rts6600_elf.lib : lowlev.obj (.fardata:_device)
                  008124a8    00000050     EVM_C6674_configuration_pe66.oe66 (.fardata:ti_sysbios_knl_Task_Object__table__V)
                  008124f8    00000050     EVM_C6674_configuration_pe66.oe66 (.fardata:ti_sysbios_timers_timer64_Timer_Object__table__V)
                  00812548    00000040     EVM_C6674_configuration_pe66.oe66 (.fardata:ti_sdo_ipc_MessageQ_Module_State_0_transports__A)
                  00812588    00000040     EVM_C6674_configuration_pe66.oe66 (.fardata:ti_sysbios_gates_GateMutex_Object__table__V)
                  008125c8    00000030     EVM_C6674_configuration_pe66.oe66 (.fardata:ti_sysbios_knl_Swi_Object__table__V)
                  008125f8    00000024     EVM_C6674_configuration_pe66.oe66 (.fardata:xdc_runtime_LoggerBuf_Object__table__V)
                  0081261c    00000004     --HOLE--
                  00812620    00000020     EVM_C6674_configuration_pe66.oe66 (.fardata:ti_sdo_ipc_MessageQ_Module_State_0_heaps__A)
                  00812640    00000020     EVM_C6674_configuration_pe66.oe66 (.fardata:ti_sdo_ipc_Notify_Module_State_0_notifyHandles__A)
                  00812660    00000020     EVM_C6674_configuration_pe66.oe66 (.fardata:ti_sdo_ipc_family_c647x_Interrupt_Module_State_0_args__A)
                  00812680    00000020     EVM_C6674_configuration_pe66.oe66 (.fardata:ti_sdo_ipc_transports_TransportShmSetup_Module_State_0_handles__A)
                  008126a0    00000020     EVM_C6674_configuration_pe66.oe66 (.fardata:ti_sdo_utils_NameServer_Module_State_0_nsRemoteHandle__A)
                  008126c0    00000020     EVM_C6674_configuration_pe66.oe66 (.fardata:xdc_runtime_System_Module_State_0_atexitHandlers__A)
                  008126e0    0000001c     EVM_C6674_configuration_pe66.oe66 (.fardata:ti_sysbios_utils_Load_Module_State_0_taskEnv__A)
                  008126fc    00000004     --HOLE--
                  00812700    00000018     EVM_C6674_configuration_pe66.oe66 (.fardata:ti_sysbios_family_c64p_Hwi_Object__table__V)
                  00812718    00000018     EVM_C6674_configuration_pe66.oe66 (.fardata:ti_sysbios_gates_GateMutexPri_Object__table__V)
                  00812730    00000014     EVM_C6674_configuration_pe66.oe66 (.fardata:ti_sysbios_family_c66_tci66xx_CpIntc_Module_State_0_initSIER__A)
                  00812744    00000004     --HOLE--
                  00812748    00000010     EVM_C6674_configuration_pe66.oe66 (.fardata:ti_sdo_utils_MultiProc_Module_State_0_clusterProcList__A)
                  00812758    00000010     EVM_C6674_configuration_pe66.oe66 (.fardata:ti_sysbios_family_c66_tci66xx_CpIntc_Module_State_0_controller__A)
                  00812768    00000010     EVM_C6674_configuration_pe66.oe66 (.fardata:ti_sysbios_gates_GateAll_Object__table__V)
                  00812778    0000000c     rts6600_elf.lib : exit.obj (.fardata)
                  00812784    00000004     --HOLE--
                  00812788    0000000c     EVM_C6674_configuration_pe66.oe66 (.fardata:ti_sysbios_gates_GateSwi_Object__table__V)
                  00812794    00000008     rts6600_elf.lib : _lock.obj (.fardata)
                  0081279c    00000004     --HOLE--
                  008127a0    00000008     EVM_C6674_configuration_pe66.oe66 (.fardata:ti_sysbios_hal_Hwi_Object__table__V)
                  008127a8    00000004     EVM_C6674_configuration_pe66.oe66 (.fardata:ti_sdo_ipc_Notify_Module_State_0_notifyHandles_0__A)
                  008127ac    00000004     --HOLE--
                  008127b0    00000004     EVM_C6674_configuration_pe66.oe66 (.fardata:ti_sdo_ipc_Notify_Module_State_0_notifyHandles_1__A)
                  008127b4    00000004     --HOLE--
                  008127b8    00000004     EVM_C6674_configuration_pe66.oe66 (.fardata:ti_sdo_ipc_Notify_Module_State_0_notifyHandles_2__A)
                  008127bc    00000004     --HOLE--
                  008127c0    00000004     EVM_C6674_configuration_pe66.oe66 (.fardata:ti_sdo_ipc_Notify_Module_State_0_notifyHandles_3__A)
                  008127c4    00000004     --HOLE--
                  008127c8    00000004     EVM_C6674_configuration_pe66.oe66 (.fardata:ti_sdo_ipc_Notify_Module_State_0_notifyHandles_4__A)
                  008127cc    00000004     --HOLE--
                  008127d0    00000004     EVM_C6674_configuration_pe66.oe66 (.fardata:ti_sdo_ipc_Notify_Module_State_0_notifyHandles_5__A)
                  008127d4    00000004     --HOLE--
                  008127d8    00000004     EVM_C6674_configuration_pe66.oe66 (.fardata:ti_sdo_ipc_Notify_Module_State_0_notifyHandles_6__A)
                  008127dc    00000004     --HOLE--
                  008127e0    00000004     EVM_C6674_configuration_pe66.oe66 (.fardata:ti_sdo_ipc_Notify_Module_State_0_notifyHandles_7__A)
                  008127e4    00000004     --HOLE--
                  008127e8    00000004     EVM_C6674_configuration_pe66.oe66 (.fardata:ti_sysbios_gates_GateHwi_Object__table__V)
                  008127ec    00000004     --HOLE--
                  008127f0    00000004     EVM_C6674_configuration_pe66.oe66 (.fardata:ti_sysbios_knl_Task_Module_State_0_idleTask__A)
                  008127f4    00000004     --HOLE--
                  008127f8    00000004     EVM_C6674_configuration_pe66.oe66 (.fardata:ti_sysbios_utils_Load_Module_State_0_runningTask__A)
                  008127fc    00000004     --HOLE--
                  00812800    00000004     EVM_C6674_configuration_pe66.oe66 (.fardata:ti_sysbios_utils_Load_Module_State_0_taskStartTime__A)
                  00812804    00000004     --HOLE--
                  00812808    00000004     EVM_C6674_configuration_pe66.oe66 (.fardata:xdc_runtime_GateNull_Object__table__V)

.bss       0    0081280c    00000000     UNINITIALIZED

.neardata 
*          0    0081280c    00000008     
                  0081280c    00000008     ti.uia.runtime.ae66 : QueueDescriptor.oe66 (.neardata)

.rodata    0    00812814    00000000     UNINITIALIZED

ti.sdo.ipc.SharedRegion_0 
*          0    0c000000    00010000     NOLOAD SECTION
                  0c000000    00010000     --HOLE--

ti.sdo.ipc.SharedRegion_3 
*          0    0c010000    00370000     NOLOAD SECTION
                  0c010000    00370000     --HOLE--

.text      0    0c380000    00015880     
                  0c380000    00000880     ti.targets.rts6000.ae66 : System.oe66 (.text:xdc_runtime_System_doPrint__I)
                  0c380880    00000780     sysbios.ae66 : BIOS.obj (.text:ti_sysbios_family_c64p_Exception_handler__I)
                  0c381000    00000760                  : BIOS.obj (.text:ti_sysbios_knl_Semaphore_pend__E)
                  0c381760    000006a0                  : BIOS.obj (.text:ti_sysbios_timers_timer64_Timer_Module_startup__E)
                  0c381e00    00000620                  : BIOS.obj (.text:ti_sysbios_heaps_HeapMem_allocUnprotected__E)
                  0c382420    000005c0     rts6600_elf.lib : divd.obj (.text:__c6xabi_divd)
                  0c3829e0    000005c0                     : _printfi.obj (.text:_getarg_diouxp)
                  0c382fa0    000005c0     sysbios.ae66 : BIOS.obj (.text:ti_sysbios_heaps_HeapMem_freeUnprotected__E)
                  0c383560    00000520     rts6600_elf.lib : _printfi.obj (.text:_setfield)
                  0c383a80    00000480     sysbios.ae66 : BIOS.obj (.text:ti_sysbios_knl_Task_Module_startup__E)
                  0c383f00    00000460     rts6600_elf.lib : _printfi.obj (.text:_printfi)
                  0c384360    00000400     sysbios.ae66 : BIOS.obj (.text:ti_sysbios_gates_GateMutexPri_enter__E)
                  0c384760    000003e0     ipc.ae66 : Ipc.obj (.text:ti_sdo_ipc_Notify_Instance_init__E)
                  0c384b40    000003e0     sysbios.ae66 : BIOS.obj (.text:ti_sysbios_knl_Task_setPri__E)
                  0c384f20    000003a0     rts6600_elf.lib : fputs.obj (.text:fputs)
                  0c3852c0    000003a0     sysbios.ae66 : BIOS.obj (.text:ti_sysbios_family_c66_Cache_startup__I)
                  0c385660    00000360                  : BIOS.obj (.text:ti_sysbios_family_c64p_Hwi_dispatchCore__I)
                  0c3859c0    00000340     rts6600_elf.lib : _printfi.obj (.text:fcvt)
                  0c385d00    00000340     sysbios.ae66 : BIOS.obj (.text:ti_sysbios_utils_Load_logLoads__I)
                  0c386040    00000320     rts6600_elf.lib : _printfi.obj (.text:_pproc_fge)
                  0c386360    00000320                     : _printfi.obj (.text:ecvt)
                  0c386680    00000300     sysbios.ae66 : BIOS.obj (.text:ti_sysbios_knl_Swi_run__I)
                  0c386980    00000300                  : BIOS.obj (.text:ti_sysbios_timers_timer64_Timer_deviceConfig__I)
                  0c386c80    000002e0     ipc.ae66 : Ipc.obj (.text:SharedRegion_getEntry)
                  0c386f60    000002e0     rts6600_elf.lib : _printfi.obj (.text:_pproc_fwp)
                  0c387240    000002e0     sysbios.ae66 : BIOS.obj (.text:ti_sysbios_heaps_HeapMem_Instance_init__E)
                  0c387520    000002c0     rts6600_elf.lib : _printfi.obj (.text:_pconv_e)
                  0c3877e0    000002c0     sysbios.ae66 : BIOS.obj (.text:ti_sysbios_family_c66_tci66xx_CpIntc_Module_startup__E)
                  0c387aa0    000002a0                  : BIOS.obj (.text:ti_sysbios_family_c64p_Hwi_Module_startup__E)
                  0c387d40    000002a0                  : BIOS.obj (.text:ti_sysbios_knl_Clock_workFunc__E)
                  0c387fe0    00000260                  : BIOS.obj (.text:ti_sysbios_knl_Swi_Module_startup__E)
                  0c388240    00000260                  : BIOS.obj (.text:ti_sysbios_utils_Load_updateThreadContexts__E)
                  0c3884a0    00000260     EVM_C6674_configuration_pe66.oe66 (.text:xdc_runtime_System_printfExtend__I)
                  0c388700    00000240     rts6600_elf.lib : imath64.obj (.text:__c6xabi_divull)
                  0c388940    00000240                     : _printfi.obj (.text:_pproc_diouxp)
                  0c388b80    00000240     sysbios.ae66 : BIOS.obj (.text:ti_sysbios_family_c64p_Exception_internalHandler__I)
                  0c388dc0    00000240                  : BIOS.obj (.text:ti_sysbios_knl_Semaphore_post__E)
                  0c389000    00000240     EVM_C6674_configuration_pe66.oe66 (.text:ti_uia_loggers_LoggerStopMode_writeMemoryRange__E)
                  0c389240    00000220     rts6600_elf.lib : _printfi.obj (.text:_pproc_str)
                  0c389460    00000220                     : fputc.obj (.text:fputc)
                  0c389680    00000220     sysbios.ae66 : BIOS.obj (.text:ti_sysbios_knl_Task_schedule__I)
                  0c3898a0    00000220                  : BIOS.obj (.text:ti_sysbios_timers_timer64_Timer_setPeriodMicroSecs__E)
                  0c389ac0    00000220     ti.targets.rts6000.ae66 : Core-mem.oe66 (.text:xdc_runtime_Core_createObject__I)
                  0c389ce0    00000200     ipc.ae66 : Ipc.obj (.text:MultiProc_getId)
                  0c389ee0    00000200     rts6600_elf.lib : _printfi.obj (.text:_pconv_g)
                  0c38a0e0    00000200     sysbios.ae66 : c64p_Hwi_disp_always.obj (.text:_ti_sysbios_family_c64p_Hwi_dispatchAlways)
                  0c38a2e0    00000200     rts6600_elf.lib : setvbuf.obj (.text:setvbuf)
                  0c38a4e0    00000200     ipc.ae66 : Ipc.obj (.text:ti_sdo_ipc_family_c647x_MultiProcSetup_init__I)
                  0c38a6e0    00000200     sysbios.ae66 : BIOS.obj (.text:ti_sysbios_knl_Task_startCore__E)
                  0c38a8e0    00000200                  : BIOS.obj (.text:ti_sysbios_utils_Load_updateLoads__E)
                  0c38aae0    000001e0                  : BIOS.obj (.text:ti_sysbios_knl_Task_exit__E)
                  0c38acc0    000001e0                  : BIOS.obj (.text:ti_sysbios_timers_timer64_Timer_getFreq__E)
                  0c38aea0    000001e0                  : BIOS.obj (.text:ti_sysbios_utils_Load_idleFxn__E)
                  0c38b080    000001e0     ti.targets.rts6000.ae66 : Error.oe66 (.text:xdc_runtime_Error_policyDefault__E)
                  0c38b260    000001e0                             : Startup.oe66 (.text:xdc_runtime_Startup_startMods__I)
                  0c38b440    000001c0     rts6600_elf.lib : _printfi.obj (.text:_mcpy)
                  0c38b600    000001c0     sysbios.ae66 : BIOS.obj (.text:ti_sysbios_family_c66_Cache_block__I)
                  0c38b7c0    000001c0                  : BIOS.obj (.text:ti_sysbios_knl_Swi_post__E)
                  0c38b980    000001c0                  : BIOS.obj (.text:ti_sysbios_knl_Task_checkStacks__E)
                  0c38bb40    000001c0     ti.targets.rts6000.ae66 : Text.oe66 (.text:xdc_runtime_Text_putSite__E)
                  0c38bd00    000001a0     rts6600_elf.lib : trgdrv.obj (.text:HOSTrename)
                  0c38bea0    000001a0     ipc.ae66 : Ipc.obj (.text:MultiProc_setLocalId)
                  0c38c040    000001a0     rts6600_elf.lib : imath40.obj (.text:__c6xabi_divul)
                  0c38c1e0    000001a0     sysbios.ae66 : BIOS.obj (.text:ti_sysbios_gates_GateMutex_enter__E)
                  0c38c380    000001a0                  : BIOS.obj (.text:ti_sysbios_knl_Task_unblockI__E)
                  0c38c520    000001a0                  : BIOS.obj (.text:ti_sysbios_timers_timer64_Timer_start__E)
                  0c38c6c0    00000180     rts6600_elf.lib : copy_decompress_rle.obj (.text:__TI_decompress_rle_core)
                  0c38c840    00000180     sysbios.ae66 : c64p_Exception_asm.obj (.text)
                  0c38c9c0    00000180                  : BIOS.obj (.text:ti_sysbios_family_c66_Cache_getL2InitSize__I)
                  0c38cb40    00000180                  : BIOS.obj (.text:ti_sysbios_utils_Load_startup__E)
                  0c38ccc0    00000180                  : BIOS.obj (.text:ti_sysbios_utils_Load_taskCreateHook__E)
                  0c38ce40    00000180     EVM_C6674_configuration_pe66.oe66 (.text:ti_uia_loggers_LoggerStopMode_write8__E)
                  0c38cfc0    00000180     ti.targets.rts6000.ae66 : Core-smem.oe66 (.text:xdc_runtime_Core_constructObject__I)
                  0c38d140    00000160     ipc.ae66 : Ipc.obj (.text:ti_sdo_ipc_Notify_Module_startup__E)
                  0c38d2a0    00000160     EVM_C6674_configuration_pe66.oe66 (.text:ti_uia_loggers_LoggerStopMode_write4__E)
                  0c38d400    00000140     boot.ae66 : autoinit.oe66 (.text:_auto_init_elf)
                  0c38d540    00000140     rts6600_elf.lib : _printfi.obj (.text:_pproc_fflags)
                  0c38d680    00000140                     : lowlev.obj (.text:getdevice)
                  0c38d7c0    00000140     ipc.ae66 : Ipc.obj (.text:ti_sdo_utils_NameServer_Module_startup__E)
                  0c38d900    00000140     sysbios.ae66 : BIOS.obj (.text:ti_sysbios_gates_GateSwi_enter__E)
                  0c38da40    00000140                  : BIOS.obj (.text:ti_sysbios_knl_Semaphore_Instance_init__E)
                  0c38db80    00000140                  : BIOS.obj (.text:ti_sysbios_knl_Task_blockI__E)
                  0c38dcc0    00000140     ti.uia.loggers.ae66 : LoggerStopMode.oe66 (.text:ti_uia_loggers_LoggerStopMode_initQueueDescriptor__E)
                  0c38de00    00000140     EVM_C6674_configuration_pe66.oe66 (.text:ti_uia_loggers_LoggerStopMode_write0__E)
                  0c38df40    00000140     EVM_C6674_configuration_pe66.oe66 (.text:ti_uia_loggers_LoggerStopMode_write1__E)
                  0c38e080    00000140     EVM_C6674_configuration_pe66.oe66 (.text:ti_uia_loggers_LoggerStopMode_write2__E)
                  0c38e1c0    00000120     rts6600_elf.lib : fclose.obj (.text:_closefile)
                  0c38e2e0    00000120                     : _printfi.obj (.text:_ltostr)
                  0c38e400    00000120                     : fseek.obj (.text:fseek)
                  0c38e520    00000120     ipc.ae66 : Ipc.obj (.text:ti_sdo_ipc_MessageQ_Module_startup__E)
                  0c38e640    00000120     sysbios.ae66 : BIOS.obj (.text:ti_sysbios_utils_Load_taskDeleteHook__E)
                  0c38e760    00000120                  : BIOS.obj (.text:ti_sysbios_utils_Load_updateCurrentThreadTime__E)
                  0c38e880    00000120     ti.uia.loggers.ae66 : LoggerStopMode.oe66 (.text:ti_uia_loggers_LoggerStopMode_Module_startup__E)
                  0c38e9a0    00000120     ti.uia.runtime.ae66 : QueueDescriptor.oe66 (.text:ti_uia_runtime_QueueDescriptor_addToList__E)
                  0c38eac0    00000120     ti.targets.rts6000.ae66 : Core-mem.oe66 (.text:xdc_runtime_Core_deleteObject__I)
                  0c38ebe0    00000120                             : Text.oe66 (.text:xdc_runtime_Text_putLab__E)
                  0c38ed00    00000120                             : Text.oe66 (.text:xdc_runtime_Text_putMod__E)
                  0c38ee20    00000100     rts6600_elf.lib : trgdrv.obj (.text:HOSTlseek)
                  0c38ef20    00000100                     : _io_perm.obj (.text:_wrt_ok)
                  0c38f020    00000100     ipc.ae66 : Ipc.obj (.text:ti_sdo_ipc_Notify_Instance_finalize__E)
                  0c38f120    00000100     EVM_C6674_configuration_pe66.oe66 (.text:ti_sdo_ipc_Notify_create)
                  0c38f220    00000100     ipc.ae66 : Ipc.obj (.text:ti_sdo_ipc_family_c647x_Interrupt_Module_startup__E)
                  0c38f320    00000100              : Ipc.obj (.text:ti_sdo_ipc_gates_GateHWSem_Module_startup__E)
                  0c38f420    00000100     sysbios.ae66 : BIOS.obj (.text:ti_sysbios_gates_GateMutexPri_leave__E)
                  0c38f520    00000100                  : BIOS.obj (.text:ti_sysbios_knl_Swi_restoreHwi__E)
                  0c38f620    00000100                  : BIOS.obj (.text:ti_sysbios_timers_timer64_Timer_initDevice__I)
                  0c38f720    00000100     EVM_C6674_configuration_pe66.oe66 (.text:ti_sysbios_utils_Load_hwiBeginHook__E)
                  0c38f820    00000100     sysbios.ae66 : BIOS.obj (.text:ti_sysbios_xdcruntime_GateThreadSupport_leave__E)
                  0c38f920    00000100     ti.targets.rts6000.ae66 : Startup.oe66 (.text:xdc_runtime_Startup_exec__E)
                  0c38fa20    000000e0     rts6600_elf.lib : trgdrv.obj (.text:HOSTopen)
                  0c38fb00    000000e0                     : trgdrv.obj (.text:HOSTread)
                  0c38fbe0    000000e0                     : _printfi.obj (.text:_div)
                  0c38fcc0    000000e0                     : atoi.obj (.text:atoi)
                  0c38fda0    000000e0                     : lowlev.obj (.text:close)
                  0c38fe80    000000e0                     : fflush.obj (.text:fflush)
                  0c38ff60    000000e0                     : ltoa.obj (.text:ltoa)
                  0c390040    000000e0                     : memset.obj (.text:memset)
                  0c390120    000000e0                     : printf.obj (.text:printf)
                  0c390200    000000e0     sysbios.ae66 : BIOS.obj (.text:ti_sysbios_knl_Swi_runLoop__I)
                  0c3902e0    000000e0                  : BIOS.obj (.text:ti_sysbios_timers_timer64_Timer_startup__E)
                  0c3903c0    000000e0     ti.targets.rts6000.ae66 : Error.oe66 (.text:xdc_runtime_Error_print__E)
                  0c3904a0    000000e0                             : Memory.oe66 (.text:xdc_runtime_Memory_alloc__E)
                  0c390580    000000e0                             : Text.oe66 (.text:xdc_runtime_Text_visitRope2__I)
                  0c390660    000000e0     EVM_C6674_configuration_pe66.oe66 (.text:xdc_runtime_knl_GateThread_Object__create__S)
                  0c390740    000000e0     EVM_C6674_configuration_pe66.oe66 (.text:xdc_runtime_knl_GateThread_create)
                  0c390820    000000c0     rts6600_elf.lib : trgdrv.obj (.text:HOSTunlink)
                  0c3908e0    000000c0                     : trgdrv.obj (.text:HOSTwrite)
                  0c3909a0    000000c0                     : divu.obj (.text:__divu)
                  0c390a60    000000c0                     : fflush.obj (.text:_doflush)
                  0c390b20    000000c0                     : exit.obj (.text:exit)
                  0c390be0    000000c0     hello.obj (.text)
                  0c390ca0    000000c0     sysbios.ae66 : BIOS.obj (.text:ti_sysbios_gates_GateAll_leave__E)
                  0c390d60    000000c0                  : BIOS.obj (.text:ti_sysbios_heaps_HeapMem_alloc__E)
                  0c390e20    000000c0                  : BIOS.obj (.text:ti_sysbios_heaps_HeapMem_getStats__E)
                  0c390ee0    000000c0                  : BIOS.obj (.text:ti_sysbios_knl_Clock_logTick__E)
                  0c390fa0    000000c0                  : BIOS.obj (.text:ti_sysbios_knl_Swi_schedule__I)
                  0c391060    000000c0                  : BIOS.obj (.text:ti_sysbios_knl_Task_allBlockedFunction__I)
                  0c391120    000000c0                  : BIOS.obj (.text:ti_sysbios_timers_timer64_Timer_stop__E)
                  0c3911e0    000000c0                  : BIOS.obj (.text:ti_sysbios_utils_Load_taskSwitchHook__E)
                  0c3912a0    000000c0     ti.uia.loggers.ae66 : LoggerStopMode.oe66 (.text:ti_uia_loggers_LoggerStopMode_flush__E)
                  0c391360    000000c0     rts6600_elf.lib : tls.obj (.text:tls:init:__TI_tls_init)
                  0c391420    000000c0     ti.targets.rts6000.ae66 : System.oe66 (.text:xdc_runtime_System_formatNum__I)
                  0c3914e0    000000a0     rts6600_elf.lib : trgdrv.obj (.text:HOSTclose)
                  0c391580    000000a0                     : remu.obj (.text:__remu)
                  0c391620    000000a0                     : fopen.obj (.text:_cleanup)
                  0c3916c0    000000a0                     : _printfi.obj (.text:_ecpy)
                  0c391760    000000a0                     : _printfi.obj (.text:_fcpy)
                  0c391800    000000a0                     : _printfi.obj (.text:_pconv_f)
                  0c3918a0    000000a0                     : lowlev.obj (.text:finddevice)
                  0c391940    000000a0                     : lowlev.obj (.text:lseek)
                  0c3919e0    000000a0                     : memcpy64.obj (.text:memcpy)
                  0c391a80    000000a0     sysbios.ae66 : BIOS.obj (.text:ti_sysbios_family_c64p_Exception_Module_startup__E)
                  0c391b20    000000a0                  : BIOS.obj (.text:ti_sysbios_heaps_HeapMem_init__I)
                  0c391bc0    000000a0                  : BIOS.obj (.text:ti_sysbios_utils_Load_swiBeginHook__E)
                  0c391c60    000000a0     rts6600_elf.lib : lowlev.obj (.text:write)
                  0c391d00    000000a0     ti.targets.rts6000.ae66 : Assert.oe66 (.text:xdc_runtime_Assert_raise__I)
                  0c391da0    000000a0                             : Error.oe66 (.text:xdc_runtime_Error_setX__E)
                  0c391e40    000000a0                             : Text.oe66 (.text:xdc_runtime_Text_xprintf__I)
                  0c391ee0    00000080     rts6600_elf.lib : llshift.obj (.text:__c6xabi_llshl)
                  0c391f60    00000080     sysbios.ae66 : c62_TaskSupport_asm.obj (.text:_ti_sysbios_family_c62_TaskSupport_swap__E)
                  0c391fe0    00000080     EVM_C6674_configuration_pe66.oe66 (.text:malloc)
                  0c392060    00000080     rts6600_elf.lib : trgmsg.obj (.text:readmsg)
                  0c3920e0    00000080     EVM_C6674_configuration_pe66.oe66 (.text:ti_sysbios_BIOS_atExitFunc__I)
                  0c392160    00000080     sysbios.ae66 : BIOS.obj (.text:ti_sysbios_family_c64p_Hwi_dispatchC__I)
                  0c3921e0    00000080                  : BIOS.obj (.text:ti_sysbios_family_c64p_Hwi_getStackInfo__E)
                  0c392260    00000080     EVM_C6674_configuration_pe66.oe66 (.text:ti_sysbios_gates_GateAll_Object__create__S)
                  0c3922e0    00000080     EVM_C6674_configuration_pe66.oe66 (.text:ti_sysbios_gates_GateHwi_Object__create__S)
                  0c392360    00000080     EVM_C6674_configuration_pe66.oe66 (.text:ti_sysbios_gates_GateMutexPri_Object__create__S)
                  0c3923e0    00000080     EVM_C6674_configuration_pe66.oe66 (.text:ti_sysbios_gates_GateMutex_Object__create__S)
                  0c392460    00000080     EVM_C6674_configuration_pe66.oe66 (.text:ti_sysbios_gates_GateSwi_Object__create__S)
                  0c3924e0    00000080     sysbios.ae66 : BIOS.obj (.text:ti_sysbios_gates_GateSwi_leave__E)
                  0c392560    00000080                  : BIOS.obj (.text:ti_sysbios_hal_Hwi_checkStack)
                  0c3925e0    00000080                  : BIOS.obj (.text:ti_sysbios_hal_Hwi_initStack)
                  0c392660    00000080     EVM_C6674_configuration_pe66.oe66 (.text:ti_sysbios_heaps_HeapMem_Object__create__S)
                  0c3926e0    00000080     EVM_C6674_configuration_pe66.oe66 (.text:ti_sysbios_knl_Clock_doTick__I)
                  0c392760    00000080     sysbios.ae66 : BIOS.obj (.text:ti_sysbios_knl_Idle_run__E)
                  0c3927e0    00000080                  : BIOS.obj (.text:ti_sysbios_knl_Swi_startup__E)
                  0c392860    00000080                  : BIOS.obj (.text:ti_sysbios_knl_Task_restore__E)
                  0c3928e0    00000080                  : BIOS.obj (.text:ti_sysbios_utils_Load_hwiEndHook__E)
                  0c392960    00000080                  : BIOS.obj (.text:ti_sysbios_utils_Load_swiEndHook__E)
                  0c3929e0    00000080     EVM_C6674_configuration_pe66.oe66 (.text:ti_sysbios_xdcruntime_GateThreadSupport_Object__create__S)
                  0c392a60    00000080     EVM_C6674_configuration_pe66.oe66 (.text:ti_uia_loggers_LoggerStopMode_Object__create__S)
                  0c392ae0    00000080     rts6600_elf.lib : lowlev.obj (.text:unlink)
                  0c392b60    00000080     ti.targets.rts6000.ae66 : Core-label.oe66 (.text:xdc_runtime_Core_assignLabel__I)
                  0c392be0    00000080                             : Core-params.oe66 (.text:xdc_runtime_Core_assignParams__I)
                  0c392c60    00000080                             : System.oe66 (.text:xdc_runtime_System_atexit__E)
                  0c392ce0    00000080                             : System.oe66 (.text:xdc_runtime_System_processAtExit__E)
                  0c392d60    00000080                             : System.oe66 (.text:xdc_runtime_System_putchar__I)
                  0c392de0    00000080                             : Text.oe66 (.text:xdc_runtime_Text_printVisFxn__I)
                  0c392e60    00000060     rts6600_elf.lib : frcmpyd_div.obj (.text:__c6xabi_frcmpyd_div)
                  0c392ec0    00000060                     : llshift.obj (.text:__c6xabi_llshru)
                  0c392f20    00000060                     : imath64.obj (.text:_subcull)
                  0c392f80    00000060     sysbios.ae66 : c64p_Hwi_asm_switch.obj (.text:_ti_sysbios_family_c64p_Hwi_switchAndDispatch__I)
                  0c392fe0    00000060                  : c64p_Hwi_asm_switch.obj (.text:_ti_sysbios_family_xxx_Hwi_switchAndRunFunc)
                  0c393040    00000060     rts6600_elf.lib : memccpy.obj (.text:memccpy)
                  0c3930a0    00000060     EVM_C6674_configuration_pe66.oe66 (.text:ti_sdo_utils_List_construct)
                  0c393100    00000060     EVM_C6674_configuration_pe66.oe66 (.text:ti_sysbios_BIOS_errorRaiseHook__I)
                  0c393160    00000060     EVM_C6674_configuration_pe66.oe66 (.text:ti_sysbios_BIOS_registerRTSLock__I)
                  0c3931c0    00000060     EVM_C6674_configuration_pe66.oe66 (.text:ti_sysbios_BIOS_removeRTSLock__I)
                  0c393220    00000060     EVM_C6674_configuration_pe66.oe66 (.text:ti_sysbios_BIOS_rtsLock__I)
                  0c393280    00000060     EVM_C6674_configuration_pe66.oe66 (.text:ti_sysbios_BIOS_startFunc__I)
                  0c3932e0    00000060     sysbios.ae66 : BIOS.obj (.text:ti_sysbios_family_c62_TaskSupport_start__E)
                  0c393340    00000060                  : BIOS.obj (.text:ti_sysbios_family_c66_Cache_Module_startup__E)
                  0c3933a0    00000060                  : BIOS.obj (.text:ti_sysbios_family_c66_tci66xx_CpIntc_unused__E)
                  0c393400    00000060                  : BIOS.obj (.text:ti_sysbios_gates_GateAll_enter__E)
                  0c393460    00000060     EVM_C6674_configuration_pe66.oe66 (.text:ti_sysbios_gates_GateMutexPri_Object__delete__S)
                  0c3934c0    00000060     EVM_C6674_configuration_pe66.oe66 (.text:ti_sysbios_gates_GateMutexPri_construct)
                  0c393520    00000060     EVM_C6674_configuration_pe66.oe66 (.text:ti_sysbios_gates_GateMutex_Object__delete__S)
                  0c393580    00000060     sysbios.ae66 : BIOS.obj (.text:ti_sysbios_heaps_HeapMem_free__E)
                  0c3935e0    00000060                  : BIOS.obj (.text:ti_sysbios_knl_Clock_Module_startup__E)
                  0c393640    00000060     EVM_C6674_configuration_pe66.oe66 (.text:ti_sysbios_knl_Queue_construct)
                  0c3936a0    00000060     EVM_C6674_configuration_pe66.oe66 (.text:ti_sysbios_knl_Semaphore_construct)
                  0c393700    00000060     sysbios.ae66 : BIOS.obj (.text:ti_sysbios_knl_Semaphore_pendTimeout__I)
                  0c393760    00000060                  : BIOS.obj (.text:ti_sysbios_knl_Task_enter__I)
                  0c3937c0    00000060     EVM_C6674_configuration_pe66.oe66 (.text:ti_sysbios_xdcruntime_GateThreadSupport_Object__delete__S)
                  0c393820    00000060     ti.uia.loggers.ae66 : LoggerStopMode.oe66 (.text:ti_uia_loggers_LoggerStopMode_Instance_init__E)
                  0c393880    00000060                         : LoggerStopMode.oe66 (.text:ti_uia_loggers_LoggerStopMode_initBuffer__I)
                  0c3938e0    00000060                         : LoggerStopMode.oe66 (.text:ti_uia_loggers_LoggerStopMode_reset__E)
                  0c393940    00000060     rts6600_elf.lib : trgmsg.obj (.text:writemsg)
                  0c3939a0    00000060     ti.targets.rts6000.ae66 : Memory.oe66 (.text:xdc_runtime_Memory_valloc__E)
                  0c393a00    00000060                             : SysStd.oe66 (.text:xdc_runtime_SysStd_abort__E)
                  0c393a60    00000060                             : System.oe66 (.text:xdc_runtime_System_avprintf__E)
                  0c393ac0    00000060                             : System.oe66 (.text:xdc_runtime_System_vprintf__E)
                  0c393b20    00000060                             : Text.oe66 (.text:xdc_runtime_Text_cordText__E)
                  0c393b80    00000060     EVM_C6674_configuration_pe66.oe66 (.text:xdc_runtime_knl_GateThread_Object__delete__S)
                  0c393be0    00000040     rts6600_elf.lib : isinf.obj (.text:__c6xabi_isinf)
                  0c393c20    00000040                     : _printfi.obj (.text:__c6xabi_isnan)
                  0c393c60    00000040                     : args_main.obj (.text:_args_main)
                  0c393ca0    00000040     sysbios.ae66 : c62_TaskSupport_asm.obj (.text:_ti_sysbios_family_c62_TaskSupport_buildTaskStack)
                  0c393ce0    00000040     EVM_C6674_configuration_pe66.oe66 (.text:free)
                  0c393d20    00000040     EVM_C6674_configuration_pe66.oe66 (.text:ti_sdo_utils_NameServer_Module__startupDone__F)
                  0c393d60    00000040     EVM_C6674_configuration_pe66.oe66 (.text:ti_sdo_utils_NameServer_Object__get__S)
                  0c393da0    00000040     EVM_C6674_configuration_pe66.oe66 (.text:ti_sysbios_BIOS_exitFunc__I)
                  0c393de0    00000040     EVM_C6674_configuration_pe66.oe66 (.text:ti_sysbios_BIOS_rtsUnlock__I)
                  0c393e20    00000040     EVM_C6674_configuration_pe66.oe66 (.text:ti_sysbios_family_c64p_Hwi_Module__startupDone__F)
                  0c393e60    00000040     sysbios.ae66 : BIOS.obj (.text:ti_sysbios_family_c64p_Hwi_disableInterrupt__E)
                  0c393ea0    00000040                  : BIOS.obj (.text:ti_sysbios_family_c64p_Hwi_enableInterrupt__E)
                  0c393ee0    00000040     EVM_C6674_configuration_pe66.oe66 (.text:ti_sysbios_gates_GateAll_Handle__label__S)
                  0c393f20    00000040     EVM_C6674_configuration_pe66.oe66 (.text:ti_sysbios_gates_GateAll_Object__delete__S)
                  0c393f60    00000040     EVM_C6674_configuration_pe66.oe66 (.text:ti_sysbios_gates_GateHwi_Handle__label__S)
                  0c393fa0    00000040     EVM_C6674_configuration_pe66.oe66 (.text:ti_sysbios_gates_GateHwi_Object__delete__S)
                  0c393fe0    00000040     EVM_C6674_configuration_pe66.oe66 (.text:ti_sysbios_gates_GateMutexPri_Handle__label__S)
                  0c394020    00000040     sysbios.ae66 : BIOS.obj (.text:ti_sysbios_gates_GateMutexPri_Instance_init__E)
                  0c394060    00000040     EVM_C6674_configuration_pe66.oe66 (.text:ti_sysbios_gates_GateMutexPri_Object__destruct__S)
                  0c3940a0    00000040     EVM_C6674_configuration_pe66.oe66 (.text:ti_sysbios_gates_GateMutex_Handle__label__S)
                  0c3940e0    00000040     sysbios.ae66 : BIOS.obj (.text:ti_sysbios_gates_GateMutex_Instance_init__E)
                  0c394120    00000040                  : BIOS.obj (.text:ti_sysbios_gates_GateMutex_leave__E)
                  0c394160    00000040     EVM_C6674_configuration_pe66.oe66 (.text:ti_sysbios_gates_GateSwi_Handle__label__S)
                  0c3941a0    00000040     EVM_C6674_configuration_pe66.oe66 (.text:ti_sysbios_gates_GateSwi_Object__delete__S)
                  0c3941e0    00000040     EVM_C6674_configuration_pe66.oe66 (.text:ti_sysbios_heaps_HeapMem_Handle__label__S)
                  0c394220    00000040     EVM_C6674_configuration_pe66.oe66 (.text:ti_sysbios_heaps_HeapMem_Object__delete__S)
                  0c394260    00000040     EVM_C6674_configuration_pe66.oe66 (.text:ti_sysbios_heaps_HeapMem_Object__get__S)
                  0c3942a0    00000040     EVM_C6674_configuration_pe66.oe66 (.text:ti_sysbios_knl_Semaphore_Object__destruct__S)
                  0c3942e0    00000040     EVM_C6674_configuration_pe66.oe66 (.text:ti_sysbios_knl_Swi_Object__get__S)
                  0c394320    00000040     EVM_C6674_configuration_pe66.oe66 (.text:ti_sysbios_knl_Task_Object__get__S)
                  0c394360    00000040     EVM_C6674_configuration_pe66.oe66 (.text:ti_sysbios_timers_timer64_Timer_Module__startupDone__F)
                  0c3943a0    00000040     sysbios.ae66 : BIOS.obj (.text:ti_sysbios_xdcruntime_GateThreadSupport_Instance_init__E)
                  0c3943e0    00000040     EVM_C6674_configuration_pe66.oe66 (.text:ti_uia_loggers_LoggerStopMode_Handle__label__S)
                  0c394420    00000040     EVM_C6674_configuration_pe66.oe66 (.text:ti_uia_loggers_LoggerStopMode_Object__delete__S)
                  0c394460    00000040     EVM_C6674_configuration_pe66.oe66 (.text:ti_uia_loggers_LoggerStopMode_Object__get__S)
                  0c3944a0    00000040     ti.uia.loggers.ae66 : LoggerStopMode.oe66 (.text:ti_uia_loggers_LoggerStopMode_disable__E)
                  0c3944e0    00000040                         : LoggerStopMode.oe66 (.text:ti_uia_loggers_LoggerStopMode_enable__E)
                  0c394520    00000040     ti.targets.rts6000.ae66 : Error.oe66 (.text:xdc_runtime_Error_check__E)
                  0c394560    00000040                             : Error.oe66 (.text:xdc_runtime_Error_init__E)
                  0c3945a0    00000040     EVM_C6674_configuration_pe66.oe66 (.text:xdc_runtime_GateNull_Handle__label__S)
                  0c3945e0    00000040     EVM_C6674_configuration_pe66.oe66 (.text:xdc_runtime_GateNull_Object__create__S)
                  0c394620    00000040     EVM_C6674_configuration_pe66.oe66 (.text:xdc_runtime_GateNull_Object__delete__S)
                  0c394660    00000040     ti.targets.rts6000.ae66 : Memory.oe66 (.text:xdc_runtime_Memory_free__E)
                  0c3946a0    00000040                             : Registry.oe66 (.text:xdc_runtime_Registry_findById__E)
                  0c3946e0    00000040                             : System.oe66 (.text:xdc_runtime_System_abort__E)
                  0c394720    00000040     EVM_C6674_configuration_pe66.oe66 (.text:xdc_runtime_System_aprintf__E)
                  0c394760    00000040     ti.targets.rts6000.ae66 : System.oe66 (.text:xdc_runtime_System_exit__E)
                  0c3947a0    00000040     EVM_C6674_configuration_pe66.oe66 (.text:xdc_runtime_System_printf__E)
                  0c3947e0    00000040     ti.targets.rts6000.ae66 : Text.oe66 (.text:xdc_runtime_Text_ropeText__E)
                  0c394820    00000040     EVM_C6674_configuration_pe66.oe66 (.text:xdc_runtime_knl_GateThread_Handle__label__S)
                  0c394860    00000040     ti.targets.rts6000.ae66 : GateThread.oe66 (.text:xdc_runtime_knl_GateThread_Instance_finalize__E)
                  0c3948a0    00000040                             : GateThread.oe66 (.text:xdc_runtime_knl_GateThread_Instance_init__E)
                  0c3948e0    00000020                             : LoggerBuf.oe66 (.text:LoggerBuf_instanceStartup)
                  0c394900    00000020     ipc.ae66 : Ipc.obj (.text:MultiProc_getNumProcessors)
                  0c394920    00000020     rts6600_elf.lib : negll.obj (.text:__c6xabi_negll)
                  0c394940    00000020     ti.targets.rts6000.ae66 : xdc_noinit.oe66 (.text:__xdc__init)
                  0c394960    00000020     rts6600_elf.lib : _lock.obj (.text:_nop)
                  0c394980    00000020                     : printf.obj (.text:_outc)
                  0c3949a0    00000020                     : printf.obj (.text:_outs)
                  0c3949c0    00000020                     : _lock.obj (.text:_register_lock)
                  0c3949e0    00000020                     : _data_synch.obj (.text:_register_synch_api)
                  0c394a00    00000020                     : _lock.obj (.text:_register_unlock)
                  0c394a20    00000020     sysbios.ae66 : c62_TaskSupport_asm.obj (.text:_ti_sysbios_family_c62_TaskSupport_glue)
                  0c394a40    00000020     rts6600_elf.lib : exit.obj (.text:abort)
                  0c394a60    00000020                     : copy_decompress_none.obj (.text:decompress:none:__TI_decompress_none)
                  0c394a80    00000020                     : copy_decompress_rle.obj (.text:decompress:rle24:__TI_decompress_rle24)
                  0c394aa0    00000020                     : fputc.obj (.text:putc)
                  0c394ac0    00000020                     : fputc.obj (.text:putchar)
                  0c394ae0    00000020     EVM_C6674_configuration_pe66.oe66 (.text:ti_sdo_ipc_MessageQ_Object__get__S)
                  0c394b00    00000020     ipc.ae66 : Ipc.obj (.text:ti_sdo_utils_List_Instance_init__E)
                  0c394b20    00000020     EVM_C6674_configuration_pe66.oe66 (.text:ti_sdo_utils_List_Object__destruct__S)
                  0c394b40    00000020     EVM_C6674_configuration_pe66.oe66 (.text:ti_sdo_utils_List_Object__get__S)
                  0c394b60    00000020     EVM_C6674_configuration_pe66.oe66 (.text:ti_sdo_utils_List_destruct)
                  0c394b80    00000020     ipc.ae66 : Ipc.obj (.text:ti_sdo_utils_MultiProc_getClusterId__F)
                  0c394ba0    00000020     EVM_C6674_configuration_pe66.oe66 (.text:ti_sysbios_BIOS_RtsGateProxy_enter__E)
                  0c394bc0    00000020     EVM_C6674_configuration_pe66.oe66 (.text:ti_sysbios_BIOS_RtsGateProxy_leave__E)
                  0c394be0    00000020     sysbios.ae66 : BIOS.obj (.text:ti_sysbios_BIOS_getCpuFreq__E)
                  0c394c00    00000020                  : BIOS.obj (.text:ti_sysbios_BIOS_linkedWithIncorrectBootLibrary__E)
                  0c394c20    00000020     EVM_C6674_configuration_pe66.oe66 (.text:ti_sysbios_BIOS_nullFunc__I)
                  0c394c40    00000020     sysbios.ae66 : BIOS.obj (.text:ti_sysbios_BIOS_setThreadType__E)
                  0c394c60    00000020     EVM_C6674_configuration_pe66.oe66 (.text:ti_sysbios_family_c62_TaskSupport_Module__startupDone__S)
                  0c394c80    00000020     sysbios.ae66 : BIOS.obj (.text:ti_sysbios_family_c62_TaskSupport_checkStack__E)
                  0c394ca0    00000020                  : BIOS.obj (.text:ti_sysbios_family_c64p_Hwi_clearInterrupt__E)
                  0c394cc0    00000020                  : BIOS.obj (.text:ti_sysbios_family_c64p_Hwi_startup__E)
                  0c394ce0    00000020                  : BIOS.obj (.text:ti_sysbios_family_c64p_Hwi_switchFromBootStack__E)
                  0c394d00    00000020                  : BIOS.obj (.text:ti_sysbios_family_c64p_TimestampProvider_Module_startup__E)
                  0c394d20    00000020                  : BIOS.obj (.text:ti_sysbios_family_c64p_TimestampProvider_get32__E)
                  0c394d40    00000020                  : BIOS.obj (.text:ti_sysbios_family_c64p_TimestampProvider_get64__E)
                  0c394d60    00000020                  : BIOS.obj (.text:ti_sysbios_family_c64p_tci6488_TimerSupport_enable__E)
                  0c394d80    00000020                  : BIOS.obj (.text:ti_sysbios_family_c66_Cache_RTSSynchInv__I)
                  0c394da0    00000020                  : BIOS.obj (.text:ti_sysbios_family_c66_Cache_RTSSynchWbInv__I)
                  0c394dc0    00000020                  : BIOS.obj (.text:ti_sysbios_family_c66_Cache_RTSSynchWb__I)
                  0c394de0    00000020                  : BIOS.obj (.text:ti_sysbios_family_c66_Cache_wait__E)
                  0c394e00    00000020                  : BIOS.obj (.text:ti_sysbios_gates_GateAll_Instance_init__E)
                  0c394e20    00000020                  : BIOS.obj (.text:ti_sysbios_gates_GateAll_query__E)
                  0c394e40    00000020                  : BIOS.obj (.text:ti_sysbios_gates_GateHwi_Instance_init__E)
                  0c394e60    00000020                  : BIOS.obj (.text:ti_sysbios_gates_GateHwi_enter__E)
                  0c394e80    00000020                  : BIOS.obj (.text:ti_sysbios_gates_GateHwi_leave__E)
                  0c394ea0    00000020                  : BIOS.obj (.text:ti_sysbios_gates_GateHwi_query__E)
                  0c394ec0    00000020                  : BIOS.obj (.text:ti_sysbios_gates_GateMutexPri_Instance_finalize__E)
                  0c394ee0    00000020     EVM_C6674_configuration_pe66.oe66 (.text:ti_sysbios_gates_GateMutexPri_destruct)
                  0c394f00    00000020     sysbios.ae66 : BIOS.obj (.text:ti_sysbios_gates_GateMutexPri_query__E)
                  0c394f20    00000020                  : BIOS.obj (.text:ti_sysbios_gates_GateMutex_Instance_finalize__E)
                  0c394f40    00000020                  : BIOS.obj (.text:ti_sysbios_gates_GateMutex_query__E)
                  0c394f60    00000020                  : BIOS.obj (.text:ti_sysbios_gates_GateSwi_Instance_init__E)
                  0c394f80    00000020                  : BIOS.obj (.text:ti_sysbios_gates_GateSwi_query__E)
                  0c394fa0    00000020     EVM_C6674_configuration_pe66.oe66 (.text:ti_sysbios_hal_Hwi_HwiProxy_Module__startupDone__S)
                  0c394fc0    00000020     sysbios.ae66 : BIOS.obj (.text:ti_sysbios_hal_Hwi_Module_startup__E)
                  0c394fe0    00000020                  : BIOS.obj (.text:ti_sysbios_hal_Timer_Module_startup__E)
                  0c395000    00000020     EVM_C6674_configuration_pe66.oe66 (.text:ti_sysbios_hal_Timer_TimerProxy_Module__startupDone__S)
                  0c395020    00000020     EVM_C6674_configuration_pe66.oe66 (.text:ti_sysbios_heaps_HeapMem_Module_GateProxy_enter__E)
                  0c395040    00000020     EVM_C6674_configuration_pe66.oe66 (.text:ti_sysbios_heaps_HeapMem_Module_GateProxy_leave__E)
                  0c395060    00000020     sysbios.ae66 : BIOS.obj (.text:ti_sysbios_heaps_HeapMem_isBlocking__E)
                  0c395080    00000020     EVM_C6674_configuration_pe66.oe66 (.text:ti_sysbios_knl_Clock_TimerProxy_Module__startupDone__S)
                  0c3950a0    00000020     EVM_C6674_configuration_pe66.oe66 (.text:ti_sysbios_knl_Clock_TimerProxy_getMaxTicks__E)
                  0c3950c0    00000020     sysbios.ae66 : BIOS.obj (.text:ti_sysbios_knl_Idle_loop__E)
                  0c3950e0    00000020                  : BIOS.obj (.text:ti_sysbios_knl_Queue_Instance_init__E)
                  0c395100    00000020     EVM_C6674_configuration_pe66.oe66 (.text:ti_sysbios_knl_Queue_Object__destruct__S)
                  0c395120    00000020     EVM_C6674_configuration_pe66.oe66 (.text:ti_sysbios_knl_Queue_Object__get__S)
                  0c395140    00000020     EVM_C6674_configuration_pe66.oe66 (.text:ti_sysbios_knl_Queue_destruct)
                  0c395160    00000020     sysbios.ae66 : BIOS.obj (.text:ti_sysbios_knl_Queue_empty__E)
                  0c395180    00000020                  : BIOS.obj (.text:ti_sysbios_knl_Semaphore_Instance_finalize__E)
                  0c3951a0    00000020     EVM_C6674_configuration_pe66.oe66 (.text:ti_sysbios_knl_Semaphore_destruct)
                  0c3951c0    00000020     sysbios.ae66 : BIOS.obj (.text:ti_sysbios_knl_Swi_disable__E)
                  0c3951e0    00000020     EVM_C6674_configuration_pe66.oe66 (.text:ti_sysbios_knl_Task_SupportProxy_Module__startupDone__S)
                  0c395200    00000020     sysbios.ae66 : BIOS.obj (.text:ti_sysbios_knl_Task_disable__E)
                  0c395220    00000020                  : BIOS.obj (.text:ti_sysbios_knl_Task_getHookContext__E)
                  0c395240    00000020                  : BIOS.obj (.text:ti_sysbios_knl_Task_startup__E)
                  0c395260    00000020                  : BIOS.obj (.text:ti_sysbios_timers_timer64_Timer_getMaxTicks__E)
                  0c395280    00000020                  : BIOS.obj (.text:ti_sysbios_utils_Load_taskRegHook__E)
                  0c3952a0    00000020                  : BIOS.obj (.text:ti_sysbios_xdcruntime_GateThreadSupport_Instance_finalize__E)
                  0c3952c0    00000020                  : BIOS.obj (.text:ti_sysbios_xdcruntime_GateThreadSupport_enter__E)
                  0c3952e0    00000020     ti.uia.loggers.ae66 : LoggerStopMode.oe66 (.text:ti_uia_loggers_LoggerStopMode_getContents__E)
                  0c395300    00000020     EVM_C6674_configuration_pe66.oe66 (.text:ti_uia_loggers_LoggerStopMode_getFilterLevel__E)
                  0c395320    00000020     ti.uia.loggers.ae66 : LoggerStopMode.oe66 (.text:ti_uia_loggers_LoggerStopMode_getInstanceId__E)
                  0c395340    00000020                         : LoggerStopMode.oe66 (.text:ti_uia_loggers_LoggerStopMode_getMaxLength__E)
                  0c395360    00000020                         : LoggerStopMode.oe66 (.text:ti_uia_loggers_LoggerStopMode_getPriority__E)
                  0c395380    00000020                         : LoggerStopMode.oe66 (.text:ti_uia_loggers_LoggerStopMode_getTransferType__E)
                  0c3953a0    00000020                         : LoggerStopMode.oe66 (.text:ti_uia_loggers_LoggerStopMode_isEmpty__E)
                  0c3953c0    00000020     EVM_C6674_configuration_pe66.oe66 (.text:ti_uia_loggers_LoggerStopMode_setFilterLevel__E)
                  0c3953e0    00000020     ti.uia.loggers.ae66 : LoggerStopMode.oe66 (.text:ti_uia_loggers_LoggerStopMode_setPriority__E)
                  0c395400    00000020     ti.targets.rts6000.ae66 : Error.oe66 (.text:xdc_runtime_Error_getSite__E)
                  0c395420    00000020                             : Error.oe66 (.text:xdc_runtime_Error_raiseX__E)
                  0c395440    00000020                             : GateNull.oe66 (.text:xdc_runtime_GateNull_enter__E)
                  0c395460    00000020                             : GateNull.oe66 (.text:xdc_runtime_GateNull_leave__E)
                  0c395480    00000020                             : GateNull.oe66 (.text:xdc_runtime_GateNull_query__E)
                  0c3954a0    00000020                             : Gate.oe66 (.text:xdc_runtime_Gate_enterSystem__E)
                  0c3954c0    00000020                             : Gate.oe66 (.text:xdc_runtime_Gate_leaveSystem__E)
                  0c3954e0    00000020     EVM_C6674_configuration_pe66.oe66 (.text:xdc_runtime_IHeap_alloc)
                  0c395500    00000020     EVM_C6674_configuration_pe66.oe66 (.text:xdc_runtime_IHeap_free)
                  0c395520    00000020     EVM_C6674_configuration_pe66.oe66 (.text:xdc_runtime_Memory_HeapProxy_alloc__E)
                  0c395540    00000020     EVM_C6674_configuration_pe66.oe66 (.text:xdc_runtime_Memory_HeapProxy_free__E)
                  0c395560    00000020     ti.targets.rts6000.ae66 : Memory.oe66 (.text:xdc_runtime_Memory_calloc__E)
                  0c395580    00000020                             : Memory.oe66 (.text:xdc_runtime_Memory_getMaxDefaultTypeAlign__E)
                  0c3955a0    00000020     EVM_C6674_configuration_pe66.oe66 (.text:xdc_runtime_Startup_Module__startupDone__S)
                  0c3955c0    00000020     EVM_C6674_configuration_pe66.oe66 (.text:xdc_runtime_Startup_exec__I)
                  0c3955e0    00000020     ti.targets.rts6000.ae66 : Startup.oe66 (.text:xdc_runtime_Startup_rtsDone__E)
                  0c395600    00000020                             : SysStd.oe66 (.text:xdc_runtime_SysStd_exit__E)
                  0c395620    00000020                             : SysStd.oe66 (.text:xdc_runtime_SysStd_putch__E)
                  0c395640    00000020                             : SysStd.oe66 (.text:xdc_runtime_SysStd_ready__E)
                  0c395660    00000020     EVM_C6674_configuration_pe66.oe66 (.text:xdc_runtime_System_Module_GateProxy_enter__E)
                  0c395680    00000020     EVM_C6674_configuration_pe66.oe66 (.text:xdc_runtime_System_Module_GateProxy_leave__E)
                  0c3956a0    00000020     ti.targets.rts6000.ae66 : System.oe66 (.text:xdc_runtime_System_Module_startup__E)
                  0c3956c0    00000020                             : System.oe66 (.text:xdc_runtime_System_aprintf_va__F)
                  0c3956e0    00000020                             : System.oe66 (.text:xdc_runtime_System_printf_va__F)
                  0c395700    00000020                             : System.oe66 (.text:xdc_runtime_System_vsnprintf__E)
                  0c395720    00000020     EVM_C6674_configuration_pe66.oe66 (.text:xdc_runtime_Text_visitRope__I)
                  0c395740    00000020     EVM_C6674_configuration_pe66.oe66 (.text:xdc_runtime_knl_GateThread_Module__startupDone__S)
                  0c395760    00000020     EVM_C6674_configuration_pe66.oe66 (.text:xdc_runtime_knl_GateThread_Proxy_Object__create__S)
                  0c395780    00000020     EVM_C6674_configuration_pe66.oe66 (.text:xdc_runtime_knl_GateThread_Proxy_Object__delete__S)
                  0c3957a0    00000020     EVM_C6674_configuration_pe66.oe66 (.text:xdc_runtime_knl_GateThread_Proxy_create)
                  0c3957c0    00000020     EVM_C6674_configuration_pe66.oe66 (.text:xdc_runtime_knl_GateThread_Proxy_delete)
                  0c3957e0    00000020     EVM_C6674_configuration_pe66.oe66 (.text:xdc_runtime_knl_GateThread_Proxy_enter__E)
                  0c395800    00000020     EVM_C6674_configuration_pe66.oe66 (.text:xdc_runtime_knl_GateThread_Proxy_leave__E)
                  0c395820    00000020     ti.targets.rts6000.ae66 : GateThread.oe66 (.text:xdc_runtime_knl_GateThread_enter__E)
                  0c395840    00000020                             : GateThread.oe66 (.text:xdc_runtime_knl_GateThread_leave__E)
                  0c395860    00000010                             : LoggerBuf.oe66 ($Tramp$S$$xdc_runtime_LoggerBuf_reset__E)
                  0c395870    00000010     --HOLE-- [fill = 00000000]

.vecs      0    0c395c00    00000200     
                  0c395c00    00000200     EVM_C6674_configuration_pe66.oe66 (.vecs)

ti.sdo.ipc.SharedRegion_1 
*          0    81000000    0e000000     NOLOAD SECTION
                  81000000    0e000000     --HOLE--

.const     0    8f000000    00005126     
                  8f000000    000033fb     EVM_C6674_configuration_pe66.oe66 (.const:xdc_runtime_Text_charTab__A)
                  8f0033fb    00000001     EVM_C6674_configuration_pe66.oe66 (.const:ti_sysbios_timers_timer64_Timer_localTimerBaseId__C)
                  8f0033fc    00000904     sysbios.ae66 : BIOS.obj (.const:.string)
                  8f003d00    00000400     EVM_C6674_configuration_pe66.oe66 (.const:ti_sysbios_family_c66_Cache_marvalues__C)
                  8f004100    000001c4     EVM_C6674_configuration_pe66.oe66 (.const:xdc_runtime_Text_nodeTab__A)
                  8f0042c4    00000004     ti.targets.rts6000.ae66 : Assert.oe66 (.const:.string)
                  8f0042c8    00000140     EVM_C6674_configuration_pe66.oe66 (.const:ti_sysbios_family_c66_tci66xx_CpIntc_sysIntToHostInt__A)
                  8f004408    00000101     rts6600_elf.lib : ctype.obj (.const:.string:_ctypes_)
                  8f004509    00000001     --HOLE-- [fill = 0]
                  8f00450a    00000002     EVM_C6674_configuration_pe66.oe66 (.const:ti_sdo_ipc_Notify_Module__id__C)
                  8f00450c    000000ff     EVM_C6674_configuration_pe66.oe66 (.const:.string)
                  8f00460b    00000001     --HOLE-- [fill = 0]
                  8f00460c    00000060     EVM_C6674_configuration_pe66.oe66 (.const:ti_uia_loggers_LoggerStopMode_Module__FXNS__C)
                  8f00466c    00000058     ti.targets.rts6000.ae66 : Error.oe66 (.const:.string)
                  8f0046c4    00000004     EVM_C6674_configuration_pe66.oe66 (.const:ti_sdo_ipc_Ipc_A_nullArgument__C)
                  8f0046c8    0000004c     EVM_C6674_configuration_pe66.oe66 (.const:xdc_runtime_Startup_sfxnTab__A)
                  8f004714    00000040     ti.targets.rts6000.ae66 : Text.oe66 (.const:.string)
                  8f004754    0000003c     EVM_C6674_configuration_pe66.oe66 (.const:xdc_runtime_LoggerBuf_Module__FXNS__C)
                  8f004790    00000030     EVM_C6674_configuration_pe66.oe66 (.const:ti_uia_loggers_LoggerStopMode_Object__PARAMS__C)
                  8f0047c0    0000002c     ti.targets.rts6000.ae66 : Startup.oe66 (.const:.string)
                  8f0047ec    00000028     EVM_C6674_configuration_pe66.oe66 (.const:ti_sysbios_heaps_HeapMem_Module__FXNS__C)
                  8f004814    00000028     EVM_C6674_configuration_pe66.oe66 (.const:xdc_runtime_LoggerBuf_Object__PARAMS__C)
                  8f00483c    00000004     EVM_C6674_configuration_pe66.oe66 (.const:ti_sdo_ipc_MessageQ_Object__count__C)
                  8f004840    00000026     EVM_C6674_configuration_pe66.oe66 (.const:xdc_runtime_Startup_sfxnRts__A)
                  8f004866    00000002     EVM_C6674_configuration_pe66.oe66 (.const:ti_sdo_ipc_Notify_numLines__C)
                  8f004868    00000024     EVM_C6674_configuration_pe66.oe66 (.const:ti_sysbios_gates_GateAll_Module__FXNS__C)
                  8f00488c    00000024     EVM_C6674_configuration_pe66.oe66 (.const:ti_sysbios_gates_GateHwi_Module__FXNS__C)
                  8f0048b0    00000024     EVM_C6674_configuration_pe66.oe66 (.const:ti_sysbios_gates_GateMutexPri_Module__FXNS__C)
                  8f0048d4    00000024     EVM_C6674_configuration_pe66.oe66 (.const:ti_sysbios_gates_GateMutex_Module__FXNS__C)
                  8f0048f8    00000024     EVM_C6674_configuration_pe66.oe66 (.const:ti_sysbios_gates_GateSwi_Module__FXNS__C)
                  8f00491c    00000024     EVM_C6674_configuration_pe66.oe66 (.const:ti_sysbios_heaps_HeapMem_Object__PARAMS__C)
                  8f004940    00000024     EVM_C6674_configuration_pe66.oe66 (.const:ti_sysbios_knl_Semaphore_Object__PARAMS__C)
                  8f004964    00000024     EVM_C6674_configuration_pe66.oe66 (.const:xdc_runtime_GateNull_Module__FXNS__C)
                  8f004988    00000024     EVM_C6674_configuration_pe66.oe66 (.const:xdc_runtime_knl_GateThread_Module__FXNS__C)
                  8f0049ac    00000023     rts6600_elf.lib : _printfi.obj (.const:.string)
                  8f0049cf    00000001     --HOLE-- [fill = 0]
                  8f0049d0    00000020     EVM_C6674_configuration_pe66.oe66 (.const:ti_sdo_ipc_Notify_Object__DESC__C)
                  8f0049f0    00000020     EVM_C6674_configuration_pe66.oe66 (.const:ti_sdo_utils_List_Object__DESC__C)
                  8f004a10    00000020     EVM_C6674_configuration_pe66.oe66 (.const:ti_sdo_utils_MultiProc_nameList__A)
                  8f004a30    00000020     EVM_C6674_configuration_pe66.oe66 (.const:ti_sysbios_gates_GateAll_Object__DESC__C)
                  8f004a50    00000020     EVM_C6674_configuration_pe66.oe66 (.const:ti_sysbios_gates_GateHwi_Object__DESC__C)
                  8f004a70    00000020     EVM_C6674_configuration_pe66.oe66 (.const:ti_sysbios_gates_GateMutexPri_Object__DESC__C)
                  8f004a90    00000020     EVM_C6674_configuration_pe66.oe66 (.const:ti_sysbios_gates_GateMutex_Object__DESC__C)
                  8f004ab0    00000020     EVM_C6674_configuration_pe66.oe66 (.const:ti_sysbios_gates_GateSwi_Object__DESC__C)
                  8f004ad0    00000020     EVM_C6674_configuration_pe66.oe66 (.const:ti_sysbios_heaps_HeapMem_Object__DESC__C)
                  8f004af0    00000020     EVM_C6674_configuration_pe66.oe66 (.const:ti_sysbios_knl_Queue_Object__DESC__C)
                  8f004b10    00000020     EVM_C6674_configuration_pe66.oe66 (.const:ti_sysbios_knl_Semaphore_Object__DESC__C)
                  8f004b30    00000020     EVM_C6674_configuration_pe66.oe66 (.const:ti_sysbios_xdcruntime_GateThreadSupport_Object__DESC__C)
                  8f004b50    00000020     EVM_C6674_configuration_pe66.oe66 (.const:ti_uia_loggers_LoggerStopMode_Object__DESC__C)
                  8f004b70    00000020     EVM_C6674_configuration_pe66.oe66 (.const:xdc_runtime_GateNull_Object__DESC__C)
                  8f004b90    00000020     EVM_C6674_configuration_pe66.oe66 (.const:xdc_runtime_LoggerBuf_Object__DESC__C)
                  8f004bb0    00000020     EVM_C6674_configuration_pe66.oe66 (.const:xdc_runtime_knl_GateThread_Object__DESC__C)
                  8f004bd0    00000018     EVM_C6674_configuration_pe66.oe66 (.const:ti_sdo_ipc_Notify_Object__PARAMS__C)
                  8f004be8    00000018     EVM_C6674_configuration_pe66.oe66 (.const:ti_sdo_utils_List_Object__PARAMS__C)
                  8f004c00    00000018     EVM_C6674_configuration_pe66.oe66 (.const:ti_sysbios_gates_GateAll_Object__PARAMS__C)
                  8f004c18    00000018     EVM_C6674_configuration_pe66.oe66 (.const:ti_sysbios_gates_GateHwi_Object__PARAMS__C)
                  8f004c30    00000018     EVM_C6674_configuration_pe66.oe66 (.const:ti_sysbios_gates_GateMutexPri_Object__PARAMS__C)
                  8f004c48    00000018     EVM_C6674_configuration_pe66.oe66 (.const:ti_sysbios_gates_GateMutex_Object__PARAMS__C)
                  8f004c60    00000018     EVM_C6674_configuration_pe66.oe66 (.const:ti_sysbios_gates_GateSwi_Object__PARAMS__C)
                  8f004c78    00000018     EVM_C6674_configuration_pe66.oe66 (.const:ti_sysbios_knl_Queue_Object__PARAMS__C)
                  8f004c90    00000018     EVM_C6674_configuration_pe66.oe66 (.const:ti_sysbios_knl_Swi_hooks__A)
                  8f004ca8    00000018     EVM_C6674_configuration_pe66.oe66 (.const:ti_sysbios_knl_Task_hooks__A)
                  8f004cc0    00000018     EVM_C6674_configuration_pe66.oe66 (.const:ti_sysbios_xdcruntime_GateThreadSupport_Object__PARAMS__C)
                  8f004cd8    00000018     EVM_C6674_configuration_pe66.oe66 (.const:xdc_runtime_GateNull_Object__PARAMS__C)
                  8f004cf0    00000018     EVM_C6674_configuration_pe66.oe66 (.const:xdc_runtime_knl_GateThread_Object__PARAMS__C)
                  8f004d08    00000014     hello.obj (.const:.string)
                  8f004d1c    00000004     EVM_C6674_configuration_pe66.oe66 (.const:ti_sdo_ipc_Notify_A_alreadyRegistered__C)
                  8f004d20    00000014     EVM_C6674_configuration_pe66.oe66 (.const:ti_sysbios_family_c64p_Hwi_hooks__A)
                  8f004d34    00000004     EVM_C6674_configuration_pe66.oe66 (.const:ti_sdo_ipc_Notify_A_invArgument__C)
                  8f004d38    00000011     ti.targets.rts6000.ae66 : System.oe66 (.const:.string:digtohex)
                  8f004d49    00000001     --HOLE-- [fill = 0]
                  8f004d4a    00000002     EVM_C6674_configuration_pe66.oe66 (.const:ti_sdo_ipc_SharedRegion_Module__id__C)
                  8f004d4c    00000004     EVM_C6674_configuration_pe66.oe66 (.const:ti_sdo_ipc_Notify_Module__diagsEnabled__C)
                  8f004d50    00000010     EVM_C6674_configuration_pe66.oe66 (.const:ti_sdo_ipc_family_c647x_MultiProcSetup_procMap__A)
                  8f004d60    00000010     EVM_C6674_configuration_pe66.oe66 (.const:xdc_runtime_Startup_firstFxns__A)
                  8f004d70    00000008     ti.targets.rts6000.ae66 : System.oe66 (.const:.string)
                  8f004d78    00000008     EVM_C6674_configuration_pe66.oe66 (.const:ti_sysbios_family_c64p_Hwi_hooks__C)
                  8f004d80    00000008     EVM_C6674_configuration_pe66.oe66 (.const:ti_sysbios_knl_Idle_funcList__A)
                  8f004d88    00000008     EVM_C6674_configuration_pe66.oe66 (.const:ti_sysbios_knl_Idle_funcList__C)
                  8f004d90    00000008     EVM_C6674_configuration_pe66.oe66 (.const:ti_sysbios_knl_Swi_hooks__C)
                  8f004d98    00000008     EVM_C6674_configuration_pe66.oe66 (.const:ti_sysbios_knl_Task_hooks__C)
                  8f004da0    00000008     EVM_C6674_configuration_pe66.oe66 (.const:xdc_runtime_Startup_firstFxns__C)
                  8f004da8    00000008     EVM_C6674_configuration_pe66.oe66 (.const:xdc_runtime_Startup_lastFxns__C)
                  8f004db0    00000004     EVM_C6674_configuration_pe66.oe66 (.const:ti_sdo_ipc_Notify_Module__diagsIncluded__C)
                  8f004db4    00000004     EVM_C6674_configuration_pe66.oe66 (.const:ti_sdo_ipc_Notify_Module__diagsMask__C)
                  8f004db8    00000004     EVM_C6674_configuration_pe66.oe66 (.const:ti_sdo_ipc_Notify_Object__heap__C)
                  8f004dbc    00000004     EVM_C6674_configuration_pe66.oe66 (.const:ti_sdo_ipc_Notify_numEvents__C)
                  8f004dc0    00000004     EVM_C6674_configuration_pe66.oe66 (.const:ti_sdo_ipc_SharedRegion_A_idTooLarge__C)
                  8f004dc4    00000004     EVM_C6674_configuration_pe66.oe66 (.const:ti_sdo_ipc_SharedRegion_Module__diagsEnabled__C)
                  8f004dc8    00000004     EVM_C6674_configuration_pe66.oe66 (.const:ti_sdo_ipc_SharedRegion_Module__diagsIncluded__C)
                  8f004dcc    00000004     EVM_C6674_configuration_pe66.oe66 (.const:ti_sdo_ipc_SharedRegion_Module__diagsMask__C)
                  8f004dd0    00000004     EVM_C6674_configuration_pe66.oe66 (.const:ti_sdo_ipc_family_c647x_Interrupt_KICK0__C)
                  8f004dd4    00000004     EVM_C6674_configuration_pe66.oe66 (.const:ti_sdo_ipc_family_c647x_Interrupt_KICK1__C)
                  8f004dd8    00000004     EVM_C6674_configuration_pe66.oe66 (.const:ti_sdo_ipc_family_c647x_MultiProcSetup_A_invalidProcessor__C)
                  8f004ddc    00000004     EVM_C6674_configuration_pe66.oe66 (.const:ti_sdo_ipc_family_c647x_MultiProcSetup_Module__diagsEnabled__C)
                  8f004de0    00000004     EVM_C6674_configuration_pe66.oe66 (.const:ti_sdo_ipc_family_c647x_MultiProcSetup_Module__diagsIncluded__C)
                  8f004de4    00000004     EVM_C6674_configuration_pe66.oe66 (.const:ti_sdo_ipc_family_c647x_MultiProcSetup_Module__diagsMask__C)
                  8f004de8    00000004     EVM_C6674_configuration_pe66.oe66 (.const:ti_sdo_ipc_family_c647x_MultiProcSetup_procMap__C)
                  8f004dec    00000004     EVM_C6674_configuration_pe66.oe66 (.const:ti_sdo_ipc_gates_GateHWSem_baseAddr__C)
                  8f004df0    00000004     EVM_C6674_configuration_pe66.oe66 (.const:ti_sdo_ipc_gates_GateHWSem_numSems__C)
                  8f004df4    00000004     EVM_C6674_configuration_pe66.oe66 (.const:ti_sdo_ipc_gates_GateHWSem_reservedMaskArr__C)
                  8f004df8    00000004     EVM_C6674_configuration_pe66.oe66 (.const:ti_sdo_ipc_gates_GateHWSem_reservedMaskArr__A)
                  8f004dfc    00000004     EVM_C6674_configuration_pe66.oe66 (.const:ti_sdo_utils_MultiProc_A_invalidMultiProcId__C)
                  8f004e00    00000004     EVM_C6674_configuration_pe66.oe66 (.const:ti_sdo_utils_MultiProc_A_invalidProcName__C)
                  8f004e04    00000004     EVM_C6674_configuration_pe66.oe66 (.const:ti_sdo_utils_MultiProc_Module__diagsEnabled__C)
                  8f004e08    00000004     EVM_C6674_configuration_pe66.oe66 (.const:ti_sdo_utils_MultiProc_Module__diagsIncluded__C)
                  8f004e0c    00000004     EVM_C6674_configuration_pe66.oe66 (.const:ti_sdo_utils_MultiProc_Module__diagsMask__C)
                  8f004e10    00000004     EVM_C6674_configuration_pe66.oe66 (.const:ti_sdo_utils_MultiProc_nameList__C)
                  8f004e14    00000004     EVM_C6674_configuration_pe66.oe66 (.const:ti_sdo_utils_NameServer_Instance_State_freeList__O)
                  8f004e18    00000004     EVM_C6674_configuration_pe66.oe66 (.const:ti_sdo_utils_NameServer_Object__count__C)
                  8f004e1c    00000004     EVM_C6674_configuration_pe66.oe66 (.const:ti_sysbios_family_c64p_Exception_E_exceptionMax__C)
                  8f004e20    00000004     EVM_C6674_configuration_pe66.oe66 (.const:ti_sysbios_family_c64p_Exception_exceptionHook__C)
                  8f004e24    00000004     EVM_C6674_configuration_pe66.oe66 (.const:ti_sysbios_family_c64p_Exception_externalHook__C)
                  8f004e28    00000004     EVM_C6674_configuration_pe66.oe66 (.const:ti_sysbios_family_c64p_Exception_internalHook__C)
                  8f004e2c    00000004     EVM_C6674_configuration_pe66.oe66 (.const:ti_sysbios_family_c64p_Exception_nmiHook__C)
                  8f004e30    00000004     EVM_C6674_configuration_pe66.oe66 (.const:ti_sysbios_family_c64p_Hwi_LD_end__C)
                  8f004e34    00000004     EVM_C6674_configuration_pe66.oe66 (.const:ti_sysbios_family_c64p_Hwi_LM_begin__C)
                  8f004e38    00000004     EVM_C6674_configuration_pe66.oe66 (.const:ti_sysbios_family_c64p_Hwi_Module__diagsEnabled__C)
                  8f004e3c    00000004     EVM_C6674_configuration_pe66.oe66 (.const:ti_sysbios_family_c64p_Hwi_Module__diagsIncluded__C)
                  8f004e40    00000004     EVM_C6674_configuration_pe66.oe66 (.const:ti_sysbios_family_c64p_Hwi_Module__diagsMask__C)
                  8f004e44    00000004     EVM_C6674_configuration_pe66.oe66 (.const:ti_sysbios_family_c64p_Hwi_Module__loggerFxn1__C)
                  8f004e48    00000004     EVM_C6674_configuration_pe66.oe66 (.const:ti_sysbios_family_c64p_Hwi_Module__loggerFxn8__C)
                  8f004e4c    00000004     EVM_C6674_configuration_pe66.oe66 (.const:ti_sysbios_family_c64p_Hwi_Module__loggerObj__C)
                  8f004e50    00000004     EVM_C6674_configuration_pe66.oe66 (.const:ti_sysbios_family_c66_Cache_E_invalidL1CacheSize__C)
                  8f004e54    00000004     EVM_C6674_configuration_pe66.oe66 (.const:ti_sysbios_family_c66_Cache_E_invalidL2CacheSize__C)
                  8f004e58    00000004     EVM_C6674_configuration_pe66.oe66 (.const:ti_sysbios_family_c66_Cache_atomicBlockSize__C)
                  8f004e5c    00000004     EVM_C6674_configuration_pe66.oe66 (.const:ti_sysbios_family_c66_tci66xx_CpIntc_E_unpluggedSysInt__C)
                  8f004e60    00000004     EVM_C6674_configuration_pe66.oe66 (.const:ti_sysbios_family_c66_tci66xx_CpIntc_numStatusRegs__C)
                  8f004e64    00000004     EVM_C6674_configuration_pe66.oe66 (.const:ti_sysbios_family_c66_tci66xx_CpIntc_numSysInts__C)
                  8f004e68    00000004     EVM_C6674_configuration_pe66.oe66 (.const:ti_sysbios_family_c66_tci66xx_CpIntc_sysIntToHostInt__C)
                  8f004e6c    00000004     EVM_C6674_configuration_pe66.oe66 (.const:ti_sysbios_gates_GateMutexPri_A_badContext__C)
                  8f004e70    00000004     EVM_C6674_configuration_pe66.oe66 (.const:ti_sysbios_gates_GateMutexPri_A_enterTaskDisabled__C)
                  8f004e74    00000004     EVM_C6674_configuration_pe66.oe66 (.const:ti_sysbios_gates_GateMutexPri_Instance_State_pendQ__O)
                  8f004e78    00000004     EVM_C6674_configuration_pe66.oe66 (.const:ti_sysbios_gates_GateMutexPri_Module__diagsEnabled__C)
                  8f004e7c    00000004     EVM_C6674_configuration_pe66.oe66 (.const:ti_sysbios_gates_GateMutexPri_Module__diagsIncluded__C)
                  8f004e80    00000004     EVM_C6674_configuration_pe66.oe66 (.const:ti_sysbios_gates_GateMutexPri_Module__diagsMask__C)
                  8f004e84    00000004     EVM_C6674_configuration_pe66.oe66 (.const:ti_sysbios_gates_GateMutex_A_badContext__C)
                  8f004e88    00000004     EVM_C6674_configuration_pe66.oe66 (.const:ti_sysbios_gates_GateMutex_Instance_State_sem__O)
                  8f004e8c    00000004     EVM_C6674_configuration_pe66.oe66 (.const:ti_sysbios_gates_GateMutex_Module__diagsEnabled__C)
                  8f004e90    00000004     EVM_C6674_configuration_pe66.oe66 (.const:ti_sysbios_gates_GateMutex_Module__diagsIncluded__C)
                  8f004e94    00000004     EVM_C6674_configuration_pe66.oe66 (.const:ti_sysbios_gates_GateMutex_Module__diagsMask__C)
                  8f004e98    00000004     EVM_C6674_configuration_pe66.oe66 (.const:ti_sysbios_gates_GateSwi_A_badContext__C)
                  8f004e9c    00000004     EVM_C6674_configuration_pe66.oe66 (.const:ti_sysbios_gates_GateSwi_Module__diagsEnabled__C)
                  8f004ea0    00000004     EVM_C6674_configuration_pe66.oe66 (.const:ti_sysbios_gates_GateSwi_Module__diagsIncluded__C)
                  8f004ea4    00000004     EVM_C6674_configuration_pe66.oe66 (.const:ti_sysbios_gates_GateSwi_Module__diagsMask__C)
                  8f004ea8    00000004     EVM_C6674_configuration_pe66.oe66 (.const:ti_sysbios_hal_Hwi_E_stackOverflow__C)
                  8f004eac    00000004     EVM_C6674_configuration_pe66.oe66 (.const:ti_sysbios_heaps_HeapMem_A_align__C)
                  8f004eb0    00000004     EVM_C6674_configuration_pe66.oe66 (.const:ti_sysbios_heaps_HeapMem_A_heapSize__C)
                  8f004eb4    00000004     EVM_C6674_configuration_pe66.oe66 (.const:ti_sysbios_heaps_HeapMem_A_invalidFree__C)
                  8f004eb8    00000004     EVM_C6674_configuration_pe66.oe66 (.const:ti_sysbios_heaps_HeapMem_A_zeroBlock__C)
                  8f004ebc    00000004     EVM_C6674_configuration_pe66.oe66 (.const:ti_sysbios_heaps_HeapMem_E_memory__C)
                  8f004ec0    00000004     EVM_C6674_configuration_pe66.oe66 (.const:ti_sysbios_heaps_HeapMem_Module__diagsEnabled__C)
                  8f004ec4    00000004     EVM_C6674_configuration_pe66.oe66 (.const:ti_sysbios_heaps_HeapMem_Module__diagsIncluded__C)
                  8f004ec8    00000004     EVM_C6674_configuration_pe66.oe66 (.const:ti_sysbios_heaps_HeapMem_Module__diagsMask__C)
                  8f004ecc    00000004     EVM_C6674_configuration_pe66.oe66 (.const:ti_sysbios_heaps_HeapMem_Module__gateObj__C)
                  8f004ed0    00000004     EVM_C6674_configuration_pe66.oe66 (.const:ti_sysbios_heaps_HeapMem_Object__count__C)
                  8f004ed4    00000004     EVM_C6674_configuration_pe66.oe66 (.const:ti_sysbios_heaps_HeapMem_reqAlign__C)
                  8f004ed8    00000004     EVM_C6674_configuration_pe66.oe66 (.const:ti_sysbios_knl_Clock_LM_begin__C)
                  8f004edc    00000004     EVM_C6674_configuration_pe66.oe66 (.const:ti_sysbios_knl_Clock_LM_tick__C)
                  8f004ee0    00000004     EVM_C6674_configuration_pe66.oe66 (.const:ti_sysbios_knl_Clock_LW_delayed__C)
                  8f004ee4    00000004     EVM_C6674_configuration_pe66.oe66 (.const:ti_sysbios_knl_Clock_Module_State_clockQ__O)
                  8f004ee8    00000004     EVM_C6674_configuration_pe66.oe66 (.const:ti_sysbios_knl_Clock_Module__diagsEnabled__C)
                  8f004eec    00000004     EVM_C6674_configuration_pe66.oe66 (.const:ti_sysbios_knl_Clock_Module__diagsIncluded__C)
                  8f004ef0    00000004     EVM_C6674_configuration_pe66.oe66 (.const:ti_sysbios_knl_Clock_Module__diagsMask__C)
                  8f004ef4    00000004     EVM_C6674_configuration_pe66.oe66 (.const:ti_sysbios_knl_Clock_Module__loggerFxn1__C)
                  8f004ef8    00000004     EVM_C6674_configuration_pe66.oe66 (.const:ti_sysbios_knl_Clock_Module__loggerFxn2__C)
                  8f004efc    00000004     EVM_C6674_configuration_pe66.oe66 (.const:ti_sysbios_knl_Clock_Module__loggerObj__C)
                  8f004f00    00000004     EVM_C6674_configuration_pe66.oe66 (.const:ti_sysbios_knl_Semaphore_A_badContext__C)
                  8f004f04    00000004     EVM_C6674_configuration_pe66.oe66 (.const:ti_sysbios_knl_Semaphore_A_noEvents__C)
                  8f004f08    00000004     EVM_C6674_configuration_pe66.oe66 (.const:ti_sysbios_knl_Semaphore_A_overflow__C)
                  8f004f0c    00000004     EVM_C6674_configuration_pe66.oe66 (.const:ti_sysbios_knl_Semaphore_A_pendTaskDisabled__C)
                  8f004f10    00000004     EVM_C6674_configuration_pe66.oe66 (.const:ti_sysbios_knl_Semaphore_Instance_State_pendQ__O)
                  8f004f14    00000004     EVM_C6674_configuration_pe66.oe66 (.const:ti_sysbios_knl_Semaphore_LM_pend__C)
                  8f004f18    00000004     EVM_C6674_configuration_pe66.oe66 (.const:ti_sysbios_knl_Semaphore_LM_post__C)
                  8f004f1c    00000004     EVM_C6674_configuration_pe66.oe66 (.const:ti_sysbios_knl_Semaphore_Module__diagsEnabled__C)
                  8f004f20    00000004     EVM_C6674_configuration_pe66.oe66 (.const:ti_sysbios_knl_Semaphore_Module__diagsIncluded__C)
                  8f004f24    00000004     EVM_C6674_configuration_pe66.oe66 (.const:ti_sysbios_knl_Semaphore_Module__diagsMask__C)
                  8f004f28    00000004     EVM_C6674_configuration_pe66.oe66 (.const:ti_sysbios_knl_Semaphore_Module__loggerFxn2__C)
                  8f004f2c    00000004     EVM_C6674_configuration_pe66.oe66 (.const:ti_sysbios_knl_Semaphore_Module__loggerFxn4__C)
                  8f004f30    00000004     EVM_C6674_configuration_pe66.oe66 (.const:ti_sysbios_knl_Semaphore_Module__loggerObj__C)
                  8f004f34    00000004     EVM_C6674_configuration_pe66.oe66 (.const:ti_sysbios_knl_Swi_LD_end__C)
                  8f004f38    00000004     EVM_C6674_configuration_pe66.oe66 (.const:ti_sysbios_knl_Swi_LM_begin__C)
                  8f004f3c    00000004     EVM_C6674_configuration_pe66.oe66 (.const:ti_sysbios_knl_Swi_LM_post__C)
                  8f004f40    00000004     EVM_C6674_configuration_pe66.oe66 (.const:ti_sysbios_knl_Swi_Module__diagsEnabled__C)
                  8f004f44    00000004     EVM_C6674_configuration_pe66.oe66 (.const:ti_sysbios_knl_Swi_Module__diagsIncluded__C)
                  8f004f48    00000004     EVM_C6674_configuration_pe66.oe66 (.const:ti_sysbios_knl_Swi_Module__diagsMask__C)
                  8f004f4c    00000004     EVM_C6674_configuration_pe66.oe66 (.const:ti_sysbios_knl_Swi_Module__loggerFxn1__C)
                  8f004f50    00000004     EVM_C6674_configuration_pe66.oe66 (.const:ti_sysbios_knl_Swi_Module__loggerFxn4__C)
                  8f004f54    00000004     EVM_C6674_configuration_pe66.oe66 (.const:ti_sysbios_knl_Swi_Module__loggerObj__C)
                  8f004f58    00000004     EVM_C6674_configuration_pe66.oe66 (.const:ti_sysbios_knl_Swi_Object__count__C)
                  8f004f5c    00000004     EVM_C6674_configuration_pe66.oe66 (.const:ti_sysbios_knl_Swi_numConstructedSwis__C)
                  8f004f60    00000004     EVM_C6674_configuration_pe66.oe66 (.const:ti_sysbios_knl_Task_A_badPriority__C)
                  8f004f64    00000004     EVM_C6674_configuration_pe66.oe66 (.const:ti_sysbios_knl_Task_E_spOutOfBounds__C)
                  8f004f68    00000004     EVM_C6674_configuration_pe66.oe66 (.const:ti_sysbios_knl_Task_E_stackOverflow__C)
                  8f004f6c    00000004     EVM_C6674_configuration_pe66.oe66 (.const:ti_sysbios_knl_Task_LD_block__C)
                  8f004f70    00000004     EVM_C6674_configuration_pe66.oe66 (.const:ti_sysbios_knl_Task_LD_exit__C)
                  8f004f74    00000004     EVM_C6674_configuration_pe66.oe66 (.const:ti_sysbios_knl_Task_LD_ready__C)
                  8f004f78    00000004     EVM_C6674_configuration_pe66.oe66 (.const:ti_sysbios_knl_Task_LM_setPri__C)
                  8f004f7c    00000004     EVM_C6674_configuration_pe66.oe66 (.const:ti_sysbios_knl_Task_LM_switch__C)
                  8f004f80    00000004     EVM_C6674_configuration_pe66.oe66 (.const:ti_sysbios_knl_Task_Module_State_inactiveQ__O)
                  8f004f84    00000004     EVM_C6674_configuration_pe66.oe66 (.const:ti_sysbios_knl_Task_Module__diagsEnabled__C)
                  8f004f88    00000004     EVM_C6674_configuration_pe66.oe66 (.const:ti_sysbios_knl_Task_Module__diagsIncluded__C)
                  8f004f8c    00000004     EVM_C6674_configuration_pe66.oe66 (.const:ti_sysbios_knl_Task_Module__diagsMask__C)
                  8f004f90    00000004     EVM_C6674_configuration_pe66.oe66 (.const:ti_sysbios_knl_Task_Module__loggerFxn2__C)
                  8f004f94    00000004     EVM_C6674_configuration_pe66.oe66 (.const:ti_sysbios_knl_Task_Module__loggerFxn4__C)
                  8f004f98    00000004     EVM_C6674_configuration_pe66.oe66 (.const:ti_sysbios_knl_Task_Module__loggerObj__C)
                  8f004f9c    00000004     EVM_C6674_configuration_pe66.oe66 (.const:ti_sysbios_knl_Task_Object__count__C)
                  8f004fa0    00000004     EVM_C6674_configuration_pe66.oe66 (.const:ti_sysbios_knl_Task_Object__heap__C)
                  8f004fa4    00000004     EVM_C6674_configuration_pe66.oe66 (.const:ti_sysbios_knl_Task_allBlockedFunc__C)
                  8f004fa8    00000004     EVM_C6674_configuration_pe66.oe66 (.const:ti_sysbios_knl_Task_numConstructedTasks__C)
                  8f004fac    00000004     EVM_C6674_configuration_pe66.oe66 (.const:ti_sysbios_timers_timer64_Timer_A_notAvailable__C)
                  8f004fb0    00000004     EVM_C6674_configuration_pe66.oe66 (.const:ti_sysbios_timers_timer64_Timer_E_cannotSupport__C)
                  8f004fb4    00000004     EVM_C6674_configuration_pe66.oe66 (.const:ti_sysbios_timers_timer64_Timer_Module__diagsEnabled__C)
                  8f004fb8    00000004     EVM_C6674_configuration_pe66.oe66 (.const:ti_sysbios_timers_timer64_Timer_Module__diagsIncluded__C)
                  8f004fbc    00000004     EVM_C6674_configuration_pe66.oe66 (.const:ti_sysbios_timers_timer64_Timer_Module__diagsMask__C)
                  8f004fc0    00000004     EVM_C6674_configuration_pe66.oe66 (.const:ti_sysbios_timers_timer64_Timer_anyMaskHigh__C)
                  8f004fc4    00000004     EVM_C6674_configuration_pe66.oe66 (.const:ti_sysbios_timers_timer64_Timer_anyMask__C)
                  8f004fc8    00000004     EVM_C6674_configuration_pe66.oe66 (.const:ti_sysbios_timers_timer64_Timer_freqDivisor__C)
                  8f004fcc    00000004     EVM_C6674_configuration_pe66.oe66 (.const:ti_sysbios_timers_timer64_Timer_numLocalTimers__C)
                  8f004fd0    00000004     EVM_C6674_configuration_pe66.oe66 (.const:ti_sysbios_timers_timer64_Timer_numTimerDevices__C)
                  8f004fd4    00000004     EVM_C6674_configuration_pe66.oe66 (.const:ti_sysbios_utils_Load_LS_cpuLoad__C)
                  8f004fd8    00000004     EVM_C6674_configuration_pe66.oe66 (.const:ti_sysbios_utils_Load_LS_hwiLoad__C)
                  8f004fdc    00000004     EVM_C6674_configuration_pe66.oe66 (.const:ti_sysbios_utils_Load_LS_swiLoad__C)
                  8f004fe0    00000004     EVM_C6674_configuration_pe66.oe66 (.const:ti_sysbios_utils_Load_LS_taskLoad__C)
                  8f004fe4    00000004     EVM_C6674_configuration_pe66.oe66 (.const:ti_sysbios_utils_Load_Module_State_taskList__O)
                  8f004fe8    00000004     EVM_C6674_configuration_pe66.oe66 (.const:ti_sysbios_utils_Load_Module__diagsEnabled__C)
                  8f004fec    00000004     EVM_C6674_configuration_pe66.oe66 (.const:ti_sysbios_utils_Load_Module__diagsIncluded__C)
                  8f004ff0    00000004     EVM_C6674_configuration_pe66.oe66 (.const:ti_sysbios_utils_Load_Module__diagsMask__C)
                  8f004ff4    00000004     EVM_C6674_configuration_pe66.oe66 (.const:ti_sysbios_utils_Load_Module__loggerFxn1__C)
                  8f004ff8    00000004     EVM_C6674_configuration_pe66.oe66 (.const:ti_sysbios_utils_Load_Module__loggerFxn2__C)
                  8f004ffc    00000004     EVM_C6674_configuration_pe66.oe66 (.const:ti_sysbios_utils_Load_Module__loggerFxn4__C)
                  8f005000    00000004     EVM_C6674_configuration_pe66.oe66 (.const:ti_sysbios_utils_Load_Module__loggerObj__C)
                  8f005004    00000004     EVM_C6674_configuration_pe66.oe66 (.const:ti_sysbios_utils_Load_postUpdate__C)
                  8f005008    00000004     EVM_C6674_configuration_pe66.oe66 (.const:ti_sysbios_utils_Load_windowInMs__C)
                  8f00500c    00000004     EVM_C6674_configuration_pe66.oe66 (.const:ti_sysbios_xdcruntime_GateThreadSupport_Instance_State_gate__O)
                  8f005010    00000004     EVM_C6674_configuration_pe66.oe66 (.const:ti_uia_loggers_LoggerStopMode_Module__diagsEnabled__C)
                  8f005014    00000004     EVM_C6674_configuration_pe66.oe66 (.const:ti_uia_loggers_LoggerStopMode_Module__diagsIncluded__C)
                  8f005018    00000004     EVM_C6674_configuration_pe66.oe66 (.const:ti_uia_loggers_LoggerStopMode_Module__diagsMask__C)
                  8f00501c    00000004     EVM_C6674_configuration_pe66.oe66 (.const:ti_uia_loggers_LoggerStopMode_Object__count__C)
                  8f005020    00000004     EVM_C6674_configuration_pe66.oe66 (.const:ti_uia_loggers_LoggerStopMode_numCores__C)
                  8f005024    00000004     EVM_C6674_configuration_pe66.oe66 (.const:ti_uia_runtime_ILoggerSnapshot_Interface__BASE__C)
                  8f005028    00000004     EVM_C6674_configuration_pe66.oe66 (.const:ti_uia_runtime_IUIATransfer_Interface__BASE__C)
                  8f00502c    00000004     EVM_C6674_configuration_pe66.oe66 (.const:xdc_runtime_Assert_E_assertFailed__C)
                  8f005030    00000004     EVM_C6674_configuration_pe66.oe66 (.const:xdc_runtime_Core_A_initializedParams__C)
                  8f005034    00000004     EVM_C6674_configuration_pe66.oe66 (.const:xdc_runtime_Core_Module__diagsEnabled__C)
                  8f005038    00000004     EVM_C6674_configuration_pe66.oe66 (.const:xdc_runtime_Core_Module__diagsIncluded__C)
                  8f00503c    00000004     EVM_C6674_configuration_pe66.oe66 (.const:xdc_runtime_Core_Module__diagsMask__C)
                  8f005040    00000004     EVM_C6674_configuration_pe66.oe66 (.const:xdc_runtime_Error_E_memory__C)
                  8f005044    00000004     EVM_C6674_configuration_pe66.oe66 (.const:xdc_runtime_Error_Module__diagsEnabled__C)
                  8f005048    00000004     EVM_C6674_configuration_pe66.oe66 (.const:xdc_runtime_Error_Module__diagsIncluded__C)
                  8f00504c    00000004     EVM_C6674_configuration_pe66.oe66 (.const:xdc_runtime_Error_Module__diagsMask__C)
                  8f005050    00000004     EVM_C6674_configuration_pe66.oe66 (.const:xdc_runtime_Error_Module__loggerFxn8__C)
                  8f005054    00000004     EVM_C6674_configuration_pe66.oe66 (.const:xdc_runtime_Error_Module__loggerObj__C)
                  8f005058    00000004     EVM_C6674_configuration_pe66.oe66 (.const:xdc_runtime_Error_policyFxn__C)
                  8f00505c    00000004     EVM_C6674_configuration_pe66.oe66 (.const:xdc_runtime_Error_policy__C)
                  8f005060    00000004     EVM_C6674_configuration_pe66.oe66 (.const:xdc_runtime_Error_raiseHook__C)
                  8f005064    00000004     EVM_C6674_configuration_pe66.oe66 (.const:xdc_runtime_IFilterLogger_Interface__BASE__C)
                  8f005068    00000004     EVM_C6674_configuration_pe66.oe66 (.const:xdc_runtime_IGateProvider_Interface__BASE__C)
                  8f00506c    00000004     EVM_C6674_configuration_pe66.oe66 (.const:xdc_runtime_IHeap_Interface__BASE__C)
                  8f005070    00000004     EVM_C6674_configuration_pe66.oe66 (.const:xdc_runtime_ILogger_Interface__BASE__C)
                  8f005074    00000004     EVM_C6674_configuration_pe66.oe66 (.const:xdc_runtime_IModule_Interface__BASE__C)
                  8f005078    00000004     EVM_C6674_configuration_pe66.oe66 (.const:xdc_runtime_Log_L_error__C)
                  8f00507c    00000004     EVM_C6674_configuration_pe66.oe66 (.const:xdc_runtime_LoggerBuf_E_badLevel__C)
                  8f005080    00000004     EVM_C6674_configuration_pe66.oe66 (.const:xdc_runtime_LoggerBuf_Module__gateObj__C)
                  8f005084    00000004     EVM_C6674_configuration_pe66.oe66 (.const:xdc_runtime_LoggerBuf_Object__count__C)
                  8f005088    00000004     EVM_C6674_configuration_pe66.oe66 (.const:xdc_runtime_LoggerBuf_statusLogger__C)
                  8f00508c    00000004     EVM_C6674_configuration_pe66.oe66 (.const:xdc_runtime_Memory_defaultHeapInstance__C)
                  8f005090    00000004     EVM_C6674_configuration_pe66.oe66 (.const:xdc_runtime_Startup_execImpl__C)
                  8f005094    00000004     EVM_C6674_configuration_pe66.oe66 (.const:xdc_runtime_Startup_maxPasses__C)
                  8f005098    00000004     EVM_C6674_configuration_pe66.oe66 (.const:xdc_runtime_Startup_sfxnRts__C)
                  8f00509c    00000004     EVM_C6674_configuration_pe66.oe66 (.const:xdc_runtime_Startup_sfxnTab__C)
                  8f0050a0    00000004     EVM_C6674_configuration_pe66.oe66 (.const:xdc_runtime_System_Module__gateObj__C)
                  8f0050a4    00000004     EVM_C6674_configuration_pe66.oe66 (.const:xdc_runtime_System_abortFxn__C)
                  8f0050a8    00000004     EVM_C6674_configuration_pe66.oe66 (.const:xdc_runtime_System_exitFxn__C)
                  8f0050ac    00000004     EVM_C6674_configuration_pe66.oe66 (.const:xdc_runtime_System_extendFxn__C)
                  8f0050b0    00000004     EVM_C6674_configuration_pe66.oe66 (.const:xdc_runtime_System_maxAtexitHandlers__C)
                  8f0050b4    00000004     EVM_C6674_configuration_pe66.oe66 (.const:xdc_runtime_Text_charTab__C)
                  8f0050b8    00000004     EVM_C6674_configuration_pe66.oe66 (.const:xdc_runtime_Text_nameEmpty__C)
                  8f0050bc    00000004     EVM_C6674_configuration_pe66.oe66 (.const:xdc_runtime_Text_nameStatic__C)
                  8f0050c0    00000004     EVM_C6674_configuration_pe66.oe66 (.const:xdc_runtime_Text_nameUnknown__C)
                  8f0050c4    00000004     EVM_C6674_configuration_pe66.oe66 (.const:xdc_runtime_Text_nodeTab__C)
                  8f0050c8    00000004     EVM_C6674_configuration_pe66.oe66 (.const:xdc_runtime_Text_visitRopeFxn__C)
                  8f0050cc    00000002     EVM_C6674_configuration_pe66.oe66 (.const:ti_sdo_ipc_SharedRegion_numEntries__C)
                  8f0050ce    00000002     EVM_C6674_configuration_pe66.oe66 (.const:ti_sdo_ipc_family_c647x_Interrupt_enableKick__C)
                  8f0050d0    00000002     EVM_C6674_configuration_pe66.oe66 (.const:ti_sdo_ipc_family_c647x_MultiProcSetup_Module__id__C)
                  8f0050d2    00000002     EVM_C6674_configuration_pe66.oe66 (.const:ti_sdo_utils_MultiProc_Module__id__C)
                  8f0050d4    00000002     EVM_C6674_configuration_pe66.oe66 (.const:ti_sdo_utils_MultiProc_numProcessors__C)
                  8f0050d6    00000002     EVM_C6674_configuration_pe66.oe66 (.const:ti_sdo_utils_MultiProc_numProcsInCluster__C)
                  8f0050d8    00000002     EVM_C6674_configuration_pe66.oe66 (.const:ti_sysbios_family_c64p_Exception_Module__id__C)
                  8f0050da    00000002     EVM_C6674_configuration_pe66.oe66 (.const:ti_sysbios_family_c64p_Exception_useInternalBuffer__C)
                  8f0050dc    00000002     EVM_C6674_configuration_pe66.oe66 (.const:ti_sysbios_family_c64p_Hwi_Module__id__C)
                  8f0050de    00000002     EVM_C6674_configuration_pe66.oe66 (.const:ti_sysbios_family_c64p_Hwi_Module__loggerDefined__C)
                  8f0050e0    00000002     EVM_C6674_configuration_pe66.oe66 (.const:ti_sysbios_family_c66_Cache_Module__id__C)
                  8f0050e2    00000002     EVM_C6674_configuration_pe66.oe66 (.const:ti_sysbios_family_c66_Cache_registerRTSSynch__C)
                  8f0050e4    00000002     EVM_C6674_configuration_pe66.oe66 (.const:ti_sysbios_family_c66_tci66xx_CpIntc_Module__id__C)
                  8f0050e6    00000002     EVM_C6674_configuration_pe66.oe66 (.const:ti_sysbios_gates_GateMutexPri_Module__id__C)
                  8f0050e8    00000002     EVM_C6674_configuration_pe66.oe66 (.const:ti_sysbios_gates_GateMutex_Module__id__C)
                  8f0050ea    00000002     EVM_C6674_configuration_pe66.oe66 (.const:ti_sysbios_gates_GateSwi_Module__id__C)
                  8f0050ec    00000002     EVM_C6674_configuration_pe66.oe66 (.const:ti_sysbios_hal_Hwi_Module__id__C)
                  8f0050ee    00000002     EVM_C6674_configuration_pe66.oe66 (.const:ti_sysbios_heaps_HeapMem_Module__id__C)
                  8f0050f0    00000002     EVM_C6674_configuration_pe66.oe66 (.const:ti_sysbios_knl_Clock_Module__id__C)
                  8f0050f2    00000002     EVM_C6674_configuration_pe66.oe66 (.const:ti_sysbios_knl_Clock_Module__loggerDefined__C)
                  8f0050f4    00000002     EVM_C6674_configuration_pe66.oe66 (.const:ti_sysbios_knl_Semaphore_Module__id__C)
                  8f0050f6    00000002     EVM_C6674_configuration_pe66.oe66 (.const:ti_sysbios_knl_Semaphore_Module__loggerDefined__C)
                  8f0050f8    00000002     EVM_C6674_configuration_pe66.oe66 (.const:ti_sysbios_knl_Swi_Module__id__C)
                  8f0050fa    00000002     EVM_C6674_configuration_pe66.oe66 (.const:ti_sysbios_knl_Swi_Module__loggerDefined__C)
                  8f0050fc    00000002     EVM_C6674_configuration_pe66.oe66 (.const:ti_sysbios_knl_Task_Module__id__C)
                  8f0050fe    00000002     EVM_C6674_configuration_pe66.oe66 (.const:ti_sysbios_knl_Task_Module__loggerDefined__C)
                  8f005100    00000002     EVM_C6674_configuration_pe66.oe66 (.const:ti_sysbios_timers_timer64_Timer_Module__id__C)
                  8f005102    00000002     EVM_C6674_configuration_pe66.oe66 (.const:ti_sysbios_timers_timer64_Timer_startupNeeded__C)
                  8f005104    00000002     EVM_C6674_configuration_pe66.oe66 (.const:ti_sysbios_timers_timer64_Timer_useTimer64pRegMap__C)
                  8f005106    00000002     EVM_C6674_configuration_pe66.oe66 (.const:ti_sysbios_utils_Load_Module__id__C)
                  8f005108    00000002     EVM_C6674_configuration_pe66.oe66 (.const:ti_sysbios_utils_Load_Module__loggerDefined__C)
                  8f00510a    00000002     EVM_C6674_configuration_pe66.oe66 (.const:ti_sysbios_utils_Load_autoAddTasks__C)
                  8f00510c    00000002     EVM_C6674_configuration_pe66.oe66 (.const:ti_sysbios_utils_Load_updateInIdle__C)
                  8f00510e    00000002     EVM_C6674_configuration_pe66.oe66 (.const:ti_uia_loggers_LoggerStopMode_Module__id__C)
                  8f005110    00000002     EVM_C6674_configuration_pe66.oe66 (.const:ti_uia_loggers_LoggerStopMode_isTimestampEnabled__C)
                  8f005112    00000002     EVM_C6674_configuration_pe66.oe66 (.const:xdc_runtime_Core_Module__id__C)
                  8f005114    00000002     EVM_C6674_configuration_pe66.oe66 (.const:xdc_runtime_Error_Module__loggerDefined__C)
                  8f005116    00000002     EVM_C6674_configuration_pe66.oe66 (.const:xdc_runtime_Error_maxDepth__C)
                  8f005118    00000002     EVM_C6674_configuration_pe66.oe66 (.const:xdc_runtime_LoggerBuf_Module__id__C)
                  8f00511a    00000002     EVM_C6674_configuration_pe66.oe66 (.const:xdc_runtime_LoggerBuf_filterByLevel__C)
                  8f00511c    00000002     EVM_C6674_configuration_pe66.oe66 (.const:xdc_runtime_Memory_Module__id__C)
                  8f00511e    00000002     EVM_C6674_configuration_pe66.oe66 (.const:xdc_runtime_Text_charCnt__C)
                  8f005120    00000002     EVM_C6674_configuration_pe66.oe66 (.const:xdc_runtime_Text_isLoaded__C)
                  8f005122    00000002     EVM_C6674_configuration_pe66.oe66 (.const:xdc_runtime_Text_registryModsLastId__C)
                  8f005124    00000002     EVM_C6674_configuration_pe66.oe66 (.const:xdc_runtime_Text_unnamedModsLastId__C)

.sysbios   0    8f005140    00000c00     
                  8f005140    00000280     ti.targets.rts6000.ae66 : LoggerBuf.oe66 (.text:xdc_runtime_LoggerBuf_write8__E)
                  8f0053c0    000001c0                             : LoggerBuf.oe66 (.text:xdc_runtime_LoggerBuf_write4__E)
                  8f005580    00000120                             : LoggerBuf.oe66 (.text:xdc_runtime_LoggerBuf_setFilterLevel__E)
                  8f0056a0    00000100                             : LoggerBuf.oe66 (.text:xdc_runtime_LoggerBuf_getFilterLevel__E)
                  8f0057a0    000000e0     EVM_C6674_configuration_pe66.oe66 (.text:xdc_runtime_LoggerBuf_Object__create__S)
                  8f005880    00000080     ti.targets.rts6000.ae66 : LoggerBuf.oe66 (.text:xdc_runtime_LoggerBuf_Instance_init__E)
                  8f005900    00000080                             : LoggerBuf.oe66 (.text:xdc_runtime_LoggerBuf_Module_startup__E)
                  8f005980    00000080                             : LoggerBuf.oe66 (.text:xdc_runtime_LoggerBuf_filterOutEvent__I)
                  8f005a00    00000060     EVM_C6674_configuration_pe66.oe66 (.text:xdc_runtime_LoggerBuf_Object__delete__S)
                  8f005a60    00000040     EVM_C6674_configuration_pe66.oe66 (.text:xdc_runtime_LoggerBuf_Handle__label__S)
                  8f005aa0    00000040     ti.targets.rts6000.ae66 : LoggerBuf.oe66 (.text:xdc_runtime_LoggerBuf_Instance_finalize__E)
                  8f005ae0    00000040     EVM_C6674_configuration_pe66.oe66 (.text:xdc_runtime_LoggerBuf_Object__get__S)
                  8f005b20    00000040     ti.targets.rts6000.ae66 : LoggerBuf.oe66 (.text:xdc_runtime_LoggerBuf_reset__E)
                  8f005b60    00000040                             : LoggerBuf.oe66 (.text:xdc_runtime_LoggerBuf_write0__E)
                  8f005ba0    00000020     EVM_C6674_configuration_pe66.oe66 (.text:xdc_runtime_LoggerBuf_Module_GateProxy_enter__E)
                  8f005bc0    00000020     EVM_C6674_configuration_pe66.oe66 (.text:xdc_runtime_LoggerBuf_Module_GateProxy_leave__E)
                  8f005be0    00000020     ti.targets.rts6000.ae66 : LoggerBuf.oe66 (.text:xdc_runtime_LoggerBuf_disable__E)
                  8f005c00    00000020                             : LoggerBuf.oe66 (.text:xdc_runtime_LoggerBuf_enable__E)
                  8f005c20    00000020                             : LoggerBuf.oe66 (.text:xdc_runtime_LoggerBuf_write1__E)
                  8f005c40    00000020                             : LoggerBuf.oe66 (.text:xdc_runtime_LoggerBuf_write2__E)
                  8f005c60    00000010     sysbios.ae66 : BIOS.obj ($Tramp$S$$ti_sysbios_family_c64p_TimestampProvider_get64__E)
                  8f005c70    00000010     ti.targets.rts6000.ae66 : Error.oe66 ($Tramp$S$$xdc_runtime_Error_init__E)
                  8f005c80    00000010                             : Error.oe66 ($Tramp$S$$xdc_runtime_Error_raiseX__E)
                  8f005c90    00000010                             : Core-mem.oe66 ($Tramp$S$$xdc_runtime_Core_createObject__I)
                  8f005ca0    00000010                             : Error.oe66 ($Tramp$S$$xdc_runtime_Error_check__E)
                  8f005cb0    00000010                             : Core-mem.oe66 ($Tramp$S$$xdc_runtime_Core_deleteObject__I)
                  8f005cc0    00000010                             : Memory.oe66 ($Tramp$S$$xdc_runtime_Memory_alloc__E)
                  8f005cd0    00000010                             : LoggerBuf.oe66 ($Tramp$S$$LoggerBuf_instanceStartup)
                  8f005ce0    00000010                             : Core-label.oe66 ($Tramp$S$$xdc_runtime_Core_assignLabel__I)
                  8f005cf0    00000010                             : Memory.oe66 ($Tramp$S$$xdc_runtime_Memory_free__E)
                  8f005d00    00000010     rts6600_elf.lib : memset.obj ($Tramp$S$$memset)
                  8f005d10    00000010     sysbios.ae66 : BIOS.obj ($Tramp$S$$ti_sysbios_gates_GateHwi_enter__E)
                  8f005d20    00000010                  : BIOS.obj ($Tramp$S$$ti_sysbios_gates_GateHwi_leave__E)
                  8f005d30    00000010     --HOLE-- [fill = 00000000]

boot       0    8f006000    00000400     
                  8f006000    000000a0     boot.ae66 : boot.oe66 (.text:_c_int00)
                  8f0060a0    00000010     sysbios.ae66 : BIOS.obj ($Tramp$S$$ti_sysbios_family_c66_Cache_startup__I)
                  8f0060b0    00000010     --HOLE-- [fill = 00000000]
                  8f0060c0    00000340     (<space>) [fill = 0]

.cinit     0    8f006400    00000f28     
                  8f006400    00000f01     (.cinit..fardata.load) [load image, compression = rle]
                  8f007301    00000003     --HOLE-- [fill = 0]
                  8f007304    00000009     (.cinit..neardata.load) [load image, compression = rle]
                  8f00730d    00000003     --HOLE-- [fill = 0]
                  8f007310    00000008     (__TI_handler_table)
                  8f007318    00000010     (__TI_cinit_table)

.sect_cine_data 
*          0    903c0000    0fc40000     UNINITIALIZED
                  903c0000    0fc40000     EVM_C6674_configuration_pe66.oe66 (.sect_cine_data)


LINKER GENERATED COPY TABLES

__TI_cinit_table @ 8f007318 records: 2, size/record: 8, table size: 16
	.fardata: load addr=8f006400, load size=00000f01 bytes, run addr=00810f68, run size=000018a4 bytes, compression=rle
	.neardata: load addr=8f007304, load size=00000009 bytes, run addr=0081280c, run size=00000008 bytes, compression=rle


LINKER GENERATED HANDLER TABLE

__TI_handler_table @ 8f007310 records: 2, size/record: 4, table size: 8
	index: 0, handler: __TI_decompress_rle24
	index: 1, handler: __TI_decompress_none


FAR CALL TRAMPOLINES

callee name               trampoline name
   callee addr  tramp addr   call addr  call info
--------------  -----------  ---------  ----------------
$.text:ti_sysbios_family_c64p_TimestampProvider_get64__E:sysbios.ae66<BIOS.obj>$0x0  $Tramp$S$$ti_sysbios_family_c64p_TimestampProvider_get64__E
   0c394d40     8f005c60     8f005298   ti.targets.rts6000.ae66 : LoggerBuf.oe66 (.text:xdc_runtime_LoggerBuf_write8__E)
                             8f0054f0                           : LoggerBuf.oe66 (.text:xdc_runtime_LoggerBuf_write4__E)
$.text:xdc_runtime_Error_init__E:ti.targets.rts6000.ae66<Error.oe66>$0x0  $Tramp$S$$xdc_runtime_Error_init__E
   0c394560     8f005c70     8f00561c   ti.targets.rts6000.ae66 : LoggerBuf.oe66 (.text:xdc_runtime_LoggerBuf_setFilterLevel__E)
                             8f005708                           : LoggerBuf.oe66 (.text:xdc_runtime_LoggerBuf_getFilterLevel__E)
$.text:xdc_runtime_Error_raiseX__E:ti.targets.rts6000.ae66<Error.oe66>$0x0  $Tramp$S$$xdc_runtime_Error_raiseX__E
   0c395420     8f005c80     8f005644   ti.targets.rts6000.ae66 : LoggerBuf.oe66 (.text:xdc_runtime_LoggerBuf_setFilterLevel__E)
                             8f005768                           : LoggerBuf.oe66 (.text:xdc_runtime_LoggerBuf_getFilterLevel__E)
$.text:xdc_runtime_Core_createObject__I:ti.targets.rts6000.ae66<Core-mem.oe66>$0x0  $Tramp$S$$xdc_runtime_Core_createObject__I
   0c389ac0     8f005c90     8f0057c8   EVM_C6674_configuration_pe66.oe66 (.text:xdc_runtime_LoggerBuf_Object__create__S)
$.text:xdc_runtime_Error_check__E:ti.targets.rts6000.ae66<Error.oe66>$0x0  $Tramp$S$$xdc_runtime_Error_check__E
   0c394520     8f005ca0     8f0057f0   EVM_C6674_configuration_pe66.oe66 (.text:xdc_runtime_LoggerBuf_Object__create__S)
$.text:xdc_runtime_Core_deleteObject__I:ti.targets.rts6000.ae66<Core-mem.oe66>$0x0  $Tramp$S$$xdc_runtime_Core_deleteObject__I
   0c38eac0     8f005cb0     8f005824   EVM_C6674_configuration_pe66.oe66 (.text:xdc_runtime_LoggerBuf_Object__create__S)
                             8f005a20   EVM_C6674_configuration_pe66.oe66 (.text:xdc_runtime_LoggerBuf_Object__delete__S)
$.text:xdc_runtime_Memory_alloc__E:ti.targets.rts6000.ae66<Memory.oe66>$0x0  $Tramp$S$$xdc_runtime_Memory_alloc__E
   0c3904a0     8f005cc0     8f0058a0   ti.targets.rts6000.ae66 : LoggerBuf.oe66 (.text:xdc_runtime_LoggerBuf_Instance_init__E)
$.text:LoggerBuf_instanceStartup:ti.targets.rts6000.ae66<LoggerBuf.oe66>$0x0  $Tramp$S$$LoggerBuf_instanceStartup
   0c3948e0     8f005cd0     8f0058c4   ti.targets.rts6000.ae66 : LoggerBuf.oe66 (.text:xdc_runtime_LoggerBuf_Instance_init__E)
                             8f005938                           : LoggerBuf.oe66 (.text:xdc_runtime_LoggerBuf_Module_startup__E)
$.text:xdc_runtime_Core_assignLabel__I:ti.targets.rts6000.ae66<Core-label.oe66>$0x0  $Tramp$S$$xdc_runtime_Core_assignLabel__I
   0c392b60     8f005ce0     8f005a80   EVM_C6674_configuration_pe66.oe66 (.text:xdc_runtime_LoggerBuf_Handle__label__S)
$.text:xdc_runtime_Memory_free__E:ti.targets.rts6000.ae66<Memory.oe66>$0x0  $Tramp$S$$xdc_runtime_Memory_free__E
   0c394660     8f005cf0     8f005aac   ti.targets.rts6000.ae66 : LoggerBuf.oe66 (.text:xdc_runtime_LoggerBuf_Instance_finalize__E)
$.text:memset:rts6600_elf.lib<memset.obj>$0x0  $Tramp$S$$memset
   0c390040     8f005d00     8f005b34   ti.targets.rts6000.ae66 : LoggerBuf.oe66 (.text:xdc_runtime_LoggerBuf_reset__E)
$.text:ti_sysbios_gates_GateHwi_enter__E:sysbios.ae66<BIOS.obj>$0x0  $Tramp$S$$ti_sysbios_gates_GateHwi_enter__E
   0c394e60     8f005d10     8f005ba0   EVM_C6674_configuration_pe66.oe66 (.text:xdc_runtime_LoggerBuf_Module_GateProxy_enter__E)
$.text:ti_sysbios_gates_GateHwi_leave__E:sysbios.ae66<BIOS.obj>$0x0  $Tramp$S$$ti_sysbios_gates_GateHwi_leave__E
   0c394e80     8f005d20     8f005bc0   EVM_C6674_configuration_pe66.oe66 (.text:xdc_runtime_LoggerBuf_Module_GateProxy_leave__E)
$.text:xdc_runtime_LoggerBuf_reset__E:ti.targets.rts6000.ae66<LoggerBuf.oe66>$0x0  $Tramp$S$$xdc_runtime_LoggerBuf_reset__E
   8f005b20     0c395860     0c3948e4   ti.targets.rts6000.ae66 : LoggerBuf.oe66 (.text:LoggerBuf_instanceStartup)
$.text:ti_sysbios_family_c66_Cache_startup__I:sysbios.ae66<BIOS.obj>$0x0  $Tramp$S$$ti_sysbios_family_c66_Cache_startup__I
   0c3852c0     8f0060a0     8f006040   boot.ae66 : boot.oe66 (.text:_c_int00)

[15 trampolines]
[20 trampoline calls]


GLOBAL SYMBOLS: SORTED ALPHABETICALLY BY Name 

address    name
--------   ----
0c394a40   C$$EXIT
0c393998   C$$IO$$
0c3914e0   HOSTclose
0c38ee20   HOSTlseek
0c38fa20   HOSTopen
0c38fb00   HOSTread
0c38bd00   HOSTrename
0c390820   HOSTunlink
0c3908e0   HOSTwrite
0c3948e0   LoggerBuf_instanceStartup
0c389ce0   MultiProc_getId
0c394900   MultiProc_getNumProcessors
0c38bea0   MultiProc_setLocalId
0c386c80   SharedRegion_getEntry
00800000   __ASM__
0080fe48   __CIOBUF_
00800070   __ISA__
00800088   __PLAT__
008000a8   __TARG__
8f007318   __TI_CINIT_Base
8f007328   __TI_CINIT_Limit
8f007310   __TI_Handler_Table_Base
8f007318   __TI_Handler_Table_Limit
UNDEFED    __TI_INITARRAY_Base
UNDEFED    __TI_INITARRAY_Limit
00810f68   __TI_STACK_END
00001000   __TI_STACK_SIZE
0081280c   __TI_STATIC_BASE
UNDEFED    __TI_TLS_INIT_Base
UNDEFED    __TI_TLS_INIT_Limit
00000001   __TI_args_main
0c394a60   __TI_decompress_none
0c394a80   __TI_decompress_rle24
00812780   __TI_enable_exit_profile_output
ffffffff   __TI_pprof_out_hndl
ffffffff   __TI_prof_data_size
ffffffff   __TI_prof_data_start
0c391360   __TI_tls_init
008000d0   __TRDR__
ffffffff   __binit__
0c382420   __c6xabi_divd
0c3909a0   __c6xabi_divu
0c38c040   __c6xabi_divul
0c388700   __c6xabi_divull
0c392e60   __c6xabi_frcmpyd_div
0c393be0   __c6xabi_isinf
0c391ee0   __c6xabi_llshl
0c392ec0   __c6xabi_llshru
0c394920   __c6xabi_negll
0c391580   __c6xabi_remu
ffffffff   __c_args__
0c3909a0   __divu
0c391580   __remu
0c394940   __xdc__init
008118ec   __xdc__init__addr
0c393c60   _args_main
00000000   _argsize
0c38d400   _auto_init_elf
8f006000   _c_int00
0c391620   _cleanup
00812778   _cleanup_ptr
0c38e1c0   _closefile
8f004408   _ctypes_
0c390a60   _doflush
0081277c   _dtors_ptr
00811d7c   _ft_end
008118f0   _ftable
00812794   _lock
0c394960   _nop
0c383f00   _printfi
0c3949c0   _register_lock
0c3949e0   _register_synch_api
0c394a00   _register_unlock
0080ff68   _stack
0c392f20   _subcull
0080fd00   _tmpnams
00812798   _unlock
0c38ef20   _wrt_ok
0c394a40   abort
0c38fcc0   atoi
ffffffff   binit
0c38fda0   close
0c390b20   exit
0c38fe80   fflush
0c389460   fputc
0c384f20   fputs
0c393ce0   free
0c38e400   fseek
0c391940   lseek
0c38ff60   ltoa
0c390c80   main
0c391fe0   malloc
0c393040   memccpy
0c3919e0   memcpy
0c390040   memset
0c390120   printf
0c394aa0   putc
0c394ac0   putchar
0c392060   readmsg
0c392ae0   remove
0c390be0   setMyId
0c38a2e0   setvbuf
00812130   ti_sdo_ipc_GateMP_Module_State_0_remoteSystemGates__A
00811468   ti_sdo_ipc_GateMP_Module__root__V
00811470   ti_sdo_ipc_GateMP_Module__state__V
8f0046c4   ti_sdo_ipc_Ipc_A_nullArgument__C
00811ec8   ti_sdo_ipc_Ipc_Module_State_0_procEntry__A
008114c0   ti_sdo_ipc_Ipc_Module__state__V
008114cc   ti_sdo_ipc_ListMP_Module__root__V
008114d4   ti_sdo_ipc_ListMP_Module__state__V
00812620   ti_sdo_ipc_MessageQ_Module_State_0_heaps__A
00812548   ti_sdo_ipc_MessageQ_Module_State_0_transports__A
008114d8   ti_sdo_ipc_MessageQ_Module__root__V
008114e0   ti_sdo_ipc_MessageQ_Module__state__V
0c38e520   ti_sdo_ipc_MessageQ_Module_startup__E
8f00483c   ti_sdo_ipc_MessageQ_Object__count__C
0c394ae0   ti_sdo_ipc_MessageQ_Object__get__S
8f004d1c   ti_sdo_ipc_Notify_A_alreadyRegistered__C
8f004d34   ti_sdo_ipc_Notify_A_invArgument__C
0c38f020   ti_sdo_ipc_Notify_Instance_finalize__E
0c384760   ti_sdo_ipc_Notify_Instance_init__E
0c394f80   ti_sdo_ipc_Notify_Module_GateProxy_query__E
008127a8   ti_sdo_ipc_Notify_Module_State_0_notifyHandles_0__A
008127b0   ti_sdo_ipc_Notify_Module_State_0_notifyHandles_1__A
008127b8   ti_sdo_ipc_Notify_Module_State_0_notifyHandles_2__A
008127c0   ti_sdo_ipc_Notify_Module_State_0_notifyHandles_3__A
008127c8   ti_sdo_ipc_Notify_Module_State_0_notifyHandles_4__A
008127d0   ti_sdo_ipc_Notify_Module_State_0_notifyHandles_5__A
008127d8   ti_sdo_ipc_Notify_Module_State_0_notifyHandles_6__A
008127e0   ti_sdo_ipc_Notify_Module_State_0_notifyHandles_7__A
00812640   ti_sdo_ipc_Notify_Module_State_0_notifyHandles__A
8f004d4c   ti_sdo_ipc_Notify_Module__diagsEnabled__C
8f004db0   ti_sdo_ipc_Notify_Module__diagsIncluded__C
8f004db4   ti_sdo_ipc_Notify_Module__diagsMask__C
8f00450a   ti_sdo_ipc_Notify_Module__id__C
00811548   ti_sdo_ipc_Notify_Module__root__V
00811550   ti_sdo_ipc_Notify_Module__state__V
0c38d140   ti_sdo_ipc_Notify_Module_startup__E
8f0049d0   ti_sdo_ipc_Notify_Object__DESC__C
8f004bd0   ti_sdo_ipc_Notify_Object__PARAMS__C
8f004db8   ti_sdo_ipc_Notify_Object__heap__C
0c38f120   ti_sdo_ipc_Notify_create
8f004dbc   ti_sdo_ipc_Notify_numEvents__C
8f004866   ti_sdo_ipc_Notify_numLines__C
8f004dc0   ti_sdo_ipc_SharedRegion_A_idTooLarge__C
008120a0   ti_sdo_ipc_SharedRegion_Module_State_0_regions__A
8f004dc4   ti_sdo_ipc_SharedRegion_Module__diagsEnabled__C
8f004dc8   ti_sdo_ipc_SharedRegion_Module__diagsIncluded__C
8f004dcc   ti_sdo_ipc_SharedRegion_Module__diagsMask__C
8f004d4a   ti_sdo_ipc_SharedRegion_Module__id__C
00811558   ti_sdo_ipc_SharedRegion_Module__state__V
8f0050cc   ti_sdo_ipc_SharedRegion_numEntries__C
8f004dd0   ti_sdo_ipc_family_c647x_Interrupt_KICK0__C
8f004dd4   ti_sdo_ipc_family_c647x_Interrupt_KICK1__C
00812660   ti_sdo_ipc_family_c647x_Interrupt_Module_State_0_args__A
0081155c   ti_sdo_ipc_family_c647x_Interrupt_Module__state__V
0c38f220   ti_sdo_ipc_family_c647x_Interrupt_Module_startup__E
8f0050ce   ti_sdo_ipc_family_c647x_Interrupt_enableKick__C
8f004dd8   ti_sdo_ipc_family_c647x_MultiProcSetup_A_invalidProcessor__C
8f004ddc   ti_sdo_ipc_family_c647x_MultiProcSetup_Module__diagsEnabled__C
8f004de0   ti_sdo_ipc_family_c647x_MultiProcSetup_Module__diagsIncluded__C
8f004de4   ti_sdo_ipc_family_c647x_MultiProcSetup_Module__diagsMask__C
8f0050d0   ti_sdo_ipc_family_c647x_MultiProcSetup_Module__id__C
0c38a4e0   ti_sdo_ipc_family_c647x_MultiProcSetup_init__I
8f004d50   ti_sdo_ipc_family_c647x_MultiProcSetup_procMap__A
8f004de8   ti_sdo_ipc_family_c647x_MultiProcSetup_procMap__C
00811568   ti_sdo_ipc_gates_GateHWSem_Module__root__V
0c38f320   ti_sdo_ipc_gates_GateHWSem_Module_startup__E
8f004dec   ti_sdo_ipc_gates_GateHWSem_baseAddr__C
8f004df0   ti_sdo_ipc_gates_GateHWSem_numSems__C
8f004df8   ti_sdo_ipc_gates_GateHWSem_reservedMaskArr__A
8f004df4   ti_sdo_ipc_gates_GateHWSem_reservedMaskArr__C
00811570   ti_sdo_ipc_gates_GateMPSupportNull_Module__root__V
00811578   ti_sdo_ipc_heaps_HeapBufMP_Module__root__V
00811580   ti_sdo_ipc_heaps_HeapBufMP_Module__state__V
00811584   ti_sdo_ipc_heaps_HeapMemMP_Module__root__V
0081158c   ti_sdo_ipc_heaps_HeapMemMP_Module__state__V
00811590   ti_sdo_ipc_notifyDrivers_NotifyDriverShm_Module__root__V
00811598   ti_sdo_ipc_nsremote_NameServerRemoteNotify_Module__root__V
00812680   ti_sdo_ipc_transports_TransportShmSetup_Module_State_0_handles__A
008115a8   ti_sdo_ipc_transports_TransportShmSetup_Module__state__V
008115a0   ti_sdo_ipc_transports_TransportShm_Module__root__V
0c394b00   ti_sdo_utils_List_Instance_init__E
008115ac   ti_sdo_utils_List_Module__root__V
8f0049f0   ti_sdo_utils_List_Object__DESC__C
8f004be8   ti_sdo_utils_List_Object__PARAMS__C
0c394b20   ti_sdo_utils_List_Object__destruct__S
0c394b40   ti_sdo_utils_List_Object__get__S
0c3930a0   ti_sdo_utils_List_construct
0c394b60   ti_sdo_utils_List_destruct
8f004dfc   ti_sdo_utils_MultiProc_A_invalidMultiProcId__C
8f004e00   ti_sdo_utils_MultiProc_A_invalidProcName__C
00812748   ti_sdo_utils_MultiProc_Module_State_0_clusterProcList__A
8f004e04   ti_sdo_utils_MultiProc_Module__diagsEnabled__C
8f004e08   ti_sdo_utils_MultiProc_Module__diagsIncluded__C
8f004e0c   ti_sdo_utils_MultiProc_Module__diagsMask__C
8f0050d2   ti_sdo_utils_MultiProc_Module__id__C
008115b4   ti_sdo_utils_MultiProc_Module__state__V
0c394b80   ti_sdo_utils_MultiProc_getClusterId__E
0c394b80   ti_sdo_utils_MultiProc_getClusterId__F
8f004a10   ti_sdo_utils_MultiProc_nameList__A
8f004e10   ti_sdo_utils_MultiProc_nameList__C
8f0050d4   ti_sdo_utils_MultiProc_numProcessors__C
8f0050d6   ti_sdo_utils_MultiProc_numProcsInCluster__C
008115d0   ti_sdo_utils_NameServerRemoteNull_Module__root__V
8f004e14   ti_sdo_utils_NameServer_Instance_State_freeList__O
008126a0   ti_sdo_utils_NameServer_Module_State_0_nsRemoteHandle__A
008115bc   ti_sdo_utils_NameServer_Module__root__V
0c393d20   ti_sdo_utils_NameServer_Module__startupDone__F
0c393d20   ti_sdo_utils_NameServer_Module__startupDone__S
008115c4   ti_sdo_utils_NameServer_Module__state__V
0c38d7c0   ti_sdo_utils_NameServer_Module_startup__E
8f004e18   ti_sdo_utils_NameServer_Object__count__C
0c393d60   ti_sdo_utils_NameServer_Object__get__S
00811c50   ti_sdo_utils_NameServer_Object__table__V
008115d8   ti_sysbios_BIOS_Module__state__V
0c394ba0   ti_sysbios_BIOS_RtsGateProxy_enter__E
0c394bc0   ti_sysbios_BIOS_RtsGateProxy_leave__E
0c394f40   ti_sysbios_BIOS_RtsGateProxy_query__E
0c3920e0   ti_sysbios_BIOS_atExitFunc__I
0c393100   ti_sysbios_BIOS_errorRaiseHook__I
0c393da0   ti_sysbios_BIOS_exitFunc__I
0c394be0   ti_sysbios_BIOS_getCpuFreq__E
0c394c00   ti_sysbios_BIOS_linkedWithIncorrectBootLibrary__E
0c394c20   ti_sysbios_BIOS_nullFunc__I
0c393160   ti_sysbios_BIOS_registerRTSLock__I
0c3931c0   ti_sysbios_BIOS_removeRTSLock__I
0c393220   ti_sysbios_BIOS_rtsLock__I
0c393de0   ti_sysbios_BIOS_rtsUnlock__I
0c394c40   ti_sysbios_BIOS_setThreadType__E
0c393280   ti_sysbios_BIOS_startFunc__I
0c394c60   ti_sysbios_family_c62_TaskSupport_Module__startupDone__S
0c393ca0   ti_sysbios_family_c62_TaskSupport_buildTaskStack
0c394c80   ti_sysbios_family_c62_TaskSupport_checkStack__E
0c394a20   ti_sysbios_family_c62_TaskSupport_glue
0c3932e0   ti_sysbios_family_c62_TaskSupport_start__E
0c391f60   ti_sysbios_family_c62_TaskSupport_swap__E
8f004e1c   ti_sysbios_family_c64p_Exception_E_exceptionMax__C
8f0050d8   ti_sysbios_family_c64p_Exception_Module__id__C
008115fc   ti_sysbios_family_c64p_Exception_Module__state__V
0c391a80   ti_sysbios_family_c64p_Exception_Module_startup__E
0c38c840   ti_sysbios_family_c64p_Exception_dispatch__E
8f004e20   ti_sysbios_family_c64p_Exception_exceptionHook__C
8f004e24   ti_sysbios_family_c64p_Exception_externalHook__C
0c380880   ti_sysbios_family_c64p_Exception_handler__I
0c388b80   ti_sysbios_family_c64p_Exception_internalHandler__I
8f004e28   ti_sysbios_family_c64p_Exception_internalHook__C
8f004e2c   ti_sysbios_family_c64p_Exception_nmiHook__C
8f0050da   ti_sysbios_family_c64p_Exception_useInternalBuffer__C
0c395c00   ti_sysbios_family_c64p_Hwi0
00800000   ti_sysbios_family_c64p_Hwi_Instance_State_0_hookEnv__A
8f004e30   ti_sysbios_family_c64p_Hwi_LD_end__C
8f004e34   ti_sysbios_family_c64p_Hwi_LM_begin__C
8f004e38   ti_sysbios_family_c64p_Hwi_Module__diagsEnabled__C
8f004e3c   ti_sysbios_family_c64p_Hwi_Module__diagsIncluded__C
8f004e40   ti_sysbios_family_c64p_Hwi_Module__diagsMask__C
8f0050dc   ti_sysbios_family_c64p_Hwi_Module__id__C
8f0050de   ti_sysbios_family_c64p_Hwi_Module__loggerDefined__C
8f004e44   ti_sysbios_family_c64p_Hwi_Module__loggerFxn1__C
8f004e48   ti_sysbios_family_c64p_Hwi_Module__loggerFxn8__C
8f004e4c   ti_sysbios_family_c64p_Hwi_Module__loggerObj__C
0081162c   ti_sysbios_family_c64p_Hwi_Module__root__V
0c393e20   ti_sysbios_family_c64p_Hwi_Module__startupDone__F
0c393e20   ti_sysbios_family_c64p_Hwi_Module__startupDone__S
00811634   ti_sysbios_family_c64p_Hwi_Module__state__V
0c387aa0   ti_sysbios_family_c64p_Hwi_Module_startup__E
00812700   ti_sysbios_family_c64p_Hwi_Object__table__V
0c394ca0   ti_sysbios_family_c64p_Hwi_clearInterrupt__E
0c393e60   ti_sysbios_family_c64p_Hwi_disableInterrupt__E
0c38a0e0   ti_sysbios_family_c64p_Hwi_dispatchAlways
0c392160   ti_sysbios_family_c64p_Hwi_dispatchC__I
0c385660   ti_sysbios_family_c64p_Hwi_dispatchCore__I
0c393ea0   ti_sysbios_family_c64p_Hwi_enableInterrupt__E
0c3921e0   ti_sysbios_family_c64p_Hwi_getStackInfo__E
8f004d20   ti_sysbios_family_c64p_Hwi_hooks__A
8f004d78   ti_sysbios_family_c64p_Hwi_hooks__C
0c395c00   ti_sysbios_family_c64p_Hwi_int0
0c395c20   ti_sysbios_family_c64p_Hwi_int1
0c395d40   ti_sysbios_family_c64p_Hwi_int10
0c395d60   ti_sysbios_family_c64p_Hwi_int11
0c395d80   ti_sysbios_family_c64p_Hwi_int12
0c395da0   ti_sysbios_family_c64p_Hwi_int13
0c395dc0   ti_sysbios_family_c64p_Hwi_int14
0c395de0   ti_sysbios_family_c64p_Hwi_int15
0c395c40   ti_sysbios_family_c64p_Hwi_int2
0c395c60   ti_sysbios_family_c64p_Hwi_int3
0c395c80   ti_sysbios_family_c64p_Hwi_int4
0c395ca0   ti_sysbios_family_c64p_Hwi_int5
0c395cc0   ti_sysbios_family_c64p_Hwi_int6
0c395ce0   ti_sysbios_family_c64p_Hwi_int7
0c395d00   ti_sysbios_family_c64p_Hwi_int8
0c395d20   ti_sysbios_family_c64p_Hwi_int9
0c394cc0   ti_sysbios_family_c64p_Hwi_startup__E
0c392f80   ti_sysbios_family_c64p_Hwi_switchAndDispatch__I
0c394ce0   ti_sysbios_family_c64p_Hwi_switchFromBootStack__E
0c394d00   ti_sysbios_family_c64p_TimestampProvider_Module_startup__E
0c394d20   ti_sysbios_family_c64p_TimestampProvider_get32__E
0c394d40   ti_sysbios_family_c64p_TimestampProvider_get64__E
0c394be0   ti_sysbios_family_c64p_TimestampProvider_getFreq__E
0c394d60   ti_sysbios_family_c64p_tci6488_TimerSupport_enable__E
8f004e50   ti_sysbios_family_c66_Cache_E_invalidL1CacheSize__C
8f004e54   ti_sysbios_family_c66_Cache_E_invalidL2CacheSize__C
8f0050e0   ti_sysbios_family_c66_Cache_Module__id__C
0c393340   ti_sysbios_family_c66_Cache_Module_startup__E
0c394d80   ti_sysbios_family_c66_Cache_RTSSynchInv__I
0c394da0   ti_sysbios_family_c66_Cache_RTSSynchWbInv__I
0c394dc0   ti_sysbios_family_c66_Cache_RTSSynchWb__I
8f004e58   ti_sysbios_family_c66_Cache_atomicBlockSize__C
0c38b600   ti_sysbios_family_c66_Cache_block__I
0c38c9c0   ti_sysbios_family_c66_Cache_getL2InitSize__I
00008000   ti_sysbios_family_c66_Cache_l1dSize
00008000   ti_sysbios_family_c66_Cache_l1pSize
00020000   ti_sysbios_family_c66_Cache_l2Size
8f003d00   ti_sysbios_family_c66_Cache_marvalues__C
8f0050e2   ti_sysbios_family_c66_Cache_registerRTSSynch__C
0c3852c0   ti_sysbios_family_c66_Cache_startup__I
0c394de0   ti_sysbios_family_c66_Cache_wait__E
8f004e5c   ti_sysbios_family_c66_tci66xx_CpIntc_E_unpluggedSysInt__C
00812758   ti_sysbios_family_c66_tci66xx_CpIntc_Module_State_0_controller__A
00810f68   ti_sysbios_family_c66_tci66xx_CpIntc_Module_State_0_dispatchTab__A
00812008   ti_sysbios_family_c66_tci66xx_CpIntc_Module_State_0_hostIntToSysInt__A
00812730   ti_sysbios_family_c66_tci66xx_CpIntc_Module_State_0_initSIER__A
8f0050e4   ti_sysbios_family_c66_tci66xx_CpIntc_Module__id__C
008116a0   ti_sysbios_family_c66_tci66xx_CpIntc_Module__state__V
0c3877e0   ti_sysbios_family_c66_tci66xx_CpIntc_Module_startup__E
8f004e60   ti_sysbios_family_c66_tci66xx_CpIntc_numStatusRegs__C
8f004e64   ti_sysbios_family_c66_tci66xx_CpIntc_numSysInts__C
8f0042c8   ti_sysbios_family_c66_tci66xx_CpIntc_sysIntToHostInt__A
8f004e68   ti_sysbios_family_c66_tci66xx_CpIntc_sysIntToHostInt__C
0c3933a0   ti_sysbios_family_c66_tci66xx_CpIntc_unused__E
0c392fe0   ti_sysbios_family_xxx_Hwi_switchAndRunFunc
0c393ee0   ti_sysbios_gates_GateAll_Handle__label__S
0c394e00   ti_sysbios_gates_GateAll_Instance_init__E
8f004868   ti_sysbios_gates_GateAll_Module__FXNS__C
008116b0   ti_sysbios_gates_GateAll_Module__root__V
8f004a30   ti_sysbios_gates_GateAll_Object__DESC__C
8f004c00   ti_sysbios_gates_GateAll_Object__PARAMS__C
0c392260   ti_sysbios_gates_GateAll_Object__create__S
0c393f20   ti_sysbios_gates_GateAll_Object__delete__S
00812768   ti_sysbios_gates_GateAll_Object__table__V
0c393400   ti_sysbios_gates_GateAll_enter__E
0c390ca0   ti_sysbios_gates_GateAll_leave__E
0c394e20   ti_sysbios_gates_GateAll_query__E
0c393f60   ti_sysbios_gates_GateHwi_Handle__label__S
0c394e40   ti_sysbios_gates_GateHwi_Instance_init__E
8f00488c   ti_sysbios_gates_GateHwi_Module__FXNS__C
008116b8   ti_sysbios_gates_GateHwi_Module__root__V
8f004a50   ti_sysbios_gates_GateHwi_Object__DESC__C
8f004c18   ti_sysbios_gates_GateHwi_Object__PARAMS__C
0c3922e0   ti_sysbios_gates_GateHwi_Object__create__S
0c393fa0   ti_sysbios_gates_GateHwi_Object__delete__S
008127e8   ti_sysbios_gates_GateHwi_Object__table__V
0c394e60   ti_sysbios_gates_GateHwi_enter__E
0c394e80   ti_sysbios_gates_GateHwi_leave__E
0c394ea0   ti_sysbios_gates_GateHwi_query__E
8f004e6c   ti_sysbios_gates_GateMutexPri_A_badContext__C
8f004e70   ti_sysbios_gates_GateMutexPri_A_enterTaskDisabled__C
0c393fe0   ti_sysbios_gates_GateMutexPri_Handle__label__S
8f004e74   ti_sysbios_gates_GateMutexPri_Instance_State_pendQ__O
0c394ec0   ti_sysbios_gates_GateMutexPri_Instance_finalize__E
0c394020   ti_sysbios_gates_GateMutexPri_Instance_init__E
8f0048b0   ti_sysbios_gates_GateMutexPri_Module__FXNS__C
8f004e78   ti_sysbios_gates_GateMutexPri_Module__diagsEnabled__C
8f004e7c   ti_sysbios_gates_GateMutexPri_Module__diagsIncluded__C
8f004e80   ti_sysbios_gates_GateMutexPri_Module__diagsMask__C
8f0050e6   ti_sysbios_gates_GateMutexPri_Module__id__C
008116c8   ti_sysbios_gates_GateMutexPri_Module__root__V
8f004a70   ti_sysbios_gates_GateMutexPri_Object__DESC__C
8f004c30   ti_sysbios_gates_GateMutexPri_Object__PARAMS__C
0c392360   ti_sysbios_gates_GateMutexPri_Object__create__S
0c393460   ti_sysbios_gates_GateMutexPri_Object__delete__S
0c394060   ti_sysbios_gates_GateMutexPri_Object__destruct__S
00812718   ti_sysbios_gates_GateMutexPri_Object__table__V
0c3934c0   ti_sysbios_gates_GateMutexPri_construct
0c394ee0   ti_sysbios_gates_GateMutexPri_destruct
0c384360   ti_sysbios_gates_GateMutexPri_enter__E
0c38f420   ti_sysbios_gates_GateMutexPri_leave__E
0c394f00   ti_sysbios_gates_GateMutexPri_query__E
8f004e84   ti_sysbios_gates_GateMutex_A_badContext__C
0c3940a0   ti_sysbios_gates_GateMutex_Handle__label__S
8f004e88   ti_sysbios_gates_GateMutex_Instance_State_sem__O
0c394f20   ti_sysbios_gates_GateMutex_Instance_finalize__E
0c3940e0   ti_sysbios_gates_GateMutex_Instance_init__E
8f0048d4   ti_sysbios_gates_GateMutex_Module__FXNS__C
8f004e8c   ti_sysbios_gates_GateMutex_Module__diagsEnabled__C
8f004e90   ti_sysbios_gates_GateMutex_Module__diagsIncluded__C
8f004e94   ti_sysbios_gates_GateMutex_Module__diagsMask__C
8f0050e8   ti_sysbios_gates_GateMutex_Module__id__C
008116c0   ti_sysbios_gates_GateMutex_Module__root__V
8f004a90   ti_sysbios_gates_GateMutex_Object__DESC__C
8f004c48   ti_sysbios_gates_GateMutex_Object__PARAMS__C
0c3923e0   ti_sysbios_gates_GateMutex_Object__create__S
0c393520   ti_sysbios_gates_GateMutex_Object__delete__S
00812588   ti_sysbios_gates_GateMutex_Object__table__V
0c38c1e0   ti_sysbios_gates_GateMutex_enter__E
0c394120   ti_sysbios_gates_GateMutex_leave__E
0c394f40   ti_sysbios_gates_GateMutex_query__E
8f004e98   ti_sysbios_gates_GateSwi_A_badContext__C
0c394160   ti_sysbios_gates_GateSwi_Handle__label__S
0c394f60   ti_sysbios_gates_GateSwi_Instance_init__E
8f0048f8   ti_sysbios_gates_GateSwi_Module__FXNS__C
8f004e9c   ti_sysbios_gates_GateSwi_Module__diagsEnabled__C
8f004ea0   ti_sysbios_gates_GateSwi_Module__diagsIncluded__C
8f004ea4   ti_sysbios_gates_GateSwi_Module__diagsMask__C
8f0050ea   ti_sysbios_gates_GateSwi_Module__id__C
008116d0   ti_sysbios_gates_GateSwi_Module__root__V
8f004ab0   ti_sysbios_gates_GateSwi_Object__DESC__C
8f004c60   ti_sysbios_gates_GateSwi_Object__PARAMS__C
0c392460   ti_sysbios_gates_GateSwi_Object__create__S
0c3941a0   ti_sysbios_gates_GateSwi_Object__delete__S
00812788   ti_sysbios_gates_GateSwi_Object__table__V
0c38d900   ti_sysbios_gates_GateSwi_enter__E
0c3924e0   ti_sysbios_gates_GateSwi_leave__E
0c394f80   ti_sysbios_gates_GateSwi_query__E
0c394de0   ti_sysbios_hal_Cache_CacheProxy_wait__E
0c394de0   ti_sysbios_hal_Cache_wait__E
8f004ea8   ti_sysbios_hal_Hwi_E_stackOverflow__C
0c394fa0   ti_sysbios_hal_Hwi_HwiProxy_Module__startupDone__S
0c394ca0   ti_sysbios_hal_Hwi_HwiProxy_clearInterrupt__E
0c393e60   ti_sysbios_hal_Hwi_HwiProxy_disableInterrupt__E
0c393ea0   ti_sysbios_hal_Hwi_HwiProxy_enableInterrupt__E
0c3921e0   ti_sysbios_hal_Hwi_HwiProxy_getStackInfo__E
0c394cc0   ti_sysbios_hal_Hwi_HwiProxy_startup__E
0c394ce0   ti_sysbios_hal_Hwi_HwiProxy_switchFromBootStack__E
8f0050ec   ti_sysbios_hal_Hwi_Module__id__C
008116d8   ti_sysbios_hal_Hwi_Module__root__V
0c394fc0   ti_sysbios_hal_Hwi_Module_startup__E
008127a0   ti_sysbios_hal_Hwi_Object__table__V
0c392560   ti_sysbios_hal_Hwi_checkStack
0c394ca0   ti_sysbios_hal_Hwi_clearInterrupt__E
0c393e60   ti_sysbios_hal_Hwi_disableInterrupt__E
0c393ea0   ti_sysbios_hal_Hwi_enableInterrupt__E
0c3921e0   ti_sysbios_hal_Hwi_getStackInfo__E
0c3925e0   ti_sysbios_hal_Hwi_initStack
0c394cc0   ti_sysbios_hal_Hwi_startup__E
008116e0   ti_sysbios_hal_Timer_Module__root__V
0c394fe0   ti_sysbios_hal_Timer_Module_startup__E
0c395000   ti_sysbios_hal_Timer_TimerProxy_Module__startupDone__S
0c3902e0   ti_sysbios_hal_Timer_TimerProxy_startup__E
0c3902e0   ti_sysbios_hal_Timer_startup__E
8f004eac   ti_sysbios_heaps_HeapMem_A_align__C
8f004eb0   ti_sysbios_heaps_HeapMem_A_heapSize__C
8f004eb4   ti_sysbios_heaps_HeapMem_A_invalidFree__C
8f004eb8   ti_sysbios_heaps_HeapMem_A_zeroBlock__C
8f004ebc   ti_sysbios_heaps_HeapMem_E_memory__C
0c3941e0   ti_sysbios_heaps_HeapMem_Handle__label__S
903c0000   ti_sysbios_heaps_HeapMem_Instance_State_0_buf__A
97160000   ti_sysbios_heaps_HeapMem_Instance_State_1_buf__A
9df00000   ti_sysbios_heaps_HeapMem_Instance_State_2_buf__A
9ef00000   ti_sysbios_heaps_HeapMem_Instance_State_3_buf__A
9ff00000   ti_sysbios_heaps_HeapMem_Instance_State_4_buf__A
9ff80000   ti_sysbios_heaps_HeapMem_Instance_State_5_buf__A
00800008   ti_sysbios_heaps_HeapMem_Instance_State_6_buf__A
0c387240   ti_sysbios_heaps_HeapMem_Instance_init__E
0c395020   ti_sysbios_heaps_HeapMem_Module_GateProxy_enter__E
0c395040   ti_sysbios_heaps_HeapMem_Module_GateProxy_leave__E
0c394f40   ti_sysbios_heaps_HeapMem_Module_GateProxy_query__E
8f0047ec   ti_sysbios_heaps_HeapMem_Module__FXNS__C
8f004ec0   ti_sysbios_heaps_HeapMem_Module__diagsEnabled__C
8f004ec4   ti_sysbios_heaps_HeapMem_Module__diagsIncluded__C
8f004ec8   ti_sysbios_heaps_HeapMem_Module__diagsMask__C
8f004ecc   ti_sysbios_heaps_HeapMem_Module__gateObj__C
8f0050ee   ti_sysbios_heaps_HeapMem_Module__id__C
008116e8   ti_sysbios_heaps_HeapMem_Module__root__V
8f004ad0   ti_sysbios_heaps_HeapMem_Object__DESC__C
8f00491c   ti_sysbios_heaps_HeapMem_Object__PARAMS__C
8f004ed0   ti_sysbios_heaps_HeapMem_Object__count__C
0c392660   ti_sysbios_heaps_HeapMem_Object__create__S
0c394220   ti_sysbios_heaps_HeapMem_Object__delete__S
0c394260   ti_sysbios_heaps_HeapMem_Object__get__S
00811d80   ti_sysbios_heaps_HeapMem_Object__table__V
0c381e00   ti_sysbios_heaps_HeapMem_allocUnprotected__E
0c390d60   ti_sysbios_heaps_HeapMem_alloc__E
0c382fa0   ti_sysbios_heaps_HeapMem_freeUnprotected__E
0c393580   ti_sysbios_heaps_HeapMem_free__E
0c390e20   ti_sysbios_heaps_HeapMem_getStats__E
0c391b20   ti_sysbios_heaps_HeapMem_init__I
0c395060   ti_sysbios_heaps_HeapMem_isBlocking__E
8f004ed4   ti_sysbios_heaps_HeapMem_reqAlign__C
8f004ed8   ti_sysbios_knl_Clock_LM_begin__C
8f004edc   ti_sysbios_knl_Clock_LM_tick__C
8f004ee0   ti_sysbios_knl_Clock_LW_delayed__C
8f004ee4   ti_sysbios_knl_Clock_Module_State_clockQ__O
8f004ee8   ti_sysbios_knl_Clock_Module__diagsEnabled__C
8f004eec   ti_sysbios_knl_Clock_Module__diagsIncluded__C
8f004ef0   ti_sysbios_knl_Clock_Module__diagsMask__C
8f0050f0   ti_sysbios_knl_Clock_Module__id__C
8f0050f2   ti_sysbios_knl_Clock_Module__loggerDefined__C
8f004ef4   ti_sysbios_knl_Clock_Module__loggerFxn1__C
8f004ef8   ti_sysbios_knl_Clock_Module__loggerFxn2__C
8f004efc   ti_sysbios_knl_Clock_Module__loggerObj__C
008116f0   ti_sysbios_knl_Clock_Module__root__V
008116f8   ti_sysbios_knl_Clock_Module__state__V
0c3935e0   ti_sysbios_knl_Clock_Module_startup__E
0c395080   ti_sysbios_knl_Clock_TimerProxy_Module__startupDone__S
0c3950a0   ti_sysbios_knl_Clock_TimerProxy_getMaxTicks__E
0c3902e0   ti_sysbios_knl_Clock_TimerProxy_startup__E
0c3926e0   ti_sysbios_knl_Clock_doTick__I
0c390ee0   ti_sysbios_knl_Clock_logTick__E
0c387d40   ti_sysbios_knl_Clock_workFunc__E
00811724   ti_sysbios_knl_Event_Module__root__V
8f004d80   ti_sysbios_knl_Idle_funcList__A
8f004d88   ti_sysbios_knl_Idle_funcList__C
0c3950c0   ti_sysbios_knl_Idle_loop__E
0c392760   ti_sysbios_knl_Idle_run__E
0c3950e0   ti_sysbios_knl_Queue_Instance_init__E
00811730   ti_sysbios_knl_Queue_Module__root__V
8f004af0   ti_sysbios_knl_Queue_Object__DESC__C
8f004c78   ti_sysbios_knl_Queue_Object__PARAMS__C
0c395100   ti_sysbios_knl_Queue_Object__destruct__S
0c395120   ti_sysbios_knl_Queue_Object__get__S
0c393640   ti_sysbios_knl_Queue_construct
0c395140   ti_sysbios_knl_Queue_destruct
0c395160   ti_sysbios_knl_Queue_empty__E
8f004f00   ti_sysbios_knl_Semaphore_A_badContext__C
8f004f04   ti_sysbios_knl_Semaphore_A_noEvents__C
8f004f08   ti_sysbios_knl_Semaphore_A_overflow__C
8f004f0c   ti_sysbios_knl_Semaphore_A_pendTaskDisabled__C
8f004f10   ti_sysbios_knl_Semaphore_Instance_State_pendQ__O
0c395180   ti_sysbios_knl_Semaphore_Instance_finalize__E
0c38da40   ti_sysbios_knl_Semaphore_Instance_init__E
8f004f14   ti_sysbios_knl_Semaphore_LM_pend__C
8f004f18   ti_sysbios_knl_Semaphore_LM_post__C
8f004f1c   ti_sysbios_knl_Semaphore_Module__diagsEnabled__C
8f004f20   ti_sysbios_knl_Semaphore_Module__diagsIncluded__C
8f004f24   ti_sysbios_knl_Semaphore_Module__diagsMask__C
8f0050f4   ti_sysbios_knl_Semaphore_Module__id__C
8f0050f6   ti_sysbios_knl_Semaphore_Module__loggerDefined__C
8f004f28   ti_sysbios_knl_Semaphore_Module__loggerFxn2__C
8f004f2c   ti_sysbios_knl_Semaphore_Module__loggerFxn4__C
8f004f30   ti_sysbios_knl_Semaphore_Module__loggerObj__C
00811738   ti_sysbios_knl_Semaphore_Module__root__V
8f004b10   ti_sysbios_knl_Semaphore_Object__DESC__C
8f004940   ti_sysbios_knl_Semaphore_Object__PARAMS__C
0c3942a0   ti_sysbios_knl_Semaphore_Object__destruct__S
0c3936a0   ti_sysbios_knl_Semaphore_construct
0c3951a0   ti_sysbios_knl_Semaphore_destruct
0c393700   ti_sysbios_knl_Semaphore_pendTimeout__I
0c381000   ti_sysbios_knl_Semaphore_pend__E
0c388dc0   ti_sysbios_knl_Semaphore_post__E
00808008   ti_sysbios_knl_Swi_Instance_State_0_hookEnv__A
8f004f34   ti_sysbios_knl_Swi_LD_end__C
8f004f38   ti_sysbios_knl_Swi_LM_begin__C
8f004f3c   ti_sysbios_knl_Swi_LM_post__C
008121b0   ti_sysbios_knl_Swi_Module_State_0_readyQ__A
8f004f40   ti_sysbios_knl_Swi_Module__diagsEnabled__C
8f004f44   ti_sysbios_knl_Swi_Module__diagsIncluded__C
8f004f48   ti_sysbios_knl_Swi_Module__diagsMask__C
8f0050f8   ti_sysbios_knl_Swi_Module__id__C
8f0050fa   ti_sysbios_knl_Swi_Module__loggerDefined__C
8f004f4c   ti_sysbios_knl_Swi_Module__loggerFxn1__C
8f004f50   ti_sysbios_knl_Swi_Module__loggerFxn4__C
8f004f54   ti_sysbios_knl_Swi_Module__loggerObj__C
00811740   ti_sysbios_knl_Swi_Module__root__V
00811748   ti_sysbios_knl_Swi_Module__state__V
0c387fe0   ti_sysbios_knl_Swi_Module_startup__E
8f004f58   ti_sysbios_knl_Swi_Object__count__C
0c3942e0   ti_sysbios_knl_Swi_Object__get__S
008125c8   ti_sysbios_knl_Swi_Object__table__V
0c3951c0   ti_sysbios_knl_Swi_disable__E
8f004c90   ti_sysbios_knl_Swi_hooks__A
8f004d90   ti_sysbios_knl_Swi_hooks__C
8f004f5c   ti_sysbios_knl_Swi_numConstructedSwis__C
0c38b7c0   ti_sysbios_knl_Swi_post__E
0c38f520   ti_sysbios_knl_Swi_restoreHwi__E
0c390200   ti_sysbios_knl_Swi_runLoop__I
0c386680   ti_sysbios_knl_Swi_run__I
0c390fa0   ti_sysbios_knl_Swi_schedule__I
0c3927e0   ti_sysbios_knl_Swi_startup__E
8f004f60   ti_sysbios_knl_Task_A_badPriority__C
8f004f64   ti_sysbios_knl_Task_E_spOutOfBounds__C
8f004f68   ti_sysbios_knl_Task_E_stackOverflow__C
00808010   ti_sysbios_knl_Task_Instance_State_0_hookEnv__A
0080f500   ti_sysbios_knl_Task_Instance_State_0_stack__A
8f004f6c   ti_sysbios_knl_Task_LD_block__C
8f004f70   ti_sysbios_knl_Task_LD_exit__C
8f004f74   ti_sysbios_knl_Task_LD_ready__C
8f004f78   ti_sysbios_knl_Task_LM_setPri__C
8f004f7c   ti_sysbios_knl_Task_LM_switch__C
008127f0   ti_sysbios_knl_Task_Module_State_0_idleTask__A
00812230   ti_sysbios_knl_Task_Module_State_0_readyQ__A
8f004f80   ti_sysbios_knl_Task_Module_State_inactiveQ__O
8f004f84   ti_sysbios_knl_Task_Module__diagsEnabled__C
8f004f88   ti_sysbios_knl_Task_Module__diagsIncluded__C
8f004f8c   ti_sysbios_knl_Task_Module__diagsMask__C
8f0050fc   ti_sysbios_knl_Task_Module__id__C
8f0050fe   ti_sysbios_knl_Task_Module__loggerDefined__C
8f004f90   ti_sysbios_knl_Task_Module__loggerFxn2__C
8f004f94   ti_sysbios_knl_Task_Module__loggerFxn4__C
8f004f98   ti_sysbios_knl_Task_Module__loggerObj__C
00811764   ti_sysbios_knl_Task_Module__root__V
00811770   ti_sysbios_knl_Task_Module__state__V
0c383a80   ti_sysbios_knl_Task_Module_startup__E
8f004f9c   ti_sysbios_knl_Task_Object__count__C
0c394320   ti_sysbios_knl_Task_Object__get__S
8f004fa0   ti_sysbios_knl_Task_Object__heap__C
008124a8   ti_sysbios_knl_Task_Object__table__V
0c3951e0   ti_sysbios_knl_Task_SupportProxy_Module__startupDone__S
0c394c80   ti_sysbios_knl_Task_SupportProxy_checkStack__E
0c3932e0   ti_sysbios_knl_Task_SupportProxy_start__E
0c391f60   ti_sysbios_knl_Task_SupportProxy_swap__E
8f004fa4   ti_sysbios_knl_Task_allBlockedFunc__C
0c391060   ti_sysbios_knl_Task_allBlockedFunction__I
0c38db80   ti_sysbios_knl_Task_blockI__E
0c38b980   ti_sysbios_knl_Task_checkStacks__E
0c395200   ti_sysbios_knl_Task_disable__E
0c393760   ti_sysbios_knl_Task_enter__I
0c38aae0   ti_sysbios_knl_Task_exit__E
0c395220   ti_sysbios_knl_Task_getHookContext__E
8f004ca8   ti_sysbios_knl_Task_hooks__A
8f004d98   ti_sysbios_knl_Task_hooks__C
8f004fa8   ti_sysbios_knl_Task_numConstructedTasks__C
0c392860   ti_sysbios_knl_Task_restore__E
0c389680   ti_sysbios_knl_Task_schedule__I
0c384b40   ti_sysbios_knl_Task_setPri__E
0c38a6e0   ti_sysbios_knl_Task_startCore__E
0c395240   ti_sysbios_knl_Task_startup__E
0c38c380   ti_sysbios_knl_Task_unblockI__E
008117b4   ti_sysbios_rts_ti_ThreadLocalStorage_Module__state__V
008117c0   ti_sysbios_syncs_SyncSem_Module__root__V
8f004fac   ti_sysbios_timers_timer64_Timer_A_notAvailable__C
8f004fb0   ti_sysbios_timers_timer64_Timer_E_cannotSupport__C
00811ad0   ti_sysbios_timers_timer64_Timer_Module_State_0_device__A
008122b0   ti_sysbios_timers_timer64_Timer_Module_State_0_gctrl__A
00812330   ti_sysbios_timers_timer64_Timer_Module_State_0_handles__A
008123b0   ti_sysbios_timers_timer64_Timer_Module_State_0_intFreqs__A
8f004fb4   ti_sysbios_timers_timer64_Timer_Module__diagsEnabled__C
8f004fb8   ti_sysbios_timers_timer64_Timer_Module__diagsIncluded__C
8f004fbc   ti_sysbios_timers_timer64_Timer_Module__diagsMask__C
8f005100   ti_sysbios_timers_timer64_Timer_Module__id__C
008117c8   ti_sysbios_timers_timer64_Timer_Module__root__V
0c394360   ti_sysbios_timers_timer64_Timer_Module__startupDone__F
0c394360   ti_sysbios_timers_timer64_Timer_Module__startupDone__S
008117d0   ti_sysbios_timers_timer64_Timer_Module__state__V
0c381760   ti_sysbios_timers_timer64_Timer_Module_startup__E
008124f8   ti_sysbios_timers_timer64_Timer_Object__table__V
0c394d60   ti_sysbios_timers_timer64_Timer_TimerSupportProxy_enable__E
8f004fc0   ti_sysbios_timers_timer64_Timer_anyMaskHigh__C
8f004fc4   ti_sysbios_timers_timer64_Timer_anyMask__C
0c386980   ti_sysbios_timers_timer64_Timer_deviceConfig__I
8f004fc8   ti_sysbios_timers_timer64_Timer_freqDivisor__C
0c38acc0   ti_sysbios_timers_timer64_Timer_getFreq__E
0c395260   ti_sysbios_timers_timer64_Timer_getMaxTicks__E
0c38f620   ti_sysbios_timers_timer64_Timer_initDevice__I
8f0033fb   ti_sysbios_timers_timer64_Timer_localTimerBaseId__C
8f004fcc   ti_sysbios_timers_timer64_Timer_numLocalTimers__C
8f004fd0   ti_sysbios_timers_timer64_Timer_numTimerDevices__C
0c3898a0   ti_sysbios_timers_timer64_Timer_setPeriodMicroSecs__E
0c38c520   ti_sysbios_timers_timer64_Timer_start__E
8f005102   ti_sysbios_timers_timer64_Timer_startupNeeded__C
0c3902e0   ti_sysbios_timers_timer64_Timer_startup__E
0c391120   ti_sysbios_timers_timer64_Timer_stop__E
8f005104   ti_sysbios_timers_timer64_Timer_useTimer64pRegMap__C
8f004fd4   ti_sysbios_utils_Load_LS_cpuLoad__C
8f004fd8   ti_sysbios_utils_Load_LS_hwiLoad__C
8f004fdc   ti_sysbios_utils_Load_LS_swiLoad__C
8f004fe0   ti_sysbios_utils_Load_LS_taskLoad__C
008127f8   ti_sysbios_utils_Load_Module_State_0_runningTask__A
008126e0   ti_sysbios_utils_Load_Module_State_0_taskEnv__A
00812800   ti_sysbios_utils_Load_Module_State_0_taskStartTime__A
8f004fe4   ti_sysbios_utils_Load_Module_State_taskList__O
8f004fe8   ti_sysbios_utils_Load_Module__diagsEnabled__C
8f004fec   ti_sysbios_utils_Load_Module__diagsIncluded__C
8f004ff0   ti_sysbios_utils_Load_Module__diagsMask__C
8f005106   ti_sysbios_utils_Load_Module__id__C
8f005108   ti_sysbios_utils_Load_Module__loggerDefined__C
8f004ff4   ti_sysbios_utils_Load_Module__loggerFxn1__C
8f004ff8   ti_sysbios_utils_Load_Module__loggerFxn2__C
8f004ffc   ti_sysbios_utils_Load_Module__loggerFxn4__C
8f005000   ti_sysbios_utils_Load_Module__loggerObj__C
008117e8   ti_sysbios_utils_Load_Module__state__V
8f00510a   ti_sysbios_utils_Load_autoAddTasks__C
0c38f720   ti_sysbios_utils_Load_hwiBeginHook__E
0c3928e0   ti_sysbios_utils_Load_hwiEndHook__E
0c38aea0   ti_sysbios_utils_Load_idleFxn__E
0c385d00   ti_sysbios_utils_Load_logLoads__I
8f005004   ti_sysbios_utils_Load_postUpdate__C
0c38cb40   ti_sysbios_utils_Load_startup__E
0c391bc0   ti_sysbios_utils_Load_swiBeginHook__E
0c392960   ti_sysbios_utils_Load_swiEndHook__E
0c38ccc0   ti_sysbios_utils_Load_taskCreateHook__E
0c38e640   ti_sysbios_utils_Load_taskDeleteHook__E
0c395280   ti_sysbios_utils_Load_taskRegHook__E
0c3911e0   ti_sysbios_utils_Load_taskSwitchHook__E
0c38e760   ti_sysbios_utils_Load_updateCurrentThreadTime__E
8f00510c   ti_sysbios_utils_Load_updateInIdle__C
0c38a8e0   ti_sysbios_utils_Load_updateLoads__E
0c388240   ti_sysbios_utils_Load_updateThreadContexts__E
0c38a8e0   ti_sysbios_utils_Load_update__E
8f005008   ti_sysbios_utils_Load_windowInMs__C
8f00500c   ti_sysbios_xdcruntime_GateThreadSupport_Instance_State_gate__O
0c3952a0   ti_sysbios_xdcruntime_GateThreadSupport_Instance_finalize__E
0c3943a0   ti_sysbios_xdcruntime_GateThreadSupport_Instance_init__E
00811880   ti_sysbios_xdcruntime_GateThreadSupport_Module__root__V
8f004b30   ti_sysbios_xdcruntime_GateThreadSupport_Object__DESC__C
8f004cc0   ti_sysbios_xdcruntime_GateThreadSupport_Object__PARAMS__C
0c3929e0   ti_sysbios_xdcruntime_GateThreadSupport_Object__create__S
0c3937c0   ti_sysbios_xdcruntime_GateThreadSupport_Object__delete__S
0c3952c0   ti_sysbios_xdcruntime_GateThreadSupport_enter__E
0c38f820   ti_sysbios_xdcruntime_GateThreadSupport_leave__E
0c394f00   ti_sysbios_xdcruntime_GateThreadSupport_query__E
0c3943e0   ti_uia_loggers_LoggerStopMode_Handle__label__S
00808080   ti_uia_loggers_LoggerStopMode_Instance_State_0_hdr__A
00808200   ti_uia_loggers_LoggerStopMode_Instance_State_0_packetArray__A
0080a200   ti_uia_loggers_LoggerStopMode_Instance_State_1_hdr__A
0080a380   ti_uia_loggers_LoggerStopMode_Instance_State_1_packetArray__A
0080c380   ti_uia_loggers_LoggerStopMode_Instance_State_2_hdr__A
0080c500   ti_uia_loggers_LoggerStopMode_Instance_State_2_packetArray__A
0c393820   ti_uia_loggers_LoggerStopMode_Instance_init__E
8f00460c   ti_uia_loggers_LoggerStopMode_Module__FXNS__C
8f005010   ti_uia_loggers_LoggerStopMode_Module__diagsEnabled__C
8f005014   ti_uia_loggers_LoggerStopMode_Module__diagsIncluded__C
8f005018   ti_uia_loggers_LoggerStopMode_Module__diagsMask__C
8f00510e   ti_uia_loggers_LoggerStopMode_Module__id__C
00811888   ti_uia_loggers_LoggerStopMode_Module__root__V
00811890   ti_uia_loggers_LoggerStopMode_Module__state__V
0c38e880   ti_uia_loggers_LoggerStopMode_Module_startup__E
8f004b50   ti_uia_loggers_LoggerStopMode_Object__DESC__C
8f004790   ti_uia_loggers_LoggerStopMode_Object__PARAMS__C
8f00501c   ti_uia_loggers_LoggerStopMode_Object__count__C
0c392a60   ti_uia_loggers_LoggerStopMode_Object__create__S
0c394420   ti_uia_loggers_LoggerStopMode_Object__delete__S
0c394460   ti_uia_loggers_LoggerStopMode_Object__get__S
00811f68   ti_uia_loggers_LoggerStopMode_Object__table__V
0c3944a0   ti_uia_loggers_LoggerStopMode_disable__E
0c3944e0   ti_uia_loggers_LoggerStopMode_enable__E
0c3912a0   ti_uia_loggers_LoggerStopMode_flush__E
0c3952e0   ti_uia_loggers_LoggerStopMode_getContents__E
0c395300   ti_uia_loggers_LoggerStopMode_getFilterLevel__E
0c395320   ti_uia_loggers_LoggerStopMode_getInstanceId__E
0c395340   ti_uia_loggers_LoggerStopMode_getMaxLength__E
0c395360   ti_uia_loggers_LoggerStopMode_getPriority__E
0c395380   ti_uia_loggers_LoggerStopMode_getTransferType__E
0c393880   ti_uia_loggers_LoggerStopMode_initBuffer__I
0c38dcc0   ti_uia_loggers_LoggerStopMode_initQueueDescriptor__E
0c3953a0   ti_uia_loggers_LoggerStopMode_isEmpty__E
8f005110   ti_uia_loggers_LoggerStopMode_isTimestampEnabled__C
8f005020   ti_uia_loggers_LoggerStopMode_numCores__C
0c3938e0   ti_uia_loggers_LoggerStopMode_reset__E
0c3953c0   ti_uia_loggers_LoggerStopMode_setFilterLevel__E
0c3953e0   ti_uia_loggers_LoggerStopMode_setPriority__E
0c38de00   ti_uia_loggers_LoggerStopMode_write0__E
0c38df40   ti_uia_loggers_LoggerStopMode_write1__E
0c38e080   ti_uia_loggers_LoggerStopMode_write2__E
0c38d2a0   ti_uia_loggers_LoggerStopMode_write4__E
0c38ce40   ti_uia_loggers_LoggerStopMode_write8__E
0c389000   ti_uia_loggers_LoggerStopMode_writeMemoryRange__E
8f005024   ti_uia_runtime_ILoggerSnapshot_Interface__BASE__C
8f005028   ti_uia_runtime_IUIATransfer_Interface__BASE__C
00811898   ti_uia_runtime_QueueDescriptor_Module__state__V
0c38e9a0   ti_uia_runtime_QueueDescriptor_addToList__E
0081280c   ti_uia_runtime_QueueDescriptor_gPtrToFirstDescriptor
00812810   ti_uia_runtime_QueueDescriptor_gUpdateCount
0c392ae0   unlink
0c391c60   write
0c393940   writemsg
8f00502c   xdc_runtime_Assert_E_assertFailed__C
0c391d00   xdc_runtime_Assert_raise__I
8f005030   xdc_runtime_Core_A_initializedParams__C
8f005034   xdc_runtime_Core_Module__diagsEnabled__C
8f005038   xdc_runtime_Core_Module__diagsIncluded__C
8f00503c   xdc_runtime_Core_Module__diagsMask__C
8f005112   xdc_runtime_Core_Module__id__C
0c392b60   xdc_runtime_Core_assignLabel__I
0c392be0   xdc_runtime_Core_assignParams__I
0c38cfc0   xdc_runtime_Core_constructObject__I
0c389ac0   xdc_runtime_Core_createObject__I
0c38eac0   xdc_runtime_Core_deleteObject__I
8f005040   xdc_runtime_Error_E_memory__C
8f005044   xdc_runtime_Error_Module__diagsEnabled__C
8f005048   xdc_runtime_Error_Module__diagsIncluded__C
8f00504c   xdc_runtime_Error_Module__diagsMask__C
8f005114   xdc_runtime_Error_Module__loggerDefined__C
8f005050   xdc_runtime_Error_Module__loggerFxn8__C
8f005054   xdc_runtime_Error_Module__loggerObj__C
008118a4   xdc_runtime_Error_Module__state__V
0c394520   xdc_runtime_Error_check__E
0c395400   xdc_runtime_Error_getSite__E
0c394560   xdc_runtime_Error_init__E
8f005116   xdc_runtime_Error_maxDepth__C
0c38b080   xdc_runtime_Error_policyDefault__E
8f005058   xdc_runtime_Error_policyFxn__C
8f00505c   xdc_runtime_Error_policy__C
0c3903c0   xdc_runtime_Error_print__E
8f005060   xdc_runtime_Error_raiseHook__C
0c395420   xdc_runtime_Error_raiseX__E
0c391da0   xdc_runtime_Error_setX__E
0c3945a0   xdc_runtime_GateNull_Handle__label__S
8f004964   xdc_runtime_GateNull_Module__FXNS__C
008118a8   xdc_runtime_GateNull_Module__root__V
8f004b70   xdc_runtime_GateNull_Object__DESC__C
8f004cd8   xdc_runtime_GateNull_Object__PARAMS__C
0c3945e0   xdc_runtime_GateNull_Object__create__S
0c394620   xdc_runtime_GateNull_Object__delete__S
00812808   xdc_runtime_GateNull_Object__table__V
0c395440   xdc_runtime_GateNull_enter__E
0c395460   xdc_runtime_GateNull_leave__E
0c395480   xdc_runtime_GateNull_query__E
0c3954a0   xdc_runtime_Gate_enterSystem__E
0c3954c0   xdc_runtime_Gate_leaveSystem__E
8f005064   xdc_runtime_IFilterLogger_Interface__BASE__C
8f005068   xdc_runtime_IGateProvider_Interface__BASE__C
8f00506c   xdc_runtime_IHeap_Interface__BASE__C
8f005070   xdc_runtime_ILogger_Interface__BASE__C
8f005074   xdc_runtime_IModule_Interface__BASE__C
8f005078   xdc_runtime_Log_L_error__C
8f00507c   xdc_runtime_LoggerBuf_E_badLevel__C
8f005a60   xdc_runtime_LoggerBuf_Handle__label__S
0080e500   xdc_runtime_LoggerBuf_Instance_State_0_entryArr__A
8f005aa0   xdc_runtime_LoggerBuf_Instance_finalize__E
8f005880   xdc_runtime_LoggerBuf_Instance_init__E
8f005ba0   xdc_runtime_LoggerBuf_Module_GateProxy_enter__E
8f005bc0   xdc_runtime_LoggerBuf_Module_GateProxy_leave__E
0c394ea0   xdc_runtime_LoggerBuf_Module_GateProxy_query__E
8f004754   xdc_runtime_LoggerBuf_Module__FXNS__C
8f005080   xdc_runtime_LoggerBuf_Module__gateObj__C
8f005118   xdc_runtime_LoggerBuf_Module__id__C
008118b0   xdc_runtime_LoggerBuf_Module__root__V
008118b8   xdc_runtime_LoggerBuf_Module__state__V
8f005900   xdc_runtime_LoggerBuf_Module_startup__E
8f004b90   xdc_runtime_LoggerBuf_Object__DESC__C
8f004814   xdc_runtime_LoggerBuf_Object__PARAMS__C
8f005084   xdc_runtime_LoggerBuf_Object__count__C
8f0057a0   xdc_runtime_LoggerBuf_Object__create__S
8f005a00   xdc_runtime_LoggerBuf_Object__delete__S
8f005ae0   xdc_runtime_LoggerBuf_Object__get__S
008125f8   xdc_runtime_LoggerBuf_Object__table__V
0c394d20   xdc_runtime_LoggerBuf_TimestampProxy_get32__E
0c394d40   xdc_runtime_LoggerBuf_TimestampProxy_get64__E
0c394be0   xdc_runtime_LoggerBuf_TimestampProxy_getFreq__E
8f005be0   xdc_runtime_LoggerBuf_disable__E
8f005c00   xdc_runtime_LoggerBuf_enable__E
8f00511a   xdc_runtime_LoggerBuf_filterByLevel__C
8f005980   xdc_runtime_LoggerBuf_filterOutEvent__I
8f0056a0   xdc_runtime_LoggerBuf_getFilterLevel__E
8f005b20   xdc_runtime_LoggerBuf_reset__E
8f005580   xdc_runtime_LoggerBuf_setFilterLevel__E
8f005088   xdc_runtime_LoggerBuf_statusLogger__C
8f005b60   xdc_runtime_LoggerBuf_write0__E
8f005c20   xdc_runtime_LoggerBuf_write1__E
8f005c40   xdc_runtime_LoggerBuf_write2__E
8f0053c0   xdc_runtime_LoggerBuf_write4__E
8f005140   xdc_runtime_LoggerBuf_write8__E
0c394ea0   xdc_runtime_Main_Module_GateProxy_query__E
008118be   xdc_runtime_Main_Module__root__V
0c395520   xdc_runtime_Memory_HeapProxy_alloc__E
0c395540   xdc_runtime_Memory_HeapProxy_free__E
8f00511c   xdc_runtime_Memory_Module__id__C
008118c0   xdc_runtime_Memory_Module__state__V
0c3904a0   xdc_runtime_Memory_alloc__E
0c395560   xdc_runtime_Memory_calloc__E
8f00508c   xdc_runtime_Memory_defaultHeapInstance__C
0c394660   xdc_runtime_Memory_free__E
0c395580   xdc_runtime_Memory_getMaxDefaultTypeAlign__E
0c3939a0   xdc_runtime_Memory_valloc__E
008118c4   xdc_runtime_Registry_Module__state__V
0c3946a0   xdc_runtime_Registry_findById__E
0c3955a0   xdc_runtime_Startup_Module__startupDone__S
008118cc   xdc_runtime_Startup_Module__state__V
00000001   xdc_runtime_Startup__EXECFXN__C
00000001   xdc_runtime_Startup__RESETFXN__C
8f005090   xdc_runtime_Startup_execImpl__C
0c38f920   xdc_runtime_Startup_exec__E
0c3955c0   xdc_runtime_Startup_exec__I
8f004d60   xdc_runtime_Startup_firstFxns__A
8f004da0   xdc_runtime_Startup_firstFxns__C
8f004da8   xdc_runtime_Startup_lastFxns__C
8f005094   xdc_runtime_Startup_maxPasses__C
0c3852c0   xdc_runtime_Startup_reset__I
0c3955e0   xdc_runtime_Startup_rtsDone__E
8f004840   xdc_runtime_Startup_sfxnRts__A
8f005098   xdc_runtime_Startup_sfxnRts__C
8f0046c8   xdc_runtime_Startup_sfxnTab__A
8f00509c   xdc_runtime_Startup_sfxnTab__C
0c38b260   xdc_runtime_Startup_startMods__I
0c393a00   xdc_runtime_SysStd_abort__E
0c395600   xdc_runtime_SysStd_exit__E
0c395620   xdc_runtime_SysStd_putch__E
0c395640   xdc_runtime_SysStd_ready__E
0c395660   xdc_runtime_System_Module_GateProxy_enter__E
0c395680   xdc_runtime_System_Module_GateProxy_leave__E
0c394ea0   xdc_runtime_System_Module_GateProxy_query__E
008126c0   xdc_runtime_System_Module_State_0_atexitHandlers__A
8f0050a0   xdc_runtime_System_Module__gateObj__C
008118d4   xdc_runtime_System_Module__state__V
0c3956a0   xdc_runtime_System_Module_startup__E
0c393a00   xdc_runtime_System_SupportProxy_abort__E
0c395600   xdc_runtime_System_SupportProxy_exit__E
0c395620   xdc_runtime_System_SupportProxy_putch__E
0c395640   xdc_runtime_System_SupportProxy_ready__E
8f0050a4   xdc_runtime_System_abortFxn__C
0c394a40   xdc_runtime_System_abortStd__E
0c3946e0   xdc_runtime_System_abort__E
0c394720   xdc_runtime_System_aprintf__E
0c3956c0   xdc_runtime_System_aprintf_va__E
0c3956c0   xdc_runtime_System_aprintf_va__F
0c392c60   xdc_runtime_System_atexit__E
0c393a60   xdc_runtime_System_avprintf__E
0c380000   xdc_runtime_System_doPrint__I
8f0050a8   xdc_runtime_System_exitFxn__C
0c390b20   xdc_runtime_System_exitStd__E
0c394760   xdc_runtime_System_exit__E
8f0050ac   xdc_runtime_System_extendFxn__C
0c391420   xdc_runtime_System_formatNum__I
8f0050b0   xdc_runtime_System_maxAtexitHandlers__C
0c3884a0   xdc_runtime_System_printfExtend__I
0c3947a0   xdc_runtime_System_printf__E
0c3956e0   xdc_runtime_System_printf_va__E
0c3956e0   xdc_runtime_System_printf_va__F
0c392ce0   xdc_runtime_System_processAtExit__E
0c392d60   xdc_runtime_System_putchar__I
0c393ac0   xdc_runtime_System_vprintf__E
0c395700   xdc_runtime_System_vsnprintf__E
008118dc   xdc_runtime_Text_Module__state__V
8f00511e   xdc_runtime_Text_charCnt__C
8f000000   xdc_runtime_Text_charTab__A
8f0050b4   xdc_runtime_Text_charTab__C
0c393b20   xdc_runtime_Text_cordText__E
8f005120   xdc_runtime_Text_isLoaded__C
8f0050b8   xdc_runtime_Text_nameEmpty__C
8f0050bc   xdc_runtime_Text_nameStatic__C
8f0050c0   xdc_runtime_Text_nameUnknown__C
8f004100   xdc_runtime_Text_nodeTab__A
8f0050c4   xdc_runtime_Text_nodeTab__C
0c392de0   xdc_runtime_Text_printVisFxn__I
0c38ebe0   xdc_runtime_Text_putLab__E
0c38ed00   xdc_runtime_Text_putMod__E
0c38bb40   xdc_runtime_Text_putSite__E
8f005122   xdc_runtime_Text_registryModsLastId__C
0c3947e0   xdc_runtime_Text_ropeText__E
8f005124   xdc_runtime_Text_unnamedModsLastId__C
0c390580   xdc_runtime_Text_visitRope2__I
8f0050c8   xdc_runtime_Text_visitRopeFxn__C
0c395720   xdc_runtime_Text_visitRope__I
0c391e40   xdc_runtime_Text_xprintf__I
0c394d20   xdc_runtime_Timestamp_SupportProxy_get32__E
0c394d40   xdc_runtime_Timestamp_SupportProxy_get64__E
0c394be0   xdc_runtime_Timestamp_SupportProxy_getFreq__E
0c394d20   xdc_runtime_Timestamp_get32__E
0c394d40   xdc_runtime_Timestamp_get64__E
0c394be0   xdc_runtime_Timestamp_getFreq__E
0c394820   xdc_runtime_knl_GateThread_Handle__label__S
0c394860   xdc_runtime_knl_GateThread_Instance_finalize__E
0c3948a0   xdc_runtime_knl_GateThread_Instance_init__E
8f004988   xdc_runtime_knl_GateThread_Module__FXNS__C
008118e4   xdc_runtime_knl_GateThread_Module__root__V
0c395740   xdc_runtime_knl_GateThread_Module__startupDone__S
8f004bb0   xdc_runtime_knl_GateThread_Object__DESC__C
8f004cf0   xdc_runtime_knl_GateThread_Object__PARAMS__C
0c390660   xdc_runtime_knl_GateThread_Object__create__S
0c393b80   xdc_runtime_knl_GateThread_Object__delete__S
0c395760   xdc_runtime_knl_GateThread_Proxy_Object__create__S
0c395780   xdc_runtime_knl_GateThread_Proxy_Object__delete__S
0c3957a0   xdc_runtime_knl_GateThread_Proxy_create
0c3957c0   xdc_runtime_knl_GateThread_Proxy_delete
0c3957e0   xdc_runtime_knl_GateThread_Proxy_enter__E
0c395800   xdc_runtime_knl_GateThread_Proxy_leave__E
0c394f00   xdc_runtime_knl_GateThread_Proxy_query__E
0c390740   xdc_runtime_knl_GateThread_create
0c395820   xdc_runtime_knl_GateThread_enter__E
0c395840   xdc_runtime_knl_GateThread_leave__E
0c394f00   xdc_runtime_knl_GateThread_query__E


GLOBAL SYMBOLS: SORTED BY Symbol Address 

address    name
--------   ----
00000000   _argsize
00000001   __TI_args_main
00000001   xdc_runtime_Startup__EXECFXN__C
00000001   xdc_runtime_Startup__RESETFXN__C
00001000   __TI_STACK_SIZE
00008000   ti_sysbios_family_c66_Cache_l1dSize
00008000   ti_sysbios_family_c66_Cache_l1pSize
00020000   ti_sysbios_family_c66_Cache_l2Size
00800000   __ASM__
00800000   ti_sysbios_family_c64p_Hwi_Instance_State_0_hookEnv__A
00800008   ti_sysbios_heaps_HeapMem_Instance_State_6_buf__A
00800070   __ISA__
00800088   __PLAT__
008000a8   __TARG__
008000d0   __TRDR__
00808008   ti_sysbios_knl_Swi_Instance_State_0_hookEnv__A
00808010   ti_sysbios_knl_Task_Instance_State_0_hookEnv__A
00808080   ti_uia_loggers_LoggerStopMode_Instance_State_0_hdr__A
00808200   ti_uia_loggers_LoggerStopMode_Instance_State_0_packetArray__A
0080a200   ti_uia_loggers_LoggerStopMode_Instance_State_1_hdr__A
0080a380   ti_uia_loggers_LoggerStopMode_Instance_State_1_packetArray__A
0080c380   ti_uia_loggers_LoggerStopMode_Instance_State_2_hdr__A
0080c500   ti_uia_loggers_LoggerStopMode_Instance_State_2_packetArray__A
0080e500   xdc_runtime_LoggerBuf_Instance_State_0_entryArr__A
0080f500   ti_sysbios_knl_Task_Instance_State_0_stack__A
0080fd00   _tmpnams
0080fe48   __CIOBUF_
0080ff68   _stack
00810f68   __TI_STACK_END
00810f68   ti_sysbios_family_c66_tci66xx_CpIntc_Module_State_0_dispatchTab__A
00811468   ti_sdo_ipc_GateMP_Module__root__V
00811470   ti_sdo_ipc_GateMP_Module__state__V
008114c0   ti_sdo_ipc_Ipc_Module__state__V
008114cc   ti_sdo_ipc_ListMP_Module__root__V
008114d4   ti_sdo_ipc_ListMP_Module__state__V
008114d8   ti_sdo_ipc_MessageQ_Module__root__V
008114e0   ti_sdo_ipc_MessageQ_Module__state__V
00811548   ti_sdo_ipc_Notify_Module__root__V
00811550   ti_sdo_ipc_Notify_Module__state__V
00811558   ti_sdo_ipc_SharedRegion_Module__state__V
0081155c   ti_sdo_ipc_family_c647x_Interrupt_Module__state__V
00811568   ti_sdo_ipc_gates_GateHWSem_Module__root__V
00811570   ti_sdo_ipc_gates_GateMPSupportNull_Module__root__V
00811578   ti_sdo_ipc_heaps_HeapBufMP_Module__root__V
00811580   ti_sdo_ipc_heaps_HeapBufMP_Module__state__V
00811584   ti_sdo_ipc_heaps_HeapMemMP_Module__root__V
0081158c   ti_sdo_ipc_heaps_HeapMemMP_Module__state__V
00811590   ti_sdo_ipc_notifyDrivers_NotifyDriverShm_Module__root__V
00811598   ti_sdo_ipc_nsremote_NameServerRemoteNotify_Module__root__V
008115a0   ti_sdo_ipc_transports_TransportShm_Module__root__V
008115a8   ti_sdo_ipc_transports_TransportShmSetup_Module__state__V
008115ac   ti_sdo_utils_List_Module__root__V
008115b4   ti_sdo_utils_MultiProc_Module__state__V
008115bc   ti_sdo_utils_NameServer_Module__root__V
008115c4   ti_sdo_utils_NameServer_Module__state__V
008115d0   ti_sdo_utils_NameServerRemoteNull_Module__root__V
008115d8   ti_sysbios_BIOS_Module__state__V
008115fc   ti_sysbios_family_c64p_Exception_Module__state__V
0081162c   ti_sysbios_family_c64p_Hwi_Module__root__V
00811634   ti_sysbios_family_c64p_Hwi_Module__state__V
008116a0   ti_sysbios_family_c66_tci66xx_CpIntc_Module__state__V
008116b0   ti_sysbios_gates_GateAll_Module__root__V
008116b8   ti_sysbios_gates_GateHwi_Module__root__V
008116c0   ti_sysbios_gates_GateMutex_Module__root__V
008116c8   ti_sysbios_gates_GateMutexPri_Module__root__V
008116d0   ti_sysbios_gates_GateSwi_Module__root__V
008116d8   ti_sysbios_hal_Hwi_Module__root__V
008116e0   ti_sysbios_hal_Timer_Module__root__V
008116e8   ti_sysbios_heaps_HeapMem_Module__root__V
008116f0   ti_sysbios_knl_Clock_Module__root__V
008116f8   ti_sysbios_knl_Clock_Module__state__V
00811724   ti_sysbios_knl_Event_Module__root__V
00811730   ti_sysbios_knl_Queue_Module__root__V
00811738   ti_sysbios_knl_Semaphore_Module__root__V
00811740   ti_sysbios_knl_Swi_Module__root__V
00811748   ti_sysbios_knl_Swi_Module__state__V
00811764   ti_sysbios_knl_Task_Module__root__V
00811770   ti_sysbios_knl_Task_Module__state__V
008117b4   ti_sysbios_rts_ti_ThreadLocalStorage_Module__state__V
008117c0   ti_sysbios_syncs_SyncSem_Module__root__V
008117c8   ti_sysbios_timers_timer64_Timer_Module__root__V
008117d0   ti_sysbios_timers_timer64_Timer_Module__state__V
008117e8   ti_sysbios_utils_Load_Module__state__V
00811880   ti_sysbios_xdcruntime_GateThreadSupport_Module__root__V
00811888   ti_uia_loggers_LoggerStopMode_Module__root__V
00811890   ti_uia_loggers_LoggerStopMode_Module__state__V
00811898   ti_uia_runtime_QueueDescriptor_Module__state__V
008118a4   xdc_runtime_Error_Module__state__V
008118a8   xdc_runtime_GateNull_Module__root__V
008118b0   xdc_runtime_LoggerBuf_Module__root__V
008118b8   xdc_runtime_LoggerBuf_Module__state__V
008118be   xdc_runtime_Main_Module__root__V
008118c0   xdc_runtime_Memory_Module__state__V
008118c4   xdc_runtime_Registry_Module__state__V
008118cc   xdc_runtime_Startup_Module__state__V
008118d4   xdc_runtime_System_Module__state__V
008118dc   xdc_runtime_Text_Module__state__V
008118e4   xdc_runtime_knl_GateThread_Module__root__V
008118ec   __xdc__init__addr
008118f0   _ftable
00811ad0   ti_sysbios_timers_timer64_Timer_Module_State_0_device__A
00811c50   ti_sdo_utils_NameServer_Object__table__V
00811d7c   _ft_end
00811d80   ti_sysbios_heaps_HeapMem_Object__table__V
00811ec8   ti_sdo_ipc_Ipc_Module_State_0_procEntry__A
00811f68   ti_uia_loggers_LoggerStopMode_Object__table__V
00812008   ti_sysbios_family_c66_tci66xx_CpIntc_Module_State_0_hostIntToSysInt__A
008120a0   ti_sdo_ipc_SharedRegion_Module_State_0_regions__A
00812130   ti_sdo_ipc_GateMP_Module_State_0_remoteSystemGates__A
008121b0   ti_sysbios_knl_Swi_Module_State_0_readyQ__A
00812230   ti_sysbios_knl_Task_Module_State_0_readyQ__A
008122b0   ti_sysbios_timers_timer64_Timer_Module_State_0_gctrl__A
00812330   ti_sysbios_timers_timer64_Timer_Module_State_0_handles__A
008123b0   ti_sysbios_timers_timer64_Timer_Module_State_0_intFreqs__A
008124a8   ti_sysbios_knl_Task_Object__table__V
008124f8   ti_sysbios_timers_timer64_Timer_Object__table__V
00812548   ti_sdo_ipc_MessageQ_Module_State_0_transports__A
00812588   ti_sysbios_gates_GateMutex_Object__table__V
008125c8   ti_sysbios_knl_Swi_Object__table__V
008125f8   xdc_runtime_LoggerBuf_Object__table__V
00812620   ti_sdo_ipc_MessageQ_Module_State_0_heaps__A
00812640   ti_sdo_ipc_Notify_Module_State_0_notifyHandles__A
00812660   ti_sdo_ipc_family_c647x_Interrupt_Module_State_0_args__A
00812680   ti_sdo_ipc_transports_TransportShmSetup_Module_State_0_handles__A
008126a0   ti_sdo_utils_NameServer_Module_State_0_nsRemoteHandle__A
008126c0   xdc_runtime_System_Module_State_0_atexitHandlers__A
008126e0   ti_sysbios_utils_Load_Module_State_0_taskEnv__A
00812700   ti_sysbios_family_c64p_Hwi_Object__table__V
00812718   ti_sysbios_gates_GateMutexPri_Object__table__V
00812730   ti_sysbios_family_c66_tci66xx_CpIntc_Module_State_0_initSIER__A
00812748   ti_sdo_utils_MultiProc_Module_State_0_clusterProcList__A
00812758   ti_sysbios_family_c66_tci66xx_CpIntc_Module_State_0_controller__A
00812768   ti_sysbios_gates_GateAll_Object__table__V
00812778   _cleanup_ptr
0081277c   _dtors_ptr
00812780   __TI_enable_exit_profile_output
00812788   ti_sysbios_gates_GateSwi_Object__table__V
00812794   _lock
00812798   _unlock
008127a0   ti_sysbios_hal_Hwi_Object__table__V
008127a8   ti_sdo_ipc_Notify_Module_State_0_notifyHandles_0__A
008127b0   ti_sdo_ipc_Notify_Module_State_0_notifyHandles_1__A
008127b8   ti_sdo_ipc_Notify_Module_State_0_notifyHandles_2__A
008127c0   ti_sdo_ipc_Notify_Module_State_0_notifyHandles_3__A
008127c8   ti_sdo_ipc_Notify_Module_State_0_notifyHandles_4__A
008127d0   ti_sdo_ipc_Notify_Module_State_0_notifyHandles_5__A
008127d8   ti_sdo_ipc_Notify_Module_State_0_notifyHandles_6__A
008127e0   ti_sdo_ipc_Notify_Module_State_0_notifyHandles_7__A
008127e8   ti_sysbios_gates_GateHwi_Object__table__V
008127f0   ti_sysbios_knl_Task_Module_State_0_idleTask__A
008127f8   ti_sysbios_utils_Load_Module_State_0_runningTask__A
00812800   ti_sysbios_utils_Load_Module_State_0_taskStartTime__A
00812808   xdc_runtime_GateNull_Object__table__V
0081280c   __TI_STATIC_BASE
0081280c   ti_uia_runtime_QueueDescriptor_gPtrToFirstDescriptor
00812810   ti_uia_runtime_QueueDescriptor_gUpdateCount
0c380000   xdc_runtime_System_doPrint__I
0c380880   ti_sysbios_family_c64p_Exception_handler__I
0c381000   ti_sysbios_knl_Semaphore_pend__E
0c381760   ti_sysbios_timers_timer64_Timer_Module_startup__E
0c381e00   ti_sysbios_heaps_HeapMem_allocUnprotected__E
0c382420   __c6xabi_divd
0c382fa0   ti_sysbios_heaps_HeapMem_freeUnprotected__E
0c383a80   ti_sysbios_knl_Task_Module_startup__E
0c383f00   _printfi
0c384360   ti_sysbios_gates_GateMutexPri_enter__E
0c384760   ti_sdo_ipc_Notify_Instance_init__E
0c384b40   ti_sysbios_knl_Task_setPri__E
0c384f20   fputs
0c3852c0   ti_sysbios_family_c66_Cache_startup__I
0c3852c0   xdc_runtime_Startup_reset__I
0c385660   ti_sysbios_family_c64p_Hwi_dispatchCore__I
0c385d00   ti_sysbios_utils_Load_logLoads__I
0c386680   ti_sysbios_knl_Swi_run__I
0c386980   ti_sysbios_timers_timer64_Timer_deviceConfig__I
0c386c80   SharedRegion_getEntry
0c387240   ti_sysbios_heaps_HeapMem_Instance_init__E
0c3877e0   ti_sysbios_family_c66_tci66xx_CpIntc_Module_startup__E
0c387aa0   ti_sysbios_family_c64p_Hwi_Module_startup__E
0c387d40   ti_sysbios_knl_Clock_workFunc__E
0c387fe0   ti_sysbios_knl_Swi_Module_startup__E
0c388240   ti_sysbios_utils_Load_updateThreadContexts__E
0c3884a0   xdc_runtime_System_printfExtend__I
0c388700   __c6xabi_divull
0c388b80   ti_sysbios_family_c64p_Exception_internalHandler__I
0c388dc0   ti_sysbios_knl_Semaphore_post__E
0c389000   ti_uia_loggers_LoggerStopMode_writeMemoryRange__E
0c389460   fputc
0c389680   ti_sysbios_knl_Task_schedule__I
0c3898a0   ti_sysbios_timers_timer64_Timer_setPeriodMicroSecs__E
0c389ac0   xdc_runtime_Core_createObject__I
0c389ce0   MultiProc_getId
0c38a0e0   ti_sysbios_family_c64p_Hwi_dispatchAlways
0c38a2e0   setvbuf
0c38a4e0   ti_sdo_ipc_family_c647x_MultiProcSetup_init__I
0c38a6e0   ti_sysbios_knl_Task_startCore__E
0c38a8e0   ti_sysbios_utils_Load_updateLoads__E
0c38a8e0   ti_sysbios_utils_Load_update__E
0c38aae0   ti_sysbios_knl_Task_exit__E
0c38acc0   ti_sysbios_timers_timer64_Timer_getFreq__E
0c38aea0   ti_sysbios_utils_Load_idleFxn__E
0c38b080   xdc_runtime_Error_policyDefault__E
0c38b260   xdc_runtime_Startup_startMods__I
0c38b600   ti_sysbios_family_c66_Cache_block__I
0c38b7c0   ti_sysbios_knl_Swi_post__E
0c38b980   ti_sysbios_knl_Task_checkStacks__E
0c38bb40   xdc_runtime_Text_putSite__E
0c38bd00   HOSTrename
0c38bea0   MultiProc_setLocalId
0c38c040   __c6xabi_divul
0c38c1e0   ti_sysbios_gates_GateMutex_enter__E
0c38c380   ti_sysbios_knl_Task_unblockI__E
0c38c520   ti_sysbios_timers_timer64_Timer_start__E
0c38c840   ti_sysbios_family_c64p_Exception_dispatch__E
0c38c9c0   ti_sysbios_family_c66_Cache_getL2InitSize__I
0c38cb40   ti_sysbios_utils_Load_startup__E
0c38ccc0   ti_sysbios_utils_Load_taskCreateHook__E
0c38ce40   ti_uia_loggers_LoggerStopMode_write8__E
0c38cfc0   xdc_runtime_Core_constructObject__I
0c38d140   ti_sdo_ipc_Notify_Module_startup__E
0c38d2a0   ti_uia_loggers_LoggerStopMode_write4__E
0c38d400   _auto_init_elf
0c38d7c0   ti_sdo_utils_NameServer_Module_startup__E
0c38d900   ti_sysbios_gates_GateSwi_enter__E
0c38da40   ti_sysbios_knl_Semaphore_Instance_init__E
0c38db80   ti_sysbios_knl_Task_blockI__E
0c38dcc0   ti_uia_loggers_LoggerStopMode_initQueueDescriptor__E
0c38de00   ti_uia_loggers_LoggerStopMode_write0__E
0c38df40   ti_uia_loggers_LoggerStopMode_write1__E
0c38e080   ti_uia_loggers_LoggerStopMode_write2__E
0c38e1c0   _closefile
0c38e400   fseek
0c38e520   ti_sdo_ipc_MessageQ_Module_startup__E
0c38e640   ti_sysbios_utils_Load_taskDeleteHook__E
0c38e760   ti_sysbios_utils_Load_updateCurrentThreadTime__E
0c38e880   ti_uia_loggers_LoggerStopMode_Module_startup__E
0c38e9a0   ti_uia_runtime_QueueDescriptor_addToList__E
0c38eac0   xdc_runtime_Core_deleteObject__I
0c38ebe0   xdc_runtime_Text_putLab__E
0c38ed00   xdc_runtime_Text_putMod__E
0c38ee20   HOSTlseek
0c38ef20   _wrt_ok
0c38f020   ti_sdo_ipc_Notify_Instance_finalize__E
0c38f120   ti_sdo_ipc_Notify_create
0c38f220   ti_sdo_ipc_family_c647x_Interrupt_Module_startup__E
0c38f320   ti_sdo_ipc_gates_GateHWSem_Module_startup__E
0c38f420   ti_sysbios_gates_GateMutexPri_leave__E
0c38f520   ti_sysbios_knl_Swi_restoreHwi__E
0c38f620   ti_sysbios_timers_timer64_Timer_initDevice__I
0c38f720   ti_sysbios_utils_Load_hwiBeginHook__E
0c38f820   ti_sysbios_xdcruntime_GateThreadSupport_leave__E
0c38f920   xdc_runtime_Startup_exec__E
0c38fa20   HOSTopen
0c38fb00   HOSTread
0c38fcc0   atoi
0c38fda0   close
0c38fe80   fflush
0c38ff60   ltoa
0c390040   memset
0c390120   printf
0c390200   ti_sysbios_knl_Swi_runLoop__I
0c3902e0   ti_sysbios_hal_Timer_TimerProxy_startup__E
0c3902e0   ti_sysbios_hal_Timer_startup__E
0c3902e0   ti_sysbios_knl_Clock_TimerProxy_startup__E
0c3902e0   ti_sysbios_timers_timer64_Timer_startup__E
0c3903c0   xdc_runtime_Error_print__E
0c3904a0   xdc_runtime_Memory_alloc__E
0c390580   xdc_runtime_Text_visitRope2__I
0c390660   xdc_runtime_knl_GateThread_Object__create__S
0c390740   xdc_runtime_knl_GateThread_create
0c390820   HOSTunlink
0c3908e0   HOSTwrite
0c3909a0   __c6xabi_divu
0c3909a0   __divu
0c390a60   _doflush
0c390b20   exit
0c390b20   xdc_runtime_System_exitStd__E
0c390be0   setMyId
0c390c80   main
0c390ca0   ti_sysbios_gates_GateAll_leave__E
0c390d60   ti_sysbios_heaps_HeapMem_alloc__E
0c390e20   ti_sysbios_heaps_HeapMem_getStats__E
0c390ee0   ti_sysbios_knl_Clock_logTick__E
0c390fa0   ti_sysbios_knl_Swi_schedule__I
0c391060   ti_sysbios_knl_Task_allBlockedFunction__I
0c391120   ti_sysbios_timers_timer64_Timer_stop__E
0c3911e0   ti_sysbios_utils_Load_taskSwitchHook__E
0c3912a0   ti_uia_loggers_LoggerStopMode_flush__E
0c391360   __TI_tls_init
0c391420   xdc_runtime_System_formatNum__I
0c3914e0   HOSTclose
0c391580   __c6xabi_remu
0c391580   __remu
0c391620   _cleanup
0c391940   lseek
0c3919e0   memcpy
0c391a80   ti_sysbios_family_c64p_Exception_Module_startup__E
0c391b20   ti_sysbios_heaps_HeapMem_init__I
0c391bc0   ti_sysbios_utils_Load_swiBeginHook__E
0c391c60   write
0c391d00   xdc_runtime_Assert_raise__I
0c391da0   xdc_runtime_Error_setX__E
0c391e40   xdc_runtime_Text_xprintf__I
0c391ee0   __c6xabi_llshl
0c391f60   ti_sysbios_family_c62_TaskSupport_swap__E
0c391f60   ti_sysbios_knl_Task_SupportProxy_swap__E
0c391fe0   malloc
0c392060   readmsg
0c3920e0   ti_sysbios_BIOS_atExitFunc__I
0c392160   ti_sysbios_family_c64p_Hwi_dispatchC__I
0c3921e0   ti_sysbios_family_c64p_Hwi_getStackInfo__E
0c3921e0   ti_sysbios_hal_Hwi_HwiProxy_getStackInfo__E
0c3921e0   ti_sysbios_hal_Hwi_getStackInfo__E
0c392260   ti_sysbios_gates_GateAll_Object__create__S
0c3922e0   ti_sysbios_gates_GateHwi_Object__create__S
0c392360   ti_sysbios_gates_GateMutexPri_Object__create__S
0c3923e0   ti_sysbios_gates_GateMutex_Object__create__S
0c392460   ti_sysbios_gates_GateSwi_Object__create__S
0c3924e0   ti_sysbios_gates_GateSwi_leave__E
0c392560   ti_sysbios_hal_Hwi_checkStack
0c3925e0   ti_sysbios_hal_Hwi_initStack
0c392660   ti_sysbios_heaps_HeapMem_Object__create__S
0c3926e0   ti_sysbios_knl_Clock_doTick__I
0c392760   ti_sysbios_knl_Idle_run__E
0c3927e0   ti_sysbios_knl_Swi_startup__E
0c392860   ti_sysbios_knl_Task_restore__E
0c3928e0   ti_sysbios_utils_Load_hwiEndHook__E
0c392960   ti_sysbios_utils_Load_swiEndHook__E
0c3929e0   ti_sysbios_xdcruntime_GateThreadSupport_Object__create__S
0c392a60   ti_uia_loggers_LoggerStopMode_Object__create__S
0c392ae0   remove
0c392ae0   unlink
0c392b60   xdc_runtime_Core_assignLabel__I
0c392be0   xdc_runtime_Core_assignParams__I
0c392c60   xdc_runtime_System_atexit__E
0c392ce0   xdc_runtime_System_processAtExit__E
0c392d60   xdc_runtime_System_putchar__I
0c392de0   xdc_runtime_Text_printVisFxn__I
0c392e60   __c6xabi_frcmpyd_div
0c392ec0   __c6xabi_llshru
0c392f20   _subcull
0c392f80   ti_sysbios_family_c64p_Hwi_switchAndDispatch__I
0c392fe0   ti_sysbios_family_xxx_Hwi_switchAndRunFunc
0c393040   memccpy
0c3930a0   ti_sdo_utils_List_construct
0c393100   ti_sysbios_BIOS_errorRaiseHook__I
0c393160   ti_sysbios_BIOS_registerRTSLock__I
0c3931c0   ti_sysbios_BIOS_removeRTSLock__I
0c393220   ti_sysbios_BIOS_rtsLock__I
0c393280   ti_sysbios_BIOS_startFunc__I
0c3932e0   ti_sysbios_family_c62_TaskSupport_start__E
0c3932e0   ti_sysbios_knl_Task_SupportProxy_start__E
0c393340   ti_sysbios_family_c66_Cache_Module_startup__E
0c3933a0   ti_sysbios_family_c66_tci66xx_CpIntc_unused__E
0c393400   ti_sysbios_gates_GateAll_enter__E
0c393460   ti_sysbios_gates_GateMutexPri_Object__delete__S
0c3934c0   ti_sysbios_gates_GateMutexPri_construct
0c393520   ti_sysbios_gates_GateMutex_Object__delete__S
0c393580   ti_sysbios_heaps_HeapMem_free__E
0c3935e0   ti_sysbios_knl_Clock_Module_startup__E
0c393640   ti_sysbios_knl_Queue_construct
0c3936a0   ti_sysbios_knl_Semaphore_construct
0c393700   ti_sysbios_knl_Semaphore_pendTimeout__I
0c393760   ti_sysbios_knl_Task_enter__I
0c3937c0   ti_sysbios_xdcruntime_GateThreadSupport_Object__delete__S
0c393820   ti_uia_loggers_LoggerStopMode_Instance_init__E
0c393880   ti_uia_loggers_LoggerStopMode_initBuffer__I
0c3938e0   ti_uia_loggers_LoggerStopMode_reset__E
0c393940   writemsg
0c393998   C$$IO$$
0c3939a0   xdc_runtime_Memory_valloc__E
0c393a00   xdc_runtime_SysStd_abort__E
0c393a00   xdc_runtime_System_SupportProxy_abort__E
0c393a60   xdc_runtime_System_avprintf__E
0c393ac0   xdc_runtime_System_vprintf__E
0c393b20   xdc_runtime_Text_cordText__E
0c393b80   xdc_runtime_knl_GateThread_Object__delete__S
0c393be0   __c6xabi_isinf
0c393c60   _args_main
0c393ca0   ti_sysbios_family_c62_TaskSupport_buildTaskStack
0c393ce0   free
0c393d20   ti_sdo_utils_NameServer_Module__startupDone__F
0c393d20   ti_sdo_utils_NameServer_Module__startupDone__S
0c393d60   ti_sdo_utils_NameServer_Object__get__S
0c393da0   ti_sysbios_BIOS_exitFunc__I
0c393de0   ti_sysbios_BIOS_rtsUnlock__I
0c393e20   ti_sysbios_family_c64p_Hwi_Module__startupDone__F
0c393e20   ti_sysbios_family_c64p_Hwi_Module__startupDone__S
0c393e60   ti_sysbios_family_c64p_Hwi_disableInterrupt__E
0c393e60   ti_sysbios_hal_Hwi_HwiProxy_disableInterrupt__E
0c393e60   ti_sysbios_hal_Hwi_disableInterrupt__E
0c393ea0   ti_sysbios_family_c64p_Hwi_enableInterrupt__E
0c393ea0   ti_sysbios_hal_Hwi_HwiProxy_enableInterrupt__E
0c393ea0   ti_sysbios_hal_Hwi_enableInterrupt__E
0c393ee0   ti_sysbios_gates_GateAll_Handle__label__S
0c393f20   ti_sysbios_gates_GateAll_Object__delete__S
0c393f60   ti_sysbios_gates_GateHwi_Handle__label__S
0c393fa0   ti_sysbios_gates_GateHwi_Object__delete__S
0c393fe0   ti_sysbios_gates_GateMutexPri_Handle__label__S
0c394020   ti_sysbios_gates_GateMutexPri_Instance_init__E
0c394060   ti_sysbios_gates_GateMutexPri_Object__destruct__S
0c3940a0   ti_sysbios_gates_GateMutex_Handle__label__S
0c3940e0   ti_sysbios_gates_GateMutex_Instance_init__E
0c394120   ti_sysbios_gates_GateMutex_leave__E
0c394160   ti_sysbios_gates_GateSwi_Handle__label__S
0c3941a0   ti_sysbios_gates_GateSwi_Object__delete__S
0c3941e0   ti_sysbios_heaps_HeapMem_Handle__label__S
0c394220   ti_sysbios_heaps_HeapMem_Object__delete__S
0c394260   ti_sysbios_heaps_HeapMem_Object__get__S
0c3942a0   ti_sysbios_knl_Semaphore_Object__destruct__S
0c3942e0   ti_sysbios_knl_Swi_Object__get__S
0c394320   ti_sysbios_knl_Task_Object__get__S
0c394360   ti_sysbios_timers_timer64_Timer_Module__startupDone__F
0c394360   ti_sysbios_timers_timer64_Timer_Module__startupDone__S
0c3943a0   ti_sysbios_xdcruntime_GateThreadSupport_Instance_init__E
0c3943e0   ti_uia_loggers_LoggerStopMode_Handle__label__S
0c394420   ti_uia_loggers_LoggerStopMode_Object__delete__S
0c394460   ti_uia_loggers_LoggerStopMode_Object__get__S
0c3944a0   ti_uia_loggers_LoggerStopMode_disable__E
0c3944e0   ti_uia_loggers_LoggerStopMode_enable__E
0c394520   xdc_runtime_Error_check__E
0c394560   xdc_runtime_Error_init__E
0c3945a0   xdc_runtime_GateNull_Handle__label__S
0c3945e0   xdc_runtime_GateNull_Object__create__S
0c394620   xdc_runtime_GateNull_Object__delete__S
0c394660   xdc_runtime_Memory_free__E
0c3946a0   xdc_runtime_Registry_findById__E
0c3946e0   xdc_runtime_System_abort__E
0c394720   xdc_runtime_System_aprintf__E
0c394760   xdc_runtime_System_exit__E
0c3947a0   xdc_runtime_System_printf__E
0c3947e0   xdc_runtime_Text_ropeText__E
0c394820   xdc_runtime_knl_GateThread_Handle__label__S
0c394860   xdc_runtime_knl_GateThread_Instance_finalize__E
0c3948a0   xdc_runtime_knl_GateThread_Instance_init__E
0c3948e0   LoggerBuf_instanceStartup
0c394900   MultiProc_getNumProcessors
0c394920   __c6xabi_negll
0c394940   __xdc__init
0c394960   _nop
0c3949c0   _register_lock
0c3949e0   _register_synch_api
0c394a00   _register_unlock
0c394a20   ti_sysbios_family_c62_TaskSupport_glue
0c394a40   C$$EXIT
0c394a40   abort
0c394a40   xdc_runtime_System_abortStd__E
0c394a60   __TI_decompress_none
0c394a80   __TI_decompress_rle24
0c394aa0   putc
0c394ac0   putchar
0c394ae0   ti_sdo_ipc_MessageQ_Object__get__S
0c394b00   ti_sdo_utils_List_Instance_init__E
0c394b20   ti_sdo_utils_List_Object__destruct__S
0c394b40   ti_sdo_utils_List_Object__get__S
0c394b60   ti_sdo_utils_List_destruct
0c394b80   ti_sdo_utils_MultiProc_getClusterId__E
0c394b80   ti_sdo_utils_MultiProc_getClusterId__F
0c394ba0   ti_sysbios_BIOS_RtsGateProxy_enter__E
0c394bc0   ti_sysbios_BIOS_RtsGateProxy_leave__E
0c394be0   ti_sysbios_BIOS_getCpuFreq__E
0c394be0   ti_sysbios_family_c64p_TimestampProvider_getFreq__E
0c394be0   xdc_runtime_LoggerBuf_TimestampProxy_getFreq__E
0c394be0   xdc_runtime_Timestamp_SupportProxy_getFreq__E
0c394be0   xdc_runtime_Timestamp_getFreq__E
0c394c00   ti_sysbios_BIOS_linkedWithIncorrectBootLibrary__E
0c394c20   ti_sysbios_BIOS_nullFunc__I
0c394c40   ti_sysbios_BIOS_setThreadType__E
0c394c60   ti_sysbios_family_c62_TaskSupport_Module__startupDone__S
0c394c80   ti_sysbios_family_c62_TaskSupport_checkStack__E
0c394c80   ti_sysbios_knl_Task_SupportProxy_checkStack__E
0c394ca0   ti_sysbios_family_c64p_Hwi_clearInterrupt__E
0c394ca0   ti_sysbios_hal_Hwi_HwiProxy_clearInterrupt__E
0c394ca0   ti_sysbios_hal_Hwi_clearInterrupt__E
0c394cc0   ti_sysbios_family_c64p_Hwi_startup__E
0c394cc0   ti_sysbios_hal_Hwi_HwiProxy_startup__E
0c394cc0   ti_sysbios_hal_Hwi_startup__E
0c394ce0   ti_sysbios_family_c64p_Hwi_switchFromBootStack__E
0c394ce0   ti_sysbios_hal_Hwi_HwiProxy_switchFromBootStack__E
0c394d00   ti_sysbios_family_c64p_TimestampProvider_Module_startup__E
0c394d20   ti_sysbios_family_c64p_TimestampProvider_get32__E
0c394d20   xdc_runtime_LoggerBuf_TimestampProxy_get32__E
0c394d20   xdc_runtime_Timestamp_SupportProxy_get32__E
0c394d20   xdc_runtime_Timestamp_get32__E
0c394d40   ti_sysbios_family_c64p_TimestampProvider_get64__E
0c394d40   xdc_runtime_LoggerBuf_TimestampProxy_get64__E
0c394d40   xdc_runtime_Timestamp_SupportProxy_get64__E
0c394d40   xdc_runtime_Timestamp_get64__E
0c394d60   ti_sysbios_family_c64p_tci6488_TimerSupport_enable__E
0c394d60   ti_sysbios_timers_timer64_Timer_TimerSupportProxy_enable__E
0c394d80   ti_sysbios_family_c66_Cache_RTSSynchInv__I
0c394da0   ti_sysbios_family_c66_Cache_RTSSynchWbInv__I
0c394dc0   ti_sysbios_family_c66_Cache_RTSSynchWb__I
0c394de0   ti_sysbios_family_c66_Cache_wait__E
0c394de0   ti_sysbios_hal_Cache_CacheProxy_wait__E
0c394de0   ti_sysbios_hal_Cache_wait__E
0c394e00   ti_sysbios_gates_GateAll_Instance_init__E
0c394e20   ti_sysbios_gates_GateAll_query__E
0c394e40   ti_sysbios_gates_GateHwi_Instance_init__E
0c394e60   ti_sysbios_gates_GateHwi_enter__E
0c394e80   ti_sysbios_gates_GateHwi_leave__E
0c394ea0   ti_sysbios_gates_GateHwi_query__E
0c394ea0   xdc_runtime_LoggerBuf_Module_GateProxy_query__E
0c394ea0   xdc_runtime_Main_Module_GateProxy_query__E
0c394ea0   xdc_runtime_System_Module_GateProxy_query__E
0c394ec0   ti_sysbios_gates_GateMutexPri_Instance_finalize__E
0c394ee0   ti_sysbios_gates_GateMutexPri_destruct
0c394f00   ti_sysbios_gates_GateMutexPri_query__E
0c394f00   ti_sysbios_xdcruntime_GateThreadSupport_query__E
0c394f00   xdc_runtime_knl_GateThread_Proxy_query__E
0c394f00   xdc_runtime_knl_GateThread_query__E
0c394f20   ti_sysbios_gates_GateMutex_Instance_finalize__E
0c394f40   ti_sysbios_BIOS_RtsGateProxy_query__E
0c394f40   ti_sysbios_gates_GateMutex_query__E
0c394f40   ti_sysbios_heaps_HeapMem_Module_GateProxy_query__E
0c394f60   ti_sysbios_gates_GateSwi_Instance_init__E
0c394f80   ti_sdo_ipc_Notify_Module_GateProxy_query__E
0c394f80   ti_sysbios_gates_GateSwi_query__E
0c394fa0   ti_sysbios_hal_Hwi_HwiProxy_Module__startupDone__S
0c394fc0   ti_sysbios_hal_Hwi_Module_startup__E
0c394fe0   ti_sysbios_hal_Timer_Module_startup__E
0c395000   ti_sysbios_hal_Timer_TimerProxy_Module__startupDone__S
0c395020   ti_sysbios_heaps_HeapMem_Module_GateProxy_enter__E
0c395040   ti_sysbios_heaps_HeapMem_Module_GateProxy_leave__E
0c395060   ti_sysbios_heaps_HeapMem_isBlocking__E
0c395080   ti_sysbios_knl_Clock_TimerProxy_Module__startupDone__S
0c3950a0   ti_sysbios_knl_Clock_TimerProxy_getMaxTicks__E
0c3950c0   ti_sysbios_knl_Idle_loop__E
0c3950e0   ti_sysbios_knl_Queue_Instance_init__E
0c395100   ti_sysbios_knl_Queue_Object__destruct__S
0c395120   ti_sysbios_knl_Queue_Object__get__S
0c395140   ti_sysbios_knl_Queue_destruct
0c395160   ti_sysbios_knl_Queue_empty__E
0c395180   ti_sysbios_knl_Semaphore_Instance_finalize__E
0c3951a0   ti_sysbios_knl_Semaphore_destruct
0c3951c0   ti_sysbios_knl_Swi_disable__E
0c3951e0   ti_sysbios_knl_Task_SupportProxy_Module__startupDone__S
0c395200   ti_sysbios_knl_Task_disable__E
0c395220   ti_sysbios_knl_Task_getHookContext__E
0c395240   ti_sysbios_knl_Task_startup__E
0c395260   ti_sysbios_timers_timer64_Timer_getMaxTicks__E
0c395280   ti_sysbios_utils_Load_taskRegHook__E
0c3952a0   ti_sysbios_xdcruntime_GateThreadSupport_Instance_finalize__E
0c3952c0   ti_sysbios_xdcruntime_GateThreadSupport_enter__E
0c3952e0   ti_uia_loggers_LoggerStopMode_getContents__E
0c395300   ti_uia_loggers_LoggerStopMode_getFilterLevel__E
0c395320   ti_uia_loggers_LoggerStopMode_getInstanceId__E
0c395340   ti_uia_loggers_LoggerStopMode_getMaxLength__E
0c395360   ti_uia_loggers_LoggerStopMode_getPriority__E
0c395380   ti_uia_loggers_LoggerStopMode_getTransferType__E
0c3953a0   ti_uia_loggers_LoggerStopMode_isEmpty__E
0c3953c0   ti_uia_loggers_LoggerStopMode_setFilterLevel__E
0c3953e0   ti_uia_loggers_LoggerStopMode_setPriority__E
0c395400   xdc_runtime_Error_getSite__E
0c395420   xdc_runtime_Error_raiseX__E
0c395440   xdc_runtime_GateNull_enter__E
0c395460   xdc_runtime_GateNull_leave__E
0c395480   xdc_runtime_GateNull_query__E
0c3954a0   xdc_runtime_Gate_enterSystem__E
0c3954c0   xdc_runtime_Gate_leaveSystem__E
0c395520   xdc_runtime_Memory_HeapProxy_alloc__E
0c395540   xdc_runtime_Memory_HeapProxy_free__E
0c395560   xdc_runtime_Memory_calloc__E
0c395580   xdc_runtime_Memory_getMaxDefaultTypeAlign__E
0c3955a0   xdc_runtime_Startup_Module__startupDone__S
0c3955c0   xdc_runtime_Startup_exec__I
0c3955e0   xdc_runtime_Startup_rtsDone__E
0c395600   xdc_runtime_SysStd_exit__E
0c395600   xdc_runtime_System_SupportProxy_exit__E
0c395620   xdc_runtime_SysStd_putch__E
0c395620   xdc_runtime_System_SupportProxy_putch__E
0c395640   xdc_runtime_SysStd_ready__E
0c395640   xdc_runtime_System_SupportProxy_ready__E
0c395660   xdc_runtime_System_Module_GateProxy_enter__E
0c395680   xdc_runtime_System_Module_GateProxy_leave__E
0c3956a0   xdc_runtime_System_Module_startup__E
0c3956c0   xdc_runtime_System_aprintf_va__E
0c3956c0   xdc_runtime_System_aprintf_va__F
0c3956e0   xdc_runtime_System_printf_va__E
0c3956e0   xdc_runtime_System_printf_va__F
0c395700   xdc_runtime_System_vsnprintf__E
0c395720   xdc_runtime_Text_visitRope__I
0c395740   xdc_runtime_knl_GateThread_Module__startupDone__S
0c395760   xdc_runtime_knl_GateThread_Proxy_Object__create__S
0c395780   xdc_runtime_knl_GateThread_Proxy_Object__delete__S
0c3957a0   xdc_runtime_knl_GateThread_Proxy_create
0c3957c0   xdc_runtime_knl_GateThread_Proxy_delete
0c3957e0   xdc_runtime_knl_GateThread_Proxy_enter__E
0c395800   xdc_runtime_knl_GateThread_Proxy_leave__E
0c395820   xdc_runtime_knl_GateThread_enter__E
0c395840   xdc_runtime_knl_GateThread_leave__E
0c395c00   ti_sysbios_family_c64p_Hwi0
0c395c00   ti_sysbios_family_c64p_Hwi_int0
0c395c20   ti_sysbios_family_c64p_Hwi_int1
0c395c40   ti_sysbios_family_c64p_Hwi_int2
0c395c60   ti_sysbios_family_c64p_Hwi_int3
0c395c80   ti_sysbios_family_c64p_Hwi_int4
0c395ca0   ti_sysbios_family_c64p_Hwi_int5
0c395cc0   ti_sysbios_family_c64p_Hwi_int6
0c395ce0   ti_sysbios_family_c64p_Hwi_int7
0c395d00   ti_sysbios_family_c64p_Hwi_int8
0c395d20   ti_sysbios_family_c64p_Hwi_int9
0c395d40   ti_sysbios_family_c64p_Hwi_int10
0c395d60   ti_sysbios_family_c64p_Hwi_int11
0c395d80   ti_sysbios_family_c64p_Hwi_int12
0c395da0   ti_sysbios_family_c64p_Hwi_int13
0c395dc0   ti_sysbios_family_c64p_Hwi_int14
0c395de0   ti_sysbios_family_c64p_Hwi_int15
8f000000   xdc_runtime_Text_charTab__A
8f0033fb   ti_sysbios_timers_timer64_Timer_localTimerBaseId__C
8f003d00   ti_sysbios_family_c66_Cache_marvalues__C
8f004100   xdc_runtime_Text_nodeTab__A
8f0042c8   ti_sysbios_family_c66_tci66xx_CpIntc_sysIntToHostInt__A
8f004408   _ctypes_
8f00450a   ti_sdo_ipc_Notify_Module__id__C
8f00460c   ti_uia_loggers_LoggerStopMode_Module__FXNS__C
8f0046c4   ti_sdo_ipc_Ipc_A_nullArgument__C
8f0046c8   xdc_runtime_Startup_sfxnTab__A
8f004754   xdc_runtime_LoggerBuf_Module__FXNS__C
8f004790   ti_uia_loggers_LoggerStopMode_Object__PARAMS__C
8f0047ec   ti_sysbios_heaps_HeapMem_Module__FXNS__C
8f004814   xdc_runtime_LoggerBuf_Object__PARAMS__C
8f00483c   ti_sdo_ipc_MessageQ_Object__count__C
8f004840   xdc_runtime_Startup_sfxnRts__A
8f004866   ti_sdo_ipc_Notify_numLines__C
8f004868   ti_sysbios_gates_GateAll_Module__FXNS__C
8f00488c   ti_sysbios_gates_GateHwi_Module__FXNS__C
8f0048b0   ti_sysbios_gates_GateMutexPri_Module__FXNS__C
8f0048d4   ti_sysbios_gates_GateMutex_Module__FXNS__C
8f0048f8   ti_sysbios_gates_GateSwi_Module__FXNS__C
8f00491c   ti_sysbios_heaps_HeapMem_Object__PARAMS__C
8f004940   ti_sysbios_knl_Semaphore_Object__PARAMS__C
8f004964   xdc_runtime_GateNull_Module__FXNS__C
8f004988   xdc_runtime_knl_GateThread_Module__FXNS__C
8f0049d0   ti_sdo_ipc_Notify_Object__DESC__C
8f0049f0   ti_sdo_utils_List_Object__DESC__C
8f004a10   ti_sdo_utils_MultiProc_nameList__A
8f004a30   ti_sysbios_gates_GateAll_Object__DESC__C
8f004a50   ti_sysbios_gates_GateHwi_Object__DESC__C
8f004a70   ti_sysbios_gates_GateMutexPri_Object__DESC__C
8f004a90   ti_sysbios_gates_GateMutex_Object__DESC__C
8f004ab0   ti_sysbios_gates_GateSwi_Object__DESC__C
8f004ad0   ti_sysbios_heaps_HeapMem_Object__DESC__C
8f004af0   ti_sysbios_knl_Queue_Object__DESC__C
8f004b10   ti_sysbios_knl_Semaphore_Object__DESC__C
8f004b30   ti_sysbios_xdcruntime_GateThreadSupport_Object__DESC__C
8f004b50   ti_uia_loggers_LoggerStopMode_Object__DESC__C
8f004b70   xdc_runtime_GateNull_Object__DESC__C
8f004b90   xdc_runtime_LoggerBuf_Object__DESC__C
8f004bb0   xdc_runtime_knl_GateThread_Object__DESC__C
8f004bd0   ti_sdo_ipc_Notify_Object__PARAMS__C
8f004be8   ti_sdo_utils_List_Object__PARAMS__C
8f004c00   ti_sysbios_gates_GateAll_Object__PARAMS__C
8f004c18   ti_sysbios_gates_GateHwi_Object__PARAMS__C
8f004c30   ti_sysbios_gates_GateMutexPri_Object__PARAMS__C
8f004c48   ti_sysbios_gates_GateMutex_Object__PARAMS__C
8f004c60   ti_sysbios_gates_GateSwi_Object__PARAMS__C
8f004c78   ti_sysbios_knl_Queue_Object__PARAMS__C
8f004c90   ti_sysbios_knl_Swi_hooks__A
8f004ca8   ti_sysbios_knl_Task_hooks__A
8f004cc0   ti_sysbios_xdcruntime_GateThreadSupport_Object__PARAMS__C
8f004cd8   xdc_runtime_GateNull_Object__PARAMS__C
8f004cf0   xdc_runtime_knl_GateThread_Object__PARAMS__C
8f004d1c   ti_sdo_ipc_Notify_A_alreadyRegistered__C
8f004d20   ti_sysbios_family_c64p_Hwi_hooks__A
8f004d34   ti_sdo_ipc_Notify_A_invArgument__C
8f004d4a   ti_sdo_ipc_SharedRegion_Module__id__C
8f004d4c   ti_sdo_ipc_Notify_Module__diagsEnabled__C
8f004d50   ti_sdo_ipc_family_c647x_MultiProcSetup_procMap__A
8f004d60   xdc_runtime_Startup_firstFxns__A
8f004d78   ti_sysbios_family_c64p_Hwi_hooks__C
8f004d80   ti_sysbios_knl_Idle_funcList__A
8f004d88   ti_sysbios_knl_Idle_funcList__C
8f004d90   ti_sysbios_knl_Swi_hooks__C
8f004d98   ti_sysbios_knl_Task_hooks__C
8f004da0   xdc_runtime_Startup_firstFxns__C
8f004da8   xdc_runtime_Startup_lastFxns__C
8f004db0   ti_sdo_ipc_Notify_Module__diagsIncluded__C
8f004db4   ti_sdo_ipc_Notify_Module__diagsMask__C
8f004db8   ti_sdo_ipc_Notify_Object__heap__C
8f004dbc   ti_sdo_ipc_Notify_numEvents__C
8f004dc0   ti_sdo_ipc_SharedRegion_A_idTooLarge__C
8f004dc4   ti_sdo_ipc_SharedRegion_Module__diagsEnabled__C
8f004dc8   ti_sdo_ipc_SharedRegion_Module__diagsIncluded__C
8f004dcc   ti_sdo_ipc_SharedRegion_Module__diagsMask__C
8f004dd0   ti_sdo_ipc_family_c647x_Interrupt_KICK0__C
8f004dd4   ti_sdo_ipc_family_c647x_Interrupt_KICK1__C
8f004dd8   ti_sdo_ipc_family_c647x_MultiProcSetup_A_invalidProcessor__C
8f004ddc   ti_sdo_ipc_family_c647x_MultiProcSetup_Module__diagsEnabled__C
8f004de0   ti_sdo_ipc_family_c647x_MultiProcSetup_Module__diagsIncluded__C
8f004de4   ti_sdo_ipc_family_c647x_MultiProcSetup_Module__diagsMask__C
8f004de8   ti_sdo_ipc_family_c647x_MultiProcSetup_procMap__C
8f004dec   ti_sdo_ipc_gates_GateHWSem_baseAddr__C
8f004df0   ti_sdo_ipc_gates_GateHWSem_numSems__C
8f004df4   ti_sdo_ipc_gates_GateHWSem_reservedMaskArr__C
8f004df8   ti_sdo_ipc_gates_GateHWSem_reservedMaskArr__A
8f004dfc   ti_sdo_utils_MultiProc_A_invalidMultiProcId__C
8f004e00   ti_sdo_utils_MultiProc_A_invalidProcName__C
8f004e04   ti_sdo_utils_MultiProc_Module__diagsEnabled__C
8f004e08   ti_sdo_utils_MultiProc_Module__diagsIncluded__C
8f004e0c   ti_sdo_utils_MultiProc_Module__diagsMask__C
8f004e10   ti_sdo_utils_MultiProc_nameList__C
8f004e14   ti_sdo_utils_NameServer_Instance_State_freeList__O
8f004e18   ti_sdo_utils_NameServer_Object__count__C
8f004e1c   ti_sysbios_family_c64p_Exception_E_exceptionMax__C
8f004e20   ti_sysbios_family_c64p_Exception_exceptionHook__C
8f004e24   ti_sysbios_family_c64p_Exception_externalHook__C
8f004e28   ti_sysbios_family_c64p_Exception_internalHook__C
8f004e2c   ti_sysbios_family_c64p_Exception_nmiHook__C
8f004e30   ti_sysbios_family_c64p_Hwi_LD_end__C
8f004e34   ti_sysbios_family_c64p_Hwi_LM_begin__C
8f004e38   ti_sysbios_family_c64p_Hwi_Module__diagsEnabled__C
8f004e3c   ti_sysbios_family_c64p_Hwi_Module__diagsIncluded__C
8f004e40   ti_sysbios_family_c64p_Hwi_Module__diagsMask__C
8f004e44   ti_sysbios_family_c64p_Hwi_Module__loggerFxn1__C
8f004e48   ti_sysbios_family_c64p_Hwi_Module__loggerFxn8__C
8f004e4c   ti_sysbios_family_c64p_Hwi_Module__loggerObj__C
8f004e50   ti_sysbios_family_c66_Cache_E_invalidL1CacheSize__C
8f004e54   ti_sysbios_family_c66_Cache_E_invalidL2CacheSize__C
8f004e58   ti_sysbios_family_c66_Cache_atomicBlockSize__C
8f004e5c   ti_sysbios_family_c66_tci66xx_CpIntc_E_unpluggedSysInt__C
8f004e60   ti_sysbios_family_c66_tci66xx_CpIntc_numStatusRegs__C
8f004e64   ti_sysbios_family_c66_tci66xx_CpIntc_numSysInts__C
8f004e68   ti_sysbios_family_c66_tci66xx_CpIntc_sysIntToHostInt__C
8f004e6c   ti_sysbios_gates_GateMutexPri_A_badContext__C
8f004e70   ti_sysbios_gates_GateMutexPri_A_enterTaskDisabled__C
8f004e74   ti_sysbios_gates_GateMutexPri_Instance_State_pendQ__O
8f004e78   ti_sysbios_gates_GateMutexPri_Module__diagsEnabled__C
8f004e7c   ti_sysbios_gates_GateMutexPri_Module__diagsIncluded__C
8f004e80   ti_sysbios_gates_GateMutexPri_Module__diagsMask__C
8f004e84   ti_sysbios_gates_GateMutex_A_badContext__C
8f004e88   ti_sysbios_gates_GateMutex_Instance_State_sem__O
8f004e8c   ti_sysbios_gates_GateMutex_Module__diagsEnabled__C
8f004e90   ti_sysbios_gates_GateMutex_Module__diagsIncluded__C
8f004e94   ti_sysbios_gates_GateMutex_Module__diagsMask__C
8f004e98   ti_sysbios_gates_GateSwi_A_badContext__C
8f004e9c   ti_sysbios_gates_GateSwi_Module__diagsEnabled__C
8f004ea0   ti_sysbios_gates_GateSwi_Module__diagsIncluded__C
8f004ea4   ti_sysbios_gates_GateSwi_Module__diagsMask__C
8f004ea8   ti_sysbios_hal_Hwi_E_stackOverflow__C
8f004eac   ti_sysbios_heaps_HeapMem_A_align__C
8f004eb0   ti_sysbios_heaps_HeapMem_A_heapSize__C
8f004eb4   ti_sysbios_heaps_HeapMem_A_invalidFree__C
8f004eb8   ti_sysbios_heaps_HeapMem_A_zeroBlock__C
8f004ebc   ti_sysbios_heaps_HeapMem_E_memory__C
8f004ec0   ti_sysbios_heaps_HeapMem_Module__diagsEnabled__C
8f004ec4   ti_sysbios_heaps_HeapMem_Module__diagsIncluded__C
8f004ec8   ti_sysbios_heaps_HeapMem_Module__diagsMask__C
8f004ecc   ti_sysbios_heaps_HeapMem_Module__gateObj__C
8f004ed0   ti_sysbios_heaps_HeapMem_Object__count__C
8f004ed4   ti_sysbios_heaps_HeapMem_reqAlign__C
8f004ed8   ti_sysbios_knl_Clock_LM_begin__C
8f004edc   ti_sysbios_knl_Clock_LM_tick__C
8f004ee0   ti_sysbios_knl_Clock_LW_delayed__C
8f004ee4   ti_sysbios_knl_Clock_Module_State_clockQ__O
8f004ee8   ti_sysbios_knl_Clock_Module__diagsEnabled__C
8f004eec   ti_sysbios_knl_Clock_Module__diagsIncluded__C
8f004ef0   ti_sysbios_knl_Clock_Module__diagsMask__C
8f004ef4   ti_sysbios_knl_Clock_Module__loggerFxn1__C
8f004ef8   ti_sysbios_knl_Clock_Module__loggerFxn2__C
8f004efc   ti_sysbios_knl_Clock_Module__loggerObj__C
8f004f00   ti_sysbios_knl_Semaphore_A_badContext__C
8f004f04   ti_sysbios_knl_Semaphore_A_noEvents__C
8f004f08   ti_sysbios_knl_Semaphore_A_overflow__C
8f004f0c   ti_sysbios_knl_Semaphore_A_pendTaskDisabled__C
8f004f10   ti_sysbios_knl_Semaphore_Instance_State_pendQ__O
8f004f14   ti_sysbios_knl_Semaphore_LM_pend__C
8f004f18   ti_sysbios_knl_Semaphore_LM_post__C
8f004f1c   ti_sysbios_knl_Semaphore_Module__diagsEnabled__C
8f004f20   ti_sysbios_knl_Semaphore_Module__diagsIncluded__C
8f004f24   ti_sysbios_knl_Semaphore_Module__diagsMask__C
8f004f28   ti_sysbios_knl_Semaphore_Module__loggerFxn2__C
8f004f2c   ti_sysbios_knl_Semaphore_Module__loggerFxn4__C
8f004f30   ti_sysbios_knl_Semaphore_Module__loggerObj__C
8f004f34   ti_sysbios_knl_Swi_LD_end__C
8f004f38   ti_sysbios_knl_Swi_LM_begin__C
8f004f3c   ti_sysbios_knl_Swi_LM_post__C
8f004f40   ti_sysbios_knl_Swi_Module__diagsEnabled__C
8f004f44   ti_sysbios_knl_Swi_Module__diagsIncluded__C
8f004f48   ti_sysbios_knl_Swi_Module__diagsMask__C
8f004f4c   ti_sysbios_knl_Swi_Module__loggerFxn1__C
8f004f50   ti_sysbios_knl_Swi_Module__loggerFxn4__C
8f004f54   ti_sysbios_knl_Swi_Module__loggerObj__C
8f004f58   ti_sysbios_knl_Swi_Object__count__C
8f004f5c   ti_sysbios_knl_Swi_numConstructedSwis__C
8f004f60   ti_sysbios_knl_Task_A_badPriority__C
8f004f64   ti_sysbios_knl_Task_E_spOutOfBounds__C
8f004f68   ti_sysbios_knl_Task_E_stackOverflow__C
8f004f6c   ti_sysbios_knl_Task_LD_block__C
8f004f70   ti_sysbios_knl_Task_LD_exit__C
8f004f74   ti_sysbios_knl_Task_LD_ready__C
8f004f78   ti_sysbios_knl_Task_LM_setPri__C
8f004f7c   ti_sysbios_knl_Task_LM_switch__C
8f004f80   ti_sysbios_knl_Task_Module_State_inactiveQ__O
8f004f84   ti_sysbios_knl_Task_Module__diagsEnabled__C
8f004f88   ti_sysbios_knl_Task_Module__diagsIncluded__C
8f004f8c   ti_sysbios_knl_Task_Module__diagsMask__C
8f004f90   ti_sysbios_knl_Task_Module__loggerFxn2__C
8f004f94   ti_sysbios_knl_Task_Module__loggerFxn4__C
8f004f98   ti_sysbios_knl_Task_Module__loggerObj__C
8f004f9c   ti_sysbios_knl_Task_Object__count__C
8f004fa0   ti_sysbios_knl_Task_Object__heap__C
8f004fa4   ti_sysbios_knl_Task_allBlockedFunc__C
8f004fa8   ti_sysbios_knl_Task_numConstructedTasks__C
8f004fac   ti_sysbios_timers_timer64_Timer_A_notAvailable__C
8f004fb0   ti_sysbios_timers_timer64_Timer_E_cannotSupport__C
8f004fb4   ti_sysbios_timers_timer64_Timer_Module__diagsEnabled__C
8f004fb8   ti_sysbios_timers_timer64_Timer_Module__diagsIncluded__C
8f004fbc   ti_sysbios_timers_timer64_Timer_Module__diagsMask__C
8f004fc0   ti_sysbios_timers_timer64_Timer_anyMaskHigh__C
8f004fc4   ti_sysbios_timers_timer64_Timer_anyMask__C
8f004fc8   ti_sysbios_timers_timer64_Timer_freqDivisor__C
8f004fcc   ti_sysbios_timers_timer64_Timer_numLocalTimers__C
8f004fd0   ti_sysbios_timers_timer64_Timer_numTimerDevices__C
8f004fd4   ti_sysbios_utils_Load_LS_cpuLoad__C
8f004fd8   ti_sysbios_utils_Load_LS_hwiLoad__C
8f004fdc   ti_sysbios_utils_Load_LS_swiLoad__C
8f004fe0   ti_sysbios_utils_Load_LS_taskLoad__C
8f004fe4   ti_sysbios_utils_Load_Module_State_taskList__O
8f004fe8   ti_sysbios_utils_Load_Module__diagsEnabled__C
8f004fec   ti_sysbios_utils_Load_Module__diagsIncluded__C
8f004ff0   ti_sysbios_utils_Load_Module__diagsMask__C
8f004ff4   ti_sysbios_utils_Load_Module__loggerFxn1__C
8f004ff8   ti_sysbios_utils_Load_Module__loggerFxn2__C
8f004ffc   ti_sysbios_utils_Load_Module__loggerFxn4__C
8f005000   ti_sysbios_utils_Load_Module__loggerObj__C
8f005004   ti_sysbios_utils_Load_postUpdate__C
8f005008   ti_sysbios_utils_Load_windowInMs__C
8f00500c   ti_sysbios_xdcruntime_GateThreadSupport_Instance_State_gate__O
8f005010   ti_uia_loggers_LoggerStopMode_Module__diagsEnabled__C
8f005014   ti_uia_loggers_LoggerStopMode_Module__diagsIncluded__C
8f005018   ti_uia_loggers_LoggerStopMode_Module__diagsMask__C
8f00501c   ti_uia_loggers_LoggerStopMode_Object__count__C
8f005020   ti_uia_loggers_LoggerStopMode_numCores__C
8f005024   ti_uia_runtime_ILoggerSnapshot_Interface__BASE__C
8f005028   ti_uia_runtime_IUIATransfer_Interface__BASE__C
8f00502c   xdc_runtime_Assert_E_assertFailed__C
8f005030   xdc_runtime_Core_A_initializedParams__C
8f005034   xdc_runtime_Core_Module__diagsEnabled__C
8f005038   xdc_runtime_Core_Module__diagsIncluded__C
8f00503c   xdc_runtime_Core_Module__diagsMask__C
8f005040   xdc_runtime_Error_E_memory__C
8f005044   xdc_runtime_Error_Module__diagsEnabled__C
8f005048   xdc_runtime_Error_Module__diagsIncluded__C
8f00504c   xdc_runtime_Error_Module__diagsMask__C
8f005050   xdc_runtime_Error_Module__loggerFxn8__C
8f005054   xdc_runtime_Error_Module__loggerObj__C
8f005058   xdc_runtime_Error_policyFxn__C
8f00505c   xdc_runtime_Error_policy__C
8f005060   xdc_runtime_Error_raiseHook__C
8f005064   xdc_runtime_IFilterLogger_Interface__BASE__C
8f005068   xdc_runtime_IGateProvider_Interface__BASE__C
8f00506c   xdc_runtime_IHeap_Interface__BASE__C
8f005070   xdc_runtime_ILogger_Interface__BASE__C
8f005074   xdc_runtime_IModule_Interface__BASE__C
8f005078   xdc_runtime_Log_L_error__C
8f00507c   xdc_runtime_LoggerBuf_E_badLevel__C
8f005080   xdc_runtime_LoggerBuf_Module__gateObj__C
8f005084   xdc_runtime_LoggerBuf_Object__count__C
8f005088   xdc_runtime_LoggerBuf_statusLogger__C
8f00508c   xdc_runtime_Memory_defaultHeapInstance__C
8f005090   xdc_runtime_Startup_execImpl__C
8f005094   xdc_runtime_Startup_maxPasses__C
8f005098   xdc_runtime_Startup_sfxnRts__C
8f00509c   xdc_runtime_Startup_sfxnTab__C
8f0050a0   xdc_runtime_System_Module__gateObj__C
8f0050a4   xdc_runtime_System_abortFxn__C
8f0050a8   xdc_runtime_System_exitFxn__C
8f0050ac   xdc_runtime_System_extendFxn__C
8f0050b0   xdc_runtime_System_maxAtexitHandlers__C
8f0050b4   xdc_runtime_Text_charTab__C
8f0050b8   xdc_runtime_Text_nameEmpty__C
8f0050bc   xdc_runtime_Text_nameStatic__C
8f0050c0   xdc_runtime_Text_nameUnknown__C
8f0050c4   xdc_runtime_Text_nodeTab__C
8f0050c8   xdc_runtime_Text_visitRopeFxn__C
8f0050cc   ti_sdo_ipc_SharedRegion_numEntries__C
8f0050ce   ti_sdo_ipc_family_c647x_Interrupt_enableKick__C
8f0050d0   ti_sdo_ipc_family_c647x_MultiProcSetup_Module__id__C
8f0050d2   ti_sdo_utils_MultiProc_Module__id__C
8f0050d4   ti_sdo_utils_MultiProc_numProcessors__C
8f0050d6   ti_sdo_utils_MultiProc_numProcsInCluster__C
8f0050d8   ti_sysbios_family_c64p_Exception_Module__id__C
8f0050da   ti_sysbios_family_c64p_Exception_useInternalBuffer__C
8f0050dc   ti_sysbios_family_c64p_Hwi_Module__id__C
8f0050de   ti_sysbios_family_c64p_Hwi_Module__loggerDefined__C
8f0050e0   ti_sysbios_family_c66_Cache_Module__id__C
8f0050e2   ti_sysbios_family_c66_Cache_registerRTSSynch__C
8f0050e4   ti_sysbios_family_c66_tci66xx_CpIntc_Module__id__C
8f0050e6   ti_sysbios_gates_GateMutexPri_Module__id__C
8f0050e8   ti_sysbios_gates_GateMutex_Module__id__C
8f0050ea   ti_sysbios_gates_GateSwi_Module__id__C
8f0050ec   ti_sysbios_hal_Hwi_Module__id__C
8f0050ee   ti_sysbios_heaps_HeapMem_Module__id__C
8f0050f0   ti_sysbios_knl_Clock_Module__id__C
8f0050f2   ti_sysbios_knl_Clock_Module__loggerDefined__C
8f0050f4   ti_sysbios_knl_Semaphore_Module__id__C
8f0050f6   ti_sysbios_knl_Semaphore_Module__loggerDefined__C
8f0050f8   ti_sysbios_knl_Swi_Module__id__C
8f0050fa   ti_sysbios_knl_Swi_Module__loggerDefined__C
8f0050fc   ti_sysbios_knl_Task_Module__id__C
8f0050fe   ti_sysbios_knl_Task_Module__loggerDefined__C
8f005100   ti_sysbios_timers_timer64_Timer_Module__id__C
8f005102   ti_sysbios_timers_timer64_Timer_startupNeeded__C
8f005104   ti_sysbios_timers_timer64_Timer_useTimer64pRegMap__C
8f005106   ti_sysbios_utils_Load_Module__id__C
8f005108   ti_sysbios_utils_Load_Module__loggerDefined__C
8f00510a   ti_sysbios_utils_Load_autoAddTasks__C
8f00510c   ti_sysbios_utils_Load_updateInIdle__C
8f00510e   ti_uia_loggers_LoggerStopMode_Module__id__C
8f005110   ti_uia_loggers_LoggerStopMode_isTimestampEnabled__C
8f005112   xdc_runtime_Core_Module__id__C
8f005114   xdc_runtime_Error_Module__loggerDefined__C
8f005116   xdc_runtime_Error_maxDepth__C
8f005118   xdc_runtime_LoggerBuf_Module__id__C
8f00511a   xdc_runtime_LoggerBuf_filterByLevel__C
8f00511c   xdc_runtime_Memory_Module__id__C
8f00511e   xdc_runtime_Text_charCnt__C
8f005120   xdc_runtime_Text_isLoaded__C
8f005122   xdc_runtime_Text_registryModsLastId__C
8f005124   xdc_runtime_Text_unnamedModsLastId__C
8f005140   xdc_runtime_LoggerBuf_write8__E
8f0053c0   xdc_runtime_LoggerBuf_write4__E
8f005580   xdc_runtime_LoggerBuf_setFilterLevel__E
8f0056a0   xdc_runtime_LoggerBuf_getFilterLevel__E
8f0057a0   xdc_runtime_LoggerBuf_Object__create__S
8f005880   xdc_runtime_LoggerBuf_Instance_init__E
8f005900   xdc_runtime_LoggerBuf_Module_startup__E
8f005980   xdc_runtime_LoggerBuf_filterOutEvent__I
8f005a00   xdc_runtime_LoggerBuf_Object__delete__S
8f005a60   xdc_runtime_LoggerBuf_Handle__label__S
8f005aa0   xdc_runtime_LoggerBuf_Instance_finalize__E
8f005ae0   xdc_runtime_LoggerBuf_Object__get__S
8f005b20   xdc_runtime_LoggerBuf_reset__E
8f005b60   xdc_runtime_LoggerBuf_write0__E
8f005ba0   xdc_runtime_LoggerBuf_Module_GateProxy_enter__E
8f005bc0   xdc_runtime_LoggerBuf_Module_GateProxy_leave__E
8f005be0   xdc_runtime_LoggerBuf_disable__E
8f005c00   xdc_runtime_LoggerBuf_enable__E
8f005c20   xdc_runtime_LoggerBuf_write1__E
8f005c40   xdc_runtime_LoggerBuf_write2__E
8f006000   _c_int00
8f007310   __TI_Handler_Table_Base
8f007318   __TI_CINIT_Base
8f007318   __TI_Handler_Table_Limit
8f007328   __TI_CINIT_Limit
903c0000   ti_sysbios_heaps_HeapMem_Instance_State_0_buf__A
97160000   ti_sysbios_heaps_HeapMem_Instance_State_1_buf__A
9df00000   ti_sysbios_heaps_HeapMem_Instance_State_2_buf__A
9ef00000   ti_sysbios_heaps_HeapMem_Instance_State_3_buf__A
9ff00000   ti_sysbios_heaps_HeapMem_Instance_State_4_buf__A
9ff80000   ti_sysbios_heaps_HeapMem_Instance_State_5_buf__A
ffffffff   __TI_pprof_out_hndl
ffffffff   __TI_prof_data_size
ffffffff   __TI_prof_data_start
ffffffff   __binit__
ffffffff   __c_args__
ffffffff   binit
UNDEFED    __TI_INITARRAY_Base
UNDEFED    __TI_INITARRAY_Limit
UNDEFED    __TI_TLS_INIT_Base
UNDEFED    __TI_TLS_INIT_Limit

[962 symbols]
